:100000000C940F170C9448170C9448170C9448172D
:100010000C94F4400C94F4400C94F4400C94F44090
:100020000C9448170C9448170C9448170C944817D4
:100030000C9448170C94742A0C9448170C94481785
:100040000C9448170C94C0260C94EBCB0C944817D6
:100050000C94E5880C94DB880C9448170C94481792
:100060000C9448170C9448170C9448170C94481794
:100070000C9448170C9448170C9448170C94481784
:100080000C9448170C9448170C9448174E414E494D
:100090004E495459494E46CDCCCC3D0AD7233C1746
:1000A000B7D13877CC2B329595E6241FB14F0A0093
:1000B0000020410000C84200401C4620BCBE4CCA83
:1000C0001B0E5AAEC59D7400407A10F35A00A07200
:1000D0004E18090010A5D4E80000E8764817000083
:1000E000E40B54020000CA9A3B000000E1F5050051
:1000F0000080969800000040420F000000A086019A
:10010000000000102700000000E803000000006469
:1001100000000000000A00000000000100000000D4
:10012000002C76D888DC674F0823DFC1DFAE59E1A9
:10013000B1B796E5E3E453C63AE651997696E8E618
:10014000C28426EB898C9B62ED407C6FFCEFBC9CEB
:100150009F40F2BAA56FA5F490055A2AF75C936BFD
:100160006CF9676DC11BFCE0E40D47FEF520E6B5B8
:1001700000D0ED902E0300943577050080841E0892
:100180000000204E0A000000C80C333333330F98B0
:100190006E12831141EF8D2114893BE65516CFFE77
:1001A000E6DB18D1844B381BF77C1D901DA4BBE403
:1001B00024203284725E228100C9F124ECA1E53D45
:1001C000275045544700504C41005072696E7420CE
:1001D00041626F72746564004D3235005061757311
:1001E000696E672E2E2E004D323400454550524F19
:1001F0004D2056657273696F6E204572726F720082
:10020000454550524F4D20496E64657820457272C5
:100210006F7200454550524F4D2043524320457266
:10022000726F72003F0049676E6F726500526573AE
:10023000657400496E697469616C697A6520454529
:1002400050524F4D0000FE0003FF8007C7C007015A
:10025000E00000E00000F00000700400700E00708C
:100260001F00703F80F00E00E00F01E007C7C003E1
:10027000FF8000FE0000FE0003FF8007C7C00F01E3
:10028000E00E00E03F80F01F00700E007004007070
:100290000000700000F00000E00701E007C7C003A5
:1002A000FF8000FE000E000E000E000E000E000E7D
:1002B000000E000E007FC03F801F000E00040004EF
:1002C000000E001F003F807FC00E000E000E000ECB
:1002D000000E000E000E000E00FFFFFF7F80FFC02B
:1002E000FFC0FFC07F807F80FFC0FFC0FFC03F0016
:1002F0001E000C0050726F6265205A204F666673B4
:1003000065740020082046616374002008204D6158
:1003100078002008204D696E004F6666004F6E0021
:100320004175746F74656D700045207374657073EA
:100330002F6D6D005A2053746570732F6D6D0059C9
:100340002053746570732F6D6D0058205374657061
:10035000732F6D6D00416476616E63656420536533
:100360007474696E67730054656D7065726174753D
:1003700072650053746570732F6D6D00436F6E6608
:10038000696775726174696F6E003F004E657874BD
:1003900020436F726E657200446F6E65004E657823
:1003A0007400486F6D696E672058595A0053746F16
:1003B00072652053657474696E6773004C6F616475
:1003C0002053657474696E677300426564205472CB
:1003D000616D6D696E670050726F6265205A204FC3
:1003E0006666736574004661646520486569676880
:1003F00074004F6666004F6E00426564204C65765F
:10040000656C696E67004C6576656C2042656400BA
:100410004732394E00473239004175746F20486FBA
:100420006D65004D6F74696F6E00526573746F7205
:10043000652044656661756C7473004C6F6164205F
:1004400053657474696E67730053746F72652053DB
:10045000657474696E67730050726F6265205A200C
:100460004F666673657400416476616E63656420EF
:1004700053657474696E6773004D61696E003F0067
:100480004261636B0053746F70004D3232004174EF
:1004900074616368204D65646961004D32310050BC
:1004A00072696E742066726F6D204D6564696100BB
:1004B00052656C65617365204D6564696100436FC9
:1004C0006E66696775726174696F6E0054656D70F0
:1004D00065726174757265004D6F74696F6E00525C
:1004E0006573756D65205072696E740054756E6524
:1004F0000053746F70205072696E74005061757390
:1005000065205072696E7400496E666F2053637285
:1005100065656E000A4D3234004D3233202573007C
:100520003F005374617274205072696E74004361AD
:100530006E63656C005072696E740043616E6E6F1D
:100540007420656E746572207375626469723A20F6
:100550000002202E2E000152656672657368004D00
:1005600061696E002100486F74656E6420746F6F5E
:1005700020636F6C64004261636B0050726F63654F
:100580006564004D6F74696F6E0044697361626CDD
:1005900065205374657070657273004D3834004285
:1005A0006564204C6576656C696E67004175746F93
:1005B00020486F6D6500473238004D61696E00500C
:1005C000726568656174202420426564005072651C
:1005D00068656174202420456E640054656D706503
:1005E00072617475726500C601C101436F6F6C64FE
:1005F0006F776E00507265686561742024004661F3
:100600006E20537065656400426564004E6F7A7AAF
:100610006C65004D61696E0050726F6265205A20F2
:100620004F666673657400466C6F770046616E2096
:10063000537065656400426564004E6F7A7A6C653C
:10064000005370656564004D61696E00486F6D69A7
:100650006E67204661696C6564006F70656E00545A
:100660005249474745524544003A20007A5F70722C
:100670006F6265007A5F6D696E00795F6D696E000B
:10068000785F6D696E005265706F7274696E672075
:10069000656E6473746F70207374617475730A008F
:1006A00020746F6F206C6F6E67206578747275733D
:1006B000696F6E2070726576656E7465640A0020DD
:1006C000636F6C6420657874727573696F6E2070E7
:1006D000726576656E7465640A00486F6D652025E5
:1006E0007325732573204669727374005761726EA7
:1006F000696E673A20486F6D696E672042756D704C
:100700002044697669736F72203C20310A0002022E
:10071000040000E0C0000000C0000000000000680D
:10072000430000634300007A430000A0400000A0A3
:100730004000000040FFFDFCFAF8F6F4F2F0EEECA9
:10074000EAE9E7E5E3E1E0DEDCDAD9D7D5D4D2D0D7
:10075000CFCDCBCAC8C7C5C3C2C0BFBDBCBAB9B76D
:10076000B6B4B3B2B0AFADACAAA9A8A6A5A4A2A1D5
:10077000A09E9D9C9A99989795949392908F8E8D18
:100780008B8A8988878684838281807F7E7D7B7A3D
:10079000797877767574737271706F6E6D6C6B6A41
:1007A000696867666564636261605F5E5D5C5B5A31
:1007B0005958585756555453525150504F4E4D4C0E
:1007C0004B4A4A4948474646454443424241403FD6
:1007D0003E3E3D3C3B3B3A3938383736353534338D
:1007E00032323130302F2E2E2D2C2B2B2A29292836
:1007F000272726252524232322212120201F1E1ED2
:100800001D1C1C1B1B1A1919181817161615151460
:10081000131312121111100F0F0E0E0D0D0C0C0BE5
:100820000A0A090908080707060605050404030360
:100830000202010000000000010000000100008031
:1008400000555555000000400033333300AAAA2A52
:10085000004992240000002000C7711C00999919DA
:1008600000D1451700555515003BB113002449121E
:100870000011111100000010000F0F0F00E3380EDF
:100880000043790D00CCCC0C00C3300C00E8A20B67
:100890000064210B00AAAA0A00703D0A009DD80935
:1008A00000427B090092240900DCD30800888808F4
:1008B000001042080000000800F0C1070087870709
:1008C0000075500700711C07003EEB0600A1BC0636
:1008D000006990060066660600703E060061180614
:1008E0000017F4050074D105005BB00500B2900557
:1008F00000627205005555050078390500B81E05DF
:1009000000050505004EEC040087D40400A1BD04D9
:100910000090A7040049920400C17D0400EE690420
:1009200000C7560400444404005C3204000821045B
:100930000041100400000004003FF00300F8E00351
:100940000026D20300C3C30300CCB503003AA803BA
:10095000000A9B0300388E0300C08103009F7503CB
:1009600000D0690300505E03001D530300344803A8
:1009700000913D03003333030016290300381F03A1
:100980000097150300300C0300030303000BFA0269
:100990000049F10200BAE802005CE002002DD80232
:1009A000002DD0020059C80200B0C0020031B902C7
:1009B00000DAB10200AAAA0200A0A30200BC9C02B5
:1009C00000FA9502005C8F0200DF8802008282023A
:1009D00000457C02002776020027700200436A026D
:1009E000007C640200D05E02003F590200C853023E
:1009F0000053746F77205A2D50726F626500446502
:100A0000706C6F79205A2D50726F62650000006122
:100A1000430000614300007A430000E0C000000092
:100A2000C00000000053657474696E6773205374CE
:100A30006F726564000000FA430000FA430000A0F2
:100A4000400000C8410000A0420000A0420000C8D1
:100A5000430080C043F4010000F401000064000082
:100A6000008813000024F4D43050C38E20C2A2406A
:100A700017828B7011127A910D816CD90AA861E1ED
:100A800008C7586607615143061E4B5D05C145A75F
:100A9000041A411104093D9803713931034036DBD2
:100AA0000265339102D4305402802E1D02632CEE75
:100AB00001752AC501B028A001102781018F256486
:100AC000012B244B01E0223401AC211F018D200DAC
:100AD00001801FFC00841EED00971DDF00B81CD2B2
:100AE00000E61BC600201BBC00641AB200B219A8A5
:100AF000000A19A0006A189900D117910040178BBD
:100B000000B516840031167E00B31579003A1573CE
:100B100000C7146F0058146A00EE13660088136350
:100B20000025135E00C7125B006C125700151254AB
:100B300000C111510070114F0021114B00D6104916
:100B4000008D1047004610440002104200C00F40C4
:100B500000800F3E00420F3C00060F3B00CB0E38DA
:100B600000930E37005C0E3500270E3400F30D3273
:100B700000C10D3100900D3000600D2E00320D2DA2
:100B800000050D2C00D90C2B00AE0C2900850C297A
:100B9000005C0C2700350C27000E0C2600E80B2407
:100BA00000C40B2400A00B23007D0B23005A0B2153
:100BB00000390B2100180B2000F80A1F00D90A1E6B
:100BC00000BB0A1E009D0A1D00800A1D00630A1C4E
:100BD00000470A1B002C0A1B00110A1A00F7091A09
:100BE00000DD091900C4091900AB091900920917A1
:100BF000007B091800630917004C09160036091616
:100C000000200916000A091500F5081500E008146F
:100C100000CC081400B8081400A4081400900813AD
:100C2000007D0812006B08130058081200460812D5
:100C300000340811002308110012081100010811E6
:100C400000F0071000E0071000D0071000C00710E8
:100C500000B0070F00A107100091070E0083070FD7
:100C60000074070F0065070E0057070E0049070EB6
:100C7000003B070D002E070E0020070D0013070D87
:100C80000006070D00F9060C00ED060D00E0060C4D
:100C900000D4060C00C8060C00BC060C00B0060C04
:100CA00000A4060B0099060C008D060B0082060BB3
:100CB0000077060B006C060B0061060A0057060B56
:100CC000004C060A0042060A0038060A002E060AF0
:100CD0000024060A001A060A001006090007060A80
:100CE00000FD050900F4050900EB050900E205090E
:100CF00000D9050900D0050900C7050900BE05098E
:100D000000B5050800AD050800A50509009C05080B
:100D100000940508008C050800840508007C05087F
:100D200000740508006C050700650508005D0507EF
:100D300000560508004E0507004705070040050856
:100D40000038050700310507002A050700230507BD
:100D5000001C050600160507000F0507000805061C
:100D60000002050700FB040600F5040700EE040678
:100D700000E8040600E2040700DB040600D50406D0
:100D800000CF040600C9040600C3040600BD040623
:100D900000B7040600B1040500AC040600A6040672
:100DA00000A00405009B04060095040500900406BD
:100DB000008A04050085040500800406007A040505
:100DC0000075040500700405006B04050066040549
:100DD00000610405005C0405005704050052040589
:100DE000004D04050048040500430405003E0404CA
:100DF000003A04050035040500300404002C040505
:100E00000027040400230405001E0404001A04043F
:100E10000016040500110404000D04040009040573
:100E2000000404040000040400FC030400F80304AC
:100E300000F4030400F0030400EC030400E80304DE
:100E400000E4030400E0030400DC030400D803040E
:100E500000D4030400D0030400CC030400C803033F
:100E600000C503030024F404D9201BC40C5C0E98B5
:100E700004C4095F0265077101F405F900FB04B3BE
:100E80000048048700C10369005803550003034567
:100E900000BE023A008402310053022A00290225D2
:100EA0000004022000E4011C00C8011900AF011772
:100EB00000980114008401130071011000610110F9
:100EC0000051010E0043010D0036010B002B010BF8
:100ED0000020010B00150109000C010900030108A5
:100EE00000FB000800F3000800EB000700E4000628
:100EF00000DE000600D8000600D2000600CC000587
:100F000000C7000500C2000500BD000400B90004D0
:100F100000B5000400B1000400AD000400A9000405
:100F200000A5000300A20003009F0004009B000333
:100F30000098000300950002009300030090000356
:100F4000008D0002008B0003008800020086000272
:100F50000084000300810002007F0002007D000287
:100F6000007B000200790002007700010076000299
:100F7000007400020072000100710002006F0002A4
:100F8000006D0001006C0002006A000100690002AF
:100F900000670001006600010065000100640002B6
:100FA000006200010061000100600001005F0002BA
:100FB000005D0001005C0001005B0001005A0001BF
:100FC00000590001005800010057000100560001BF
:100FD00000550001005400010053000000530001BF
:100FE000005200010051000100500001004F0001BB
:100FF000004E0000004E0001004D0001004C0001B9
:10100000004B0000004B0001004A000100490001B4
:1010100000480000004800010047000100460000B1
:1010200000460001004500000045000100440001A9
:1010300000430000004300010042000000420001A4
:10104000004100000041000100400001003F00009D
:10105000003F0001003E0000003E0001003D000096
:10106000003D0001003C0000003C0000003C00018D
:10107000003B0000003B0001003A0000003A000184
:10108000003900000039000100380000003800007D
:101090000038000100370000003700010036000072
:1010A0000036000000360001003500000035000069
:1010B000003500010034000000340000003400015D
:1010C0000033000000330000003300010032000054
:1010D0000032000000320001003100000031000049
:1010E000003100010030000000300000003000013D
:1010F000002F0000002F0000002F0000002F000133
:10110000002E0000002E0000002E0001002D000027
:10111000002D0000002D0000002D0001002C00001B
:10112000002C0000002C0000002C0001002B00000F
:10113000002B0000002B0000002B0001002A000003
:10114000002A0000002A0000002A000100290000F7
:1011500000290000002900000029000000290001EA
:1011600000280000002800000028000000280000DF
:1011700000280001002700000027000000270000D1
:1011800000270000002700010026000000260000C4
:1011900000260000002600000026000100250000B7
:1011A00000250000002500000025000000250000AB
:1011B000002500010024000000240000002400009D
:1011C0000024000000240001002300000023000090
:1011D0000023000000230000002300000023000083
:1011E0000023000100220000002200000022000075
:1011F0000022000000220000002200010021000067
:10120000002100000021000000210000002100005A
:10121000002100000021000100200000002000004B
:10122000002000000020000000200000002000003E
:101230000020000000200001001F0000001F00002F
:10124000001F0000001F0000001F0000001F000022
:10125000001F0001001E0000001E0000001E000014
:10126000001E0000003930000033250000871900FF
:1012700000B00F0000DB080000BD04000074020095
:10128000003F01000020436F756E7420583A004201
:101290006564004531004500626564002C20737967
:1012A0007374656D2073746F707065642120486578
:1012B000617465725F49443A20004572723A204D6C
:1012C000415854454D50004D415854454D5020749F
:1012D00072696767657265640048656174696E6705
:1012E000204661696C65640048656174696E6720B9
:1012F0006661696C6564004572723A204D494E54CE
:10130000454D50004D494E54454D5020747269670B
:10131000676572656400544845524D414C205255F2
:101320004E4157415900546865726D616C20527589
:101330006E6177617900202F002042403A00204002
:101340003A007C3C3E5E2B3D3F2F5B5D3B2C2A22CE
:101350005C00434F4D4D554E49434154494F4E005B
:1013600044525952554E004552524F525300494E25
:10137000464F004543484F0053544F505045442E6C
:1013800020005072696E7465722073746F7070659E
:10139000642064756520746F206572726F72732E9D
:1013A0002046697820746865206572726F722061CA
:1013B0006E6420757365204D39393920746F207241
:1013C0006573746172742E202854656D7065726146
:1013D000747572652069732072657365742E20536D
:1013E0006574206974206166746572207265737417
:1013F000617274696E67290A004E6F2043686563E5
:101400006B73756D2077697468206C696E65206EEA
:10141000756D6265722C204C617374204C696E6529
:101420003A20004E6F20436865636B73756D2077BB
:10143000697468206C696E65206E756D6265722CCA
:10144000204C617374204C696E653A2000636865B6
:10145000636B73756D206D69736D617463682C20A7
:101460004C617374204C696E653A20004C696E655E
:10147000204E756D626572206973206E6F74204C0A
:10148000617374204C696E65204E756D6265722BB8
:10149000312C204C617374204C696E653A20004DEC
:1014A0003131300053657269616C207374617475F9
:1014B00073206D69736D617463680A005344207210
:1014C000656164206572726F720A002121204B49A8
:1014D0004C4C2063617573656420627920746F6F72
:1014E000206D75636820696E616374697665207428
:1014F000696D65202D2063757272656E7420636F4F
:101500006D6D616E643A20004D6564696120496EBD
:1015100073657274656400627573793A20706175E1
:1015200073656420666F7220696E7075740A00625C
:101530007573793A2070617573656420666F7220E7
:10154000757365720A00627573793A2070726F6301
:10155000657373696E670A00506C6561736520522C
:1015600065736574005052494E5445522048414CB1
:101570005445440025533A202553004B494C4C45D3
:10158000442E20005072696E7465722068616C741C
:1015900065642E206B696C6C28292063616C6C6516
:1015A00064210A006563686F3A004572726F723A8F
:1015B000004F4646004F4E0042696C696E6561728D
:1015C000204C6576656C696E6720477269643A0ADB
:1015D000004F46460A0046616465204865696768B1
:1015E000742000426564204C6576656C696E6720E6
:1015F000004661696C656420746F20656E61626C81
:101600006520426564204C6576656C696E670A00EA
:10161000496E76616C6964206D6573682E0A0050AE
:10162000726F62696E6720506F696E740025532077
:1016300025692F2569002E0A002F0050726F6269FC
:101640006E67206D65736820706F696E742000206E
:101650002844525952554E29004732392041757459
:101660006F20426564204C6576656C696E67003F4B
:1016700020284C2C522C462C4229206F7574206F48
:101680006620626F756E64732E0A003F28562965C6
:1016900072626F7365206C6576656C20696D706C25
:1016A00061757369626C652028302D34292E0A001B
:1016B000426164205A2076616C75650A004E6F2085
:1016C00062696C696E65617220677269640A0047BD
:1016D00032384C300020204D3230312058004D61DE
:1016E0007820416363656C65726174696F6E202850
:1016F000756E6974732F7332290020204D32303398
:101700002058004D61782066656564726174657368
:101710002028756E6974732F7329002052002020D1
:101720004D323034205000416363656C65726174E2
:10173000696F6E2028756E6974732F7332292028A3
:10174000503C7072696E742D616363656C3E20520B
:101750003C726574726163742D616363656C3E20D5
:10176000543C74726176656C2D616363656C3E29CF
:1017700000204A0020540020530020204D323035F4
:10178000204200416476616E6365642028423C6DAE
:10179000696E5F7365676D656E745F74696D655FB3
:1017A00075733E20533C6D696E5F6665656472615A
:1017B00074653E20543C6D696E5F74726176656C31
:1017C0005F66656564726174653E204A3C6A756E49
:1017D000635F6465763E2900204400204900202094
:1017E0004D333031205000486F74656E642050498D
:1017F000440020440020490020204D333034205044
:101800000042656420504944002E0A00206E6F7427
:101810002064697361626C65642E2053686172652F
:101820006420776974680020496E76616C69642071
:1018300065787472756465722000536C6565702EEE
:101840002E2E005A2050726F6265205061737420F2
:101850004265640A005A2050726F626520506173BD
:10186000742042656400205A3A200020593A200032
:1018700042656420583A20004D65736820706F6996
:101880006E74206F7574206F662072616E67650AD2
:1018900000436C69636B20746F20526573756D65CE
:1018A0002E2E2E00616C736F20656E61626C656414
:1018B000290A004E6F204D6F76652E004E6F206D09
:1018C000656469610A00456E642066696C65206C18
:1018D0006973740A00426567696E2066696C6520E9
:1018E0006C6973740A00286E6F2066696C65290044
:1018F0004E6F74205344207072696E74696E670A6B
:10190000005344207072696E74696E672062797446
:1019100065200043757272656E742066696C653A65
:1019200020002E0A0044656C6574696F6E20666144
:10193000696C65642C2046696C653A200046696CC8
:10194000652064656C657465643A002569730025DB
:10195000696D20256973002569682025696D20253A
:10196000697300256964202569682025696D202533
:101970006973002569792025696420256968202517
:10198000696D20256973005072696E742074696DE9
:10199000653A20006F6B006F66660073136E136705
:1019A000136013521344454255473A004D313132CA
:1019B0002053687574646F776E004D313133205356
:1019C000004D656761205A65726F20322E30204FBE
:1019D00046462E00434F4E4649475F4558504F52AA
:1019E00054004D4541545041434B00434F4F4C45EB
:1019F000525F54454D50455241545552450043485D
:101A0000414D4245525F54454D5045524154555207
:101A10004500424142595354455050494E470041B8
:101A2000524353004D4F54494F4E5F4D4F44455321
:101A300000544845524D414C5F50524F5445435419
:101A4000494F4E00455854454E4445445F4D323051
:101A5000004C4F4E475F46494C454E414D45004175
:101A600055544F5245504F52545F53445F53544165
:101A70005455530053445F57524954450052455002
:101A8000454154005344434152440050524F4D503D
:101A9000545F535550504F525400484F53545F4178
:101AA0004354494F4E5F434F4D4D414E44530045C3
:101AB0004D455247454E43595F50415253455200A0
:101AC000434153455F4C494748545F425249474858
:101AD000544E45535300544F47474C455F4C49477C
:101AE00048545300534F4654574152455F504F5747
:101AF0004552004255494C445F50455243454E546F
:101B0000004C4556454C494E475F44415441005AAC
:101B10005F50524F42450052554E4F55540041556B
:101B2000544F4C4556454C005052494E545F4A4F15
:101B3000420050524F4752455353004155544F5263
:101B400045504F52545F54454D50004155544F52EB
:101B500045504F52545F504F5300564F4C554D45D2
:101B60005452494300454550524F4D0042494E4161
:101B700052595F46494C455F5452414E5346455277
:101B80000053455249414C5F584F4E5F584F4646AF
:101B9000004649524D574152455F4E414D453A4DE1
:101BA00061726C696E20322E302E392E332D6B61AE
:101BB00064312028446563203237203230323120AE
:101BC00031333A34353A35382920534F555243454D
:101BD0005F434F44455F55524C3A6769746875627C
:101BE0002E636F6D2F6B61642F4D61726C696E2077
:101BF00050524F544F434F4C5F56455253494F4EEE
:101C00003A312E30204D414348494E455F5459509A
:101C1000453A4D656761205A65726F20322E30203B
:101C200045585452554445525F434F554E543A31EE
:101C300020555549443A64626663636435352D65C1
:101C40006262612D343631352D616264372D313950
:101C5000366161343338663330340A002F2F004D3B
:101C600031343520533C696E6465783E206F75745D
:101C7000206F662072616E67652028302D31290A39
:101C8000003F4A206F7574206F662072616E676531
:101C90002028302E303120746F20302E33290A0056
:101CA00020580020204D61783A2000200020204D4F
:101CB000696E3A2000203B200020204D3231312037
:101CC000530046523A0020466C6F773A200050721B
:101CD0006F6265204F6666736574205A0050726F9C
:101CE0006265204F6666736574205A0064697300EC
:101CF000656E0043290A0061626C656420286D6985
:101D00006E2074656D702000436F6C64206578747C
:101D100072756465732061726520004D3432312024
:101D2000696E636F727265637420706172616D6554
:101D30007465722075736167650A004D657368206C
:101D4000706F696E74206F7574206F662072616E9B
:101D500067650A00203B204C6576656C696E6720DC
:101D60000020204D3432302053004175746F2042E2
:101D70006564204C6576656C696E670020460020BE
:101D8000420020480020204D3134352053004D6161
:101D900074657269616C206865617475702070612A
:101DA00072616D657465727300204A0020204732AD
:101DB00039205720490020204D3134392043203B21
:101DC00020556E69747320696E2043656C73697564
:101DD000730A0054656D7065726174757265205583
:101DE0006E697473002020473231203B004C696ECD
:101DF00065617220556E69747300454550524F4DB0
:101E0000204F4B0A00290A0020746F20003F5A20FF
:101E10006F7574206F662072616E676520280029D7
:101E20000A0020746F20003F59206F7574206F6680
:101E30002072616E676520282D00290A0020746FCA
:101E400020003F58206F7574206F662072616E67A6
:101E50006520282D004D383400446F6E6520707267
:101E6000696E74696E672066696C650A004D373764
:101E7000004D333100496E76616C69642065787479
:101E800072756465720A004361703A0020286D6DB6
:101E90002900203B0020204D3835312058005A2D94
:101EA00050726F6265204F666673657400436F6F92
:101EB0006C696E672E2E2E0048656174696E672E00
:101EC0002E2E0045312025530020573A0020573A46
:101ED0000042656420436F6F6C696E672E2E2E0082
:101EE0004265642048656174696E672E2E2E00235A
:101EF000646566696E652044454641554C545F00F3
:101F0000626564004B6420004B6920004B70200028
:101F1000504944204175746F74756E652066696E12
:101F20006973686564212050757420746865206C3D
:101F3000617374204B702C204B6920616E64204BC0
:101F40006420636F6E7374616E74732066726F6D5C
:101F50002062656C6F7720696E746F20436F6E66C8
:101F6000696775726174696F6E2E680A0050494422
:101F7000204175746F74756E65206661696C656467
:101F8000212074696D656F75740A005049442041C1
:101F900075746F74756E65206661696C6564212067
:101FA00054656D706572617475726520746F6F2011
:101FB000686967680A00504944204379636C657317
:101FC0000025532025692F256900204B643A200005
:101FD000204B693A2000204B703A200020436C616E
:101FE0007373696320504944200A00204E6F206FAC
:101FF00076657273686F6F740A002054753A20001A
:10200000204B753A2000206D61783A2000206D69E0
:102010006E3A200020643A200020626961733A2001
:10202000005761697420666F72206865617420755D
:10203000702E2E2E00504944204175746F74756EB9
:10204000652073746172740A0050494420417574AC
:102050006F74756E65206661696C656421205465D6
:102060006D706572617475726520746F6F20686938
:1020700067680A00504944204175746F74756E6535
:1020800000504944204175746F74756E6520666117
:10209000696C6564212042616420686561746572C1
:1020A0002069640A004572723A20757466382066A9
:1020B0006F6E74206E6F7420696E697469616C69EB
:1020C0007A65642E004572723A207574663820660F
:1020D0006F6E74206E6F7420696E697469616C69CB
:1020E0007A65642E004572723A20757466382066EF
:1020F0006F6E74206E6F7420696E697469616C69AB
:102100007A65642E0042656400456E636C6F73757A
:102110007265002568753A253032687500253032C1
:1021200068753A2530326875002530326875272584
:102130003032687500202020202020200020202020
:102140002000657272001FE0201020102010102067
:1021500010202010201030300840048003001FE0C1
:102160003FF03FF03FF01FE01FE03FF03FF03FF057
:102170000FC0078003003FFFF038007030FC3020B4
:10218000FC102078102030102C00D02E31D02F7B66
:10219000D02F7BD02E31D02C00D0203010207810C2
:1021A00020FC1030FC303800703FFFF03FFFF0386B
:1021B00000703186302387102787902F87D02F0318
:1021C000D02030102078102078102030102F03D02D
:1021D0002F87D02787902387103186303800703FB3
:1021E000FFF01FFFF81FFFF804104002082002084C
:1021F0002004104008208010410010410008208079
:102200000410400000001FFFF81FFFF8001DC43F2E
:102210000000000C86198000000D0E198000000FD0
:102220000B198000000D9F198000000DD3998000CC
:10223000001CFBFF00000000000000000000000088
:102240000000F380001F80007700001980005B1CF5
:10225000F6131DAE5B35AB0635FB5B3DA70CBD9B96
:102260004B30EB19B19BE39D8E9F9D8E0001E000EA
:1022700000000001200000000001E0000000000C50
:102280000F00FE07022503BB017FFE08FE08FE05C6
:10229000080806000040F0C88888987810050808EB
:1022A000060000C0F88888888888F80505050600BB
:1022B000012030F830200508080600002070F820C2
:1022C000202020E00509090600FF2070A8A8B88892
:1022D000887020070505070001D86C366CD8050901
:1022E000090600FFF8A88888888888A8F8050A0ADF
:1022F0000600FE205050505088A8A88870030303A1
:1023000006000340A040FFFFFFFFFFFFFFFFFFFFAE
:10231000FFFFFFFFFFFFFFFFFFFFFFFF00000006C3
:1023200005FF01070706020080808080800080038F
:102330000303060105A0A0A005060606000050F84C
:102340005050F8500509090600FF2070A8A0702819
:10235000A87020050707060000C8C81020409898FC
:1023600005070706000040A0A040A89068010303ED
:102370000602058080800309090601FF2040408095
:1023800080804040200309090601FF804040202052
:102390002040408005070706000020A8702070A894
:1023A000200505050600012020F820200203030671
:1023B00001FFC04080050101060003F80202020689
:1023C0000100C0C0050707060000081010204040AB
:1023D00080050707060000708898A8C88870030762
:1023E0000706010040C040404040E00507070600E6
:1023F00000708808102040F8050707060000F8085C
:10240000103008887005070706000010305090F85B
:102410001010050707060000F880F008088870050E
:102420000707060000304080F0888870050707061F
:102430000000F80810102020200507070600007093
:10244000888870888870050707060000708888787B
:10245000081060020505060100C0C000C0C00206E9
:10246000060601FFC0C000C040800305050601014B
:102470002040804020050303060002F800F8030511
:102480000506010180402040800507070600007016
:102490008810202000200507070600007088B8A8D3
:1024A000B88070050707060000708888F88888885B
:1024B000050707060000F04848704848F005070780
:1024C000060000708880808088700507070600007D
:1024D000F04848484848F0050707060000F88080A3
:1024E000F08080F8050707060000F88080F0808003
:1024F00080050707060000708880809888700507AF
:1025000007060000888888F888888803070706017E
:1025100000E04040404040E005070706000038105A
:1025200010101090600507070600008890A0C0A05A
:102530009088050707060000808080808080F8056D
:10254000070706000088D8A8888888880507070636
:1025500000008888C8A898888805070706000070CA
:10256000888888888870050707060000F08888F04A
:1025700080808005070706000070888888A890681A
:10258000050707060000F08888F0A0908805070777
:102590000600007088807008887005070706000034
:1025A000F8202020202020050707060000888888C2
:1025B000888888700507070600008888888850503A
:1025C0002005070706000088888888A8A850050706
:1025D00007060000888850205088880507070600F5
:1025E0000088885020202020050707060000F808F2
:1025F00010204080F80309090601FFE080808080F8
:10260000808080E005070706000080404020101011
:10261000080309090601FFE020202020202020E0F7
:102620000503030600052050880501010600FEF899
:102630000303030601058040200505050600007020
:10264000087888780507070600008080F088888869
:10265000F0050505060000708080887005070706F4
:10266000000008087888888878050505060000704D
:1026700088F08070050707060000304840E04040C1
:10268000400507070600FE708888887808700507EF
:10269000070600008080F088888888030707060105
:1026A000004000C0404040E00409090601FE10005F
:1026B0003010101010906005070706000080808819
:1026C00090E09088030707060100C040404040406A
:1026D000E0050505060000D0A8A8A8A80505050680
:1026E0000000B0C888888805050506000070888845
:1026F00088700507070600FEF0888888F08080054E
:1027000007070600FE78888888780808050505060A
:102710000000B0C880808005050506000078807044
:1027200008F00507070600002020F82020201805E3
:1027300005050600008888889868050505060000DC
:1027400088888850200505050600008888A8A850BC
:10275000050505060000885020508805070706007B
:10276000FE88888850204080050505060000F81086
:102770002040F80309090601FF2040404080404006
:1027800040200109090602FF8080808080808080CF
:10279000800309090601FF804040402040404080FE
:1027A00005030306000248A890FF43616E6E6F7434
:1027B000206F70656E2073756264697220005344E7
:1027C0002063617264206F6B0A006F70656E526FD8
:1027D0006F74206661696C65640A00766F6C756D54
:1027E000652E696E6974206661696C65640A004EC5
:1027F0006F20534420636172640A002E0A006F70D8
:10280000656E206661696C65642C2046696C653A6A
:10281000200046696C652073656C65637465640AA5
:10282000002053697A653A200046696C65206F7014
:10283000656E65643A2000454E4420535542524F20
:102840005554494E450A002220706F7300222070B3
:102850006172656E743A2200535542524F55544985
:102860004E452043414C4C207461726765743A2296
:102870000053756263616C6C204F766572666C6F95
:1028800077004578636565646564206D61782053E1
:102890005542524F5554494E452064657074683A0C
:1028A00000667265736800646F696E670020666910
:1028B0006C653A20004E6F77200057726974696E1C
:1028C0006720746F2066696C653A20006D61726CD8
:1028D000696E66772E6F726700322E302E392E3376
:1028E0002D6B616431001FFFFFFFFFFFFF600000E1
:1028F000000001FF400000000000FF800000000019
:10290000007F83CF00000C303F87FF80000C301F1A
:10291000867980000C000F8C30C7838C30E78C30B8
:10292000CFC7CC31F38C30DCECEC33B98C30D86CC5
:102930006C33198C30D06C0C33198C30D86C0C3350
:10294000198C30DC6C0E3B198C30CF7C079F198CB6
:1029500030C77C038F1940000000000002600000B7
:10296000000000061FFFFFFFFFFFF870012C019021
:10297000012701B0012201C0011D01F00118011061
:1029800002130130020E016002090190020401C02D
:1029900002FF000003FA004003F5008003F000D0BE
:1029A00003EB002004E6007004E100E004DC0040DA
:1029B00005D700C005D2004006CD00D006C8008073
:1029C00007C3003008BE00F008B900C009B400B069
:1029D0000AAF00B00BAA00D00CA500000EA000505A
:1029E0000F9B00C01096005012910000148C00C084
:1029F000158700B0178200B0197D00D01B78000049
:102A00001E730040206E0090226900F02464004094
:102A1000275F0090295A00E02B5500102E5000200F
:102A2000304B0010324600E033410090353C00103E
:102A300037370070383200A0392D00B03A2800A096
:102A40003B2300603C1E00103D1900903D14001017
:102A50003E0F00703E0A00C03E0500003F000040EF
:102A60003FFBFF803FF6FFC03FF1FF2020506C612D
:102A70006E6E657242756666657242797465733A08
:102A800020002046726565204D656D6F72793A2091
:102A90000020436F6D70696C65643A204465632063
:102AA000323720323032310A00204C6173742055A5
:102AB0007064617465643A20323032312D30392DC2
:102AC0003033207C20417574686F723A20286B6126
:102AD000642C20416E796375626963204D6567617E
:102AE000205A65726F20322E302041424C20323401
:102AF00056290A004D61726C696E20322E302E39D3
:102B00002E332D6B6164310A0020536F6674776138
:102B100072652052657365740A002057617463689A
:102B2000646F672052657365740A002042726F7784
:102B30006E206F75742052657365740A00204578A5
:102B40007465726E616C2052657365740A00506F13
:102B500077657255700A0073746172740A004732A7
:102B6000385859004D31303031006572726F722023
:102B700077726974696E6720746F2066696C650A84
:102B800000446F6E6520736176696E672066696CBC
:102B9000652E0A004D323900456E6473746F707390
:102BA000002553202563202563202563202563000D
:102BB00020503A00205A3A0020593A0020583A0052
:102BC000656E6473746F7073206869743A200000D6
:102BD0000000010200090A000000000403080700C9
:102BE00000000000000000000000000000000000E5
:102BF0004D6F76652025736D6D004D6F76652030C5
:102C00002E316D6D004D6F766520316D6D004D6F0D
:102C100076652031306D6D004D6F766520417869A5
:102C200073004D6F76652045787472756465720027
:102C30004D6F7665205A004D6F76652059004D6FB7
:102C400076652058005072696E742066726F6D2030
:102C50004D6564696100FFFFFF205A3A200020594A
:102C60003A200042656420583A20004D6567612093
:102C70005A65726F20322E302052656164792E00C1
:102C80005072696E74696E672E2E2E005072696ED6
:102C9000742050617573656400204500205A00203F
:102CA000590020204D39322058005374657073202C
:102CB00070657220756E6974003B2000220A005511
:102CC0006E6B6E6F776E20636F6D6D616E643A2010
:102CD00022006F6B00DB0FC93F45BCDA3F8FB302A8
:102CE00040FCF0274056946140FE4B9B4084A5D8A1
:102CF00040E0231841346A5641E859974164DBD5D6
:102D0000416E271742B4B75542CE1A9742C8AED586
:102D100042B5885A43D40684BFA65FA7BF7443E078
:102D2000BF10B11AC01C2C58C0E8F697C0B849D6DD
:102D3000C04E4E17C124D355C1802497C1A0B5D52C
:102D4000C1121A17C244AE55C2781797C26CACD5DF
:102D5000C267885AC320746F6F206C6F6E672065DE
:102D60007874727573696F6E2070726576656E74B3
:102D700065640A0020636F6C6420657874727573F3
:102D8000696F6E2070726576656E7465640A006F97
:102D90006B0A00526573656E643A200020453A0064
:102DA000205A3A0020593A00583A000000220025E3
:102DB0000028002B0000002100240027002A000228
:102DC00002020202020202040404040404040403D2
:102DD00003030303030303010101010101010101D5
:102DE00002040810204080010204081020408001E5
:102DF0000204081020408080402010080402014591
:102E000072726F722077726974696E6720746F20B6
:102E1000454550524F4D210A0000DFD879DF11247B
:102E20001FBECFEFD0E4DEBFCDBF84B7809368155F
:102E300014BE0FB6F894A8958091600088618093C5
:102E40006000109260000FBE12E0A0E0B1E0E0E28E
:102E5000FBED01E00BBF02C007900D92AE38B10749
:102E6000D9F725E1AEE8B2E001C01D92A836B2075D
:102E7000E1F717E1CEE0D7E104C02197FE010E94FF
:102E8000D8EACD30D107C9F70E9493D90C9484EDCC
:102E90000C940000A0E1B0E0E0E5F7E10C9407EB52
:102EA0008C01DC01ED91FC910280F381E02DBE01EB
:102EB0006F5F7F4F0995882309F45DC08981807C0D
:102EC00091F56F81637070E0762F6627770F770F2B
:102ED0008885B4E08B9FC0011124682B792B8985EC
:102EE0008295869586958370682B6F5F7F4F90E003
:102EF00080E02A852370220F3B8537FB332730F98A
:102F0000232B3E813F70230F3327331F2750310976
:102F100004C0660F771F881F991F2A95D2F7609605
:102F2000E4E00C9423EB803419F56885669566958A
:102F300070E090E080E0CB01772766272A85622B3E
:102F4000098510E0102F0027012E000C220B330BF7
:102F5000602B712B822B932B6F5F7F4F8F4F9F4F77
:102F60004AE0660F771F881F991F4A95D1F7D7CF80
:102F70008BE0F801848360E070E0CB01D0CF08954E
:102F8000FC01828108954F925F926F927F928F929F
:102F90009F92AF92BF92CF92DF92EF92FF92CF9328
:102FA000DF93CDB7DEB728970FB6F894DEBF0FBE1C
:102FB000CDBF60913307709134076115710511F130
:102FC00080912F0790913007A0913107B09132077F
:102FD00089839A83AB83BC83072E000C880B990BE3
:102FE0000E9419E429813A814B815C810E9430EB77
:102FF0004B015C0120E030E040E251EC0E9413E420
:1030000087FF07C081E080933201C12CD12C76016B
:1030100013C020E030E040E251E4C501B4010E9459
:1030200094EC181604F581E080933201C12CD12C68
:103030009FE7E92E93E4F92EC701B60128960FB653
:10304000F894DEBF0FBECDBFDF91CF91FF90EF9020
:10305000DF90CF90BF90AF909F908F907F906F90B8
:103060005F904F90089580913A0790913B07A0910F
:103070003C07B0913D078D839E83AF83B8878091D5
:103080003201882391F010929104109292041092D0
:1030900093041092940410928D0410928E04109256
:1030A0008F0410929004109232012091910430917B
:1030B00092044091930450919404C501B4010E947C
:1030C00031EB2B013C0120E030E0A9010E9494EC9F
:1030D000C12CD12C760187FD14C02D813E814F81FA
:1030E000588560E070E08FE793E40E94A8EB6B01E5
:1030F0007C01A30192010E9413E4181614F47301D9
:103100006201C0929104D0929204E0929304F092F2
:103110009404209136073091370740913807509139
:103120003907C501B4010E9478E44B015C0180922B
:10313000850490928604A0928704B0928804A70127
:1031400096016D817E818F8198850E9478E46B0164
:103150007C01C0928904D0928A04E0928B04F092A0
:103160008C0440908D0450908E0460908F04709079
:10317000900429813A814B815C8160918104709136
:10318000820480918304909184040E9430EB20910A
:103190003E0730913F0740914007509141070E9400
:1031A00078E4A30192010E9430EB20ED3CEC4CE46A
:1031B0005DE30E9478E4A30192010E9431EB9B0140
:1031C000AC0120938D0430938E0440938F04509370
:1031D000900489819A81AB81BC8180938104909312
:1031E0008204A0938304B0938404C501B4010E94B7
:1031F00031EBA70196010E9431EB6B017C0120E0CD
:1032000030E04FE753E40E9413E4181634F4C12C65
:10321000D12C8FE7E82E83E4F82E20E030E0A901DE
:10322000C701B6010E9494EC87FF06CFEECE6091F5
:103230002F077091300780913107909132070895E0
:10324000FC0190E1A0E7B4E001900D929A95E1F7BE
:103250000895EF92FF920F931F93E0928903F092EB
:103260008A0300938B0310938C03B62F172F022F22
:10327000F32E242F582FB0938D0310938E03509369
:103280008F036FEFFF27B01B1F09520B30F45095CF
:103290001095B195160B560B66276093A604A6E011
:1032A000BA9F00929A04712DEE271A9F700DE11DAE
:1032B0005A9FE00D70939B04E0939C04AFE0BA9F8B
:1032C00000929E04712DEE271A9F700DE11D5A9FEA
:1032D000E00D70939F04E093A004AAE0BA9F0092CF
:1032E000A204712DEE271A9F700DE11D5A9FE00D6B
:1032F0007093A304E093A4041F910F91FF90EF90AB
:103300000895A5E0B0E0E7E8F9E10C9400EB6F3632
:1033100071058105910578F4FB01EE0FFF1FEE0F9B
:10332000FF1FEB5CF74F6591759185919491259600
:10333000EBE00C941CEBF62EE72E282FE5E3F7E0EC
:103340000027BB275F2D8E2D922F992341F4982FB4
:10335000852FB85F992319F4982F8827B85F90318B
:1033600038F482959295582F5F70807F952BBC5FC3
:10337000903428F4880F991F880F991FBE5F9038EA
:1033800018F4880F991FB395880F991FE90FF01F44
:10339000549181E09927B85079F1C0F0B0FF02C094
:1033A000550F881FB1FF04C0550F881F550F881F88
:1033B000B2FF06C082955295152F1F70507F812B4A
:1033C000B3FF1AC0982F852F552716C0B195B0FFAF
:1033D00002C085955795B1FF04C085955795859591
:1033E0005795B2FF05C08295507F5295582B8F702C
:1033F000B3FF02C0582F8827BB247727AA27B2E043
:10340000F59EB0187109A00BB00BE59E7019A109CB
:10341000B00B259FA019B109F89E7019A109B00B36
:10342000E89EA019B109289FB019F99EA019B10909
:10343000E99EB0195B9DA12C992444276627332768
:103440008B9DA00C911C401F601F301F9B9D900CFA
:10345000411D601F301F579FA00C911C401F601F13
:10346000301F879F900C411D601F301F979F400D9C
:10347000611D301F5A9F900C411D601F301F8A9F95
:10348000400D611D301F9A9F600D311D5B9F400DE7
:10349000611D301F8B9F600D311D9B9F300DB1E072
:1034A000AA277727BB24F49EB0187109A00BB00B94
:1034B000E49E7019A109B00B249FA019B109F69ED2
:1034C0007019A109B00BE69EA019B109269FB01989
:1034D000F39EA019B109E39EB019BF187E09A20B93
:1034E00020F0B1E04B0F601F301F1124762F642FA6
:1034F00090E0832F1CCFFC017081472F50E0062EF7
:1035000002C0559547950A94E2F740FF14C04091D8
:10351000080450E0062E02C0559547950A94E2F73C
:1035200040FF09C021E030E001C0220F6A95EAF7B0
:1035300020952723208308958F929F92AF92BF9268
:10354000CF92DF92EF92FF92FC01C080D180E280A7
:10355000F38020E030E048EC52E4C701B6010E945D
:1035600078E44B015C0120E030E0A901C701B6011D
:103570000E9413E420E030E040EA50E487FF04C0FA
:1035800020E030E040EA50ECC501B4010E9431EB8C
:103590002DEC3CEC4CEC5DE30E9478E40E9410ECD6
:1035A0009B018BE237FF05C022273327261B370BF1
:1035B0008DE280939702C90168EE73E00E94A9EA48
:1035C000CB01EAE0F0E0BF010E94A9EA805D8093B0
:1035D0009802C90164E670E00E94A9EACB01BF012C
:1035E0000E94A9EA805D80939902C901BF010E94EF
:1035F000A9EA9C01CB01BF010E94A9EA805D8093EA
:103600009A028EE280939B02205D20939C0287E9C0
:1036100092E0FF90EF90DF90CF90BF90AF909F909F
:103620008F9008954F925F926F927F928F929F92A8
:10363000AF92BF92CF92DF92EF92FF92FC01C080D7
:10364000D180E280F38020E030E04AE754E4C70113
:10365000B6010E9478E44B015C0120E030E040E2DA
:1036600051ECC701B6010E9413E4181654F420E08F
:1036700030E048EC52E4C701B6010E9494EC87FDAB
:103680008AC020E030E0A901C701B6010E9413E41E
:1036900087FF72C060E070E080EA90ECA5019401C1
:1036A0000E9431EB2DEC3CEC4CEC5DE30E9478E4A5
:1036B0000E9410EC6B017C01F7FC63C020E137E253
:1036C00040E050E00E94BCEACA01B9012AE030E0C3
:1036D00040E050E00E94BCEA605D60939702C70141
:1036E000B60128EE33E040E050E00E94BCEA9AE0E8
:1036F000892E912CA12CB12CCA01B901A5019401EC
:103700000E94BCEA605D60939802C701B60124E69E
:1037100030E040E050E00E94BCEACA01B901A501D6
:1037200094010E94BCEA605D609399028EE28093EE
:103730009A02C701B601A50194010E94BCEA6B017F
:10374000CA01B901A50194010E94BCEA605D6093C1
:103750009B02F0E3CF0EC0929C0287E992E0FF90BB
:10376000EF90DF90CF90BF90AF909F908F907F9021
:103770006F905F904F90089560E070E080EA90E471
:103780008DCFF094E094D094C094C11CD11CE11C66
:10379000F11C6DE2A2CF20E030E0A901C701B60123
:1037A0000E9413E487FF6BC060E070E080EA90EC59
:1037B000A50194010E9431EB2DEC3CEC4CEC5DE357
:1037C0000E9478E40E9410EC4B015C0120E030E0A4
:1037D000A901C701B6010E9413E487FD0BC020E0D8
:1037E00030E040E251E4C701B6010E9494EC60E28F
:1037F00087FD13C0B7FC48C0C501B40128EE33E013
:1038000040E050E00E94BCEACA01B9012AE030E081
:1038100040E050E00E94BCEA605D60939802C50100
:10382000B40124E630E040E050E00E94BCEA8AE0C7
:10383000482E512C612C712CCA01B901A3019201AF
:103840000E94BCEA605D609399028EE280939A02C6
:10385000C501B401A30192010E94BCEA6B01CA0137
:10386000B901A30192010E94BCEA605D60939B02D2
:1038700080E3C80EC0929C0288E992E070CF60E0BD
:1038800070E080EA90E494CFB094A09490948094F7
:10389000811C911CA11CB11C6DE2BFCF282F81E3BC
:1038A000243609F080E28093990290E22A3040F0B9
:1038B0003AE0822F632F0E947CEA0E947CEA905DAE
:1038C00090939A02822F6AE00E947CEA905D909326
:1038D0009B0285E280939C0289E992E008956091C1
:1038E0002C0170912D01072E000C880B990B0E9462
:1038F00019E42AE037ED43E25CE30E9478E4609348
:103900006F0170937001809371019093720108951B
:10391000CF93DF93EC01CB01BA010E9419E423E3BA
:1039200033E343E250E40E9478E420E030E040E0FA
:103930005FE30E9431EB0E9415EC6883DF91CF9129
:1039400008950E9419E423E333E343E250E40E9424
:1039500078E420E030E040E05FE30E9431EB0E9439
:1039600015EC24E6629FC001112481589F4F6FEF30
:1039700070E00E94A9EA862F91CF80917307811190
:1039800004C0809127078093A90708958091AD1402
:103990008823C1F081508093AD14EBEFF2E18823CE
:1039A00051F08150990B2BE1289FF001299FF00DD8
:1039B0001124E156FC4E8BE1A0EEB2E101900D9294
:1039C0008A95E1F72091AD14211105C08091B714BB
:1039D00080648093B71481E090E0A0E0B0E0211112
:1039E00003C080E090E0DC018093690790936A0750
:1039F000A0936B07B0936C071092640781E08093EB
:103A0000660783E080936A010895CF93DF93EC010A
:103A1000CB01BA010E9419E4688379838A839B836E
:103A2000DF91CF910895CF93DF93EC01CB01BA01E1
:103A30000E9419E42DEC3CEC4CEC5DE30E9478E430
:103A4000688379838A839B83DF91CF910895CF9395
:103A5000DF93EC01CB01BA010E9419E42AE037EDB3
:103A600043E25CE30E9478E4688379838A839B83E2
:103A7000DF91CF910895CF92DF92EF92FF92CF9393
:103A8000DF9300D000D0CDB7DEB70E9419E42AE062
:103A900037ED43E25CE30E9478E46B017C0120E0B7
:103AA00030E0A9010E9413E42DEB37E346E055E333
:103AB00087FF04C02DEB37E346E055EBC701B601A5
:103AC0000E9431EB69837A838B839C83CE010196BC
:103AD000A9DD0F900F900F900F90DF91CF91FF9085
:103AE000EF90DF90CF900895CF93DF93EC01CB015F
:103AF000BA010E9419E40E9410EC79836883DF9177
:103B0000CF9108958F929F92AF92BF92CF92DF9202
:103B1000EF92FF92FC01C080D180E280F38020E030
:103B200030E0A901C701B6010E9413E487FD99C0E6
:103B30006DEB77E386E095E3A70196010E9431EBF8
:103B40009F7720E030E048EC52E40E9478E420E0E7
:103B500030E040EA50E40E9431EB2DEC3CEC4CECC0
:103B60005DE30E9478E40E9410EC6B017C0180E22E
:103B70008093960260E2F0E1CF16F7E2DF06E104FF
:103B8000F1048CF0C701B60120E137E240E050E0DB
:103B90000E94BCEACA01B9012AE030E040E050E0EE
:103BA0000E94BCEA605D6093970260E288EEC816EE
:103BB00083E0D806E104F1048CF0C701B60128EED9
:103BC00033E040E050E00E94BCEACA01B9012AE0BB
:103BD00030E040E050E00E94BCEA605D60939802F3
:103BE00060E2E4E6CE16D104E104F1048CF0C701F2
:103BF000B60124E630E040E050E00E94BCEACA0191
:103C0000B9012AE030E040E050E00E94BCEA605D8B
:103C1000609399028AE0882E912CA12CB12CC701C7
:103C2000B601A50194010E94BCEA6B01CA01B90169
:103C3000A50194010E94BCEA605D60939A028EE245
:103C400080939B02F0E3CF0EC0929C0286E992E043
:103C5000FF90EF90DF90CF90BF90AF909F908F90AC
:103C600008956DEB77E386E095EB66CFA4E0B0E0D6
:103C7000ECE3FEE10C9409EB0E9419E42DEC3CEC22
:103C80004CEC5DE30E9478E469837A838B839C83A8
:103C9000CE01019637DF2496E2E00C9425EBCF931A
:103CA000DF93EC018D810E941B8960E08B810E9473
:103CB00018CADF91CF910895CF92DF92EF92FF92D1
:103CC0000F931F93CF938C01C62F69017A01E7DF11
:103CD0000E94CBCB8C2F80640E940F898F2D0E9475
:103CE0000F898E2D0E940F898D2D0E940F898C2D9A
:103CF0000E940F8987E8C11101C085E90E940F89E0
:103D0000CC3011F40E941489C0E00E941489F8019B
:103D1000868387FF04C0CF3F11F0CF5FF6CFCF91EE
:103D20001F910F91FF90EF90DF90CF90089561E089
:103D3000FC0183810E9418CA8FEF0C940F890F93A6
:103D40001F93CF938C01ABDF0E94CBCBC82F88236E
:103D500069F08DEF0E940F890E94CBCBC82FC8015C
:103D6000E6DF8C2FCF911F910F91089582E1F8012A
:103D70008483F5CFB0E0A0E0E0ECFEE10C94FFEA34
:103D8000EC016A017B014801590120E030E0A90102
:103D900067E392DFA501980167E1CE018DDF811114
:103DA0001DC08F81833039F089E0CC0CDD1CEE1C06
:103DB000FF1C8A95D1F7A701960169E1CE017CDF4E
:103DC00011E0882319F010E087E08C83CE01AFDF8B
:103DD000812FCDB7DEB7ECE00C941BEB89E08C8330
:103DE00010E0F4CFCF93DF93EC016EBDFA01CA016E
:103DF0009E5F0DB407FEFDCF20812EBD0DB407FEE2
:103E0000FDCF21812EBD3296E817F90791F70DB449
:103E100007FEFDCF8FEF0E940F898FEF0E940F8961
:103E20000E9414898E838F71853041F083E18C83E9
:103E3000CE017DDF80E0DF91CF91089581E0FBCF5F
:103E40000F931F93CF93DF93EC018B0128DF0E9428
:103E5000CBCB81110BC085E18C8310E0CE0167DFF5
:103E6000812FDF91CF911F910F910895A8016CEFE1
:103E7000CE01B8DF182F882371F3F0CF0F931F9373
:103E8000CF93DF93EC0189018F81833039F089E092
:103E9000440F551F661F771F8A95D1F79A01AB0112
:103EA00068E1CE0109DF811127C0A8016EEFCE01C4
:103EB00099DF182F8823A9F00E94CBCB182F8823D5
:103EC000C1F020E030E0A9016DE0CE01F5DE8823ED
:103ED00021F086E18C8310E004C00E9414898111D6
:103EE000F8CFCE0124DF812FDF91CF911F910F9169
:103EF000089587E18C83F5CF86E0ECCF1F93CF93B5
:103F0000DF93EC01CCDE20E030E0A9016CE0CE01D3
:103F1000D3DE11E0882319F010E083E08C83CE011A
:103F200006DF812FDF91CF911F9108951F93CF93CB
:103F3000DF93EC018F81833039F089E0440F551F06
:103F4000661F771F8A95D1F79A01AB0162E1CE0116
:103F5000B3DE11E0882319F010E085E08C83CE01F8
:103F6000E6DE812FDF91CF911F9108958F929F926E
:103F7000AF92BF92EF92FF920F931F93CF93DF9375
:103F80008C01EB017A010E9400CB4B015C012CE219
:103F9000820E21E0921EA11CB11C0E941489F8011E
:103FA00086838F3F69F40E9400CB681979098A09DA
:103FB0009B0997FDF2CF81E1F8018483C0E021C025
:103FC0008E3F69F5F1E0EF1AF1088FEF8EBDFE012B
:103FD0002FEF0DB407FEFDCF8EB581932EBDCF011F
:103FE0008C1B9D0B8E159F05A0F30DB407FEFDCF16
:103FF0008EB5CE0DDF1D88830E9414890E9414891E
:10400000C1E0C80194DE8C2FDF91CF911F910F91F9
:10401000FF90EF90BF90AF909F908F9008958FE0AA
:10402000CBCF0F931F93CF93DF93EC018B0137DE40
:1040300040E052E0B801CE0199DFDF91CF911F91AE
:104040000F9108950F931F93CF93DF93EC01890194
:104050008F81833039F089E0440F551F661F771F29
:104060008A95D1F79A01AB0161E1CE0125DE882363
:1040700051F084E08C83CE015ADE80E0DF91CF9155
:104080001F910F91089540E052E0B801CE016EDF1C
:10409000F5CFB0E0A0E0EFE4F0E20C94FFEAEC0131
:1040A000162F1F821C824B830E9400CB6B017C0168
:1040B00020EDC20E27E0D21EE11CF11CA89561E0A4
:1040C0008B810E9418CA8B810E94D6AF249A2C9AA9
:1040D000279A2698259A81E00E941B8985E08D8386
:1040E0000E941B890AE08FEF0E940F890150D9F7C7
:1040F000A89520E030E0A90160E0CE01DDDD8E83EF
:10410000813079F00E9400CB6C197D098E099F09DE
:1041100097FDEFCF81E08C83CE0109DE1A8280E02B
:1041200065C0A8952AEA31E040E050E068E0CE01A1
:10413000C3DD853031F581E08F83A8958F81812C97
:10414000912C5401823029F4812C912CA12C80E4F3
:10415000B82E20E030E0A90167E3CE01ADDDA50176
:10416000940169E2CE01A8DD8E838823F1F00E94DC
:1041700000CB6C197D098E099F0997FDEACF8AE073
:10418000CACF04E00E9414898E830150D9F78A3A7D
:1041900011F482E0D1CF0E9400CB6C197D098E0909
:1041A0009F0997FDBFCF82E0B6CF8F818230B9F4EF
:1041B00020E030E0A9016AE3CE017EDD882311F022
:1041C00088E0A9CF0E941489807C803C11F483E0B0
:1041D0008F830E9414890E9414890E941489CE0141
:1041E000A6DD81E08A83173030F41D83CDB7DEB7BA
:1041F000ECE00C941BEB88E18C8391CF0F931F9321
:10420000CF93DF93EC018B0120E030E0A90169E05E
:1042100053DD882351F080E18C83CE0188DD80E07E
:10422000DF91CF911F910F91089540E150E0B801C7
:10423000CE019CDEF5CFEF92FF920F931F93CF93A9
:104240007B018A01C2E48F3F09F0C4E580E20E944D
:104250008C7F8C2F0E948C7F8AE30E948C7FF701D9
:10426000608171818281938142E00E94F5AF86E393
:1042700093E10E94AD7FF801608171818281938119
:1042800042E00E94F5AF62E070E080E090E00E94C2
:1042900074CACF911F910F91FF90EF9008950C94E5
:1042A0000CCB4091870321E042276CE070E00C9436
:1042B000AAAF4091870321E0422764E070E00C94AC
:1042C000AAAF4091870321E0422761E070E00C949F
:1042D000AAAF4091870321E0422761E070E00C948F
:1042E000AAAF4091870321E0422768E070E00C9478
:1042F000AAAF4091870321E042276CE070E00C9464
:10430000AAAF41E061E070E00C94AAAF409187034E
:1043100021E042270C94AAAF6CE070E00C94A7CA8D
:1043200061E070E00C94A7CA6CE070E00C94A7CA3E
:1043300064E070E00C94A7CA9091AE0281E08927F6
:104340000C94437761E087E297E00C94CF77CF93AA
:10435000C82FCB010E94AD7F89E696E00E94AD7F19
:104360008AE596E0CC2311F08FE596E00E940C8858
:10437000CF91089520E030E0A901BC0185E791E0EC
:104380000C94C4C080E090E0A0E8B0E480937D018C
:1043900090937E01A0937F01B09380018AE192E027
:1043A000E9DF80E090E0A0EFB1E4809375019093A5
:1043B0007601A0937701B09378018093790190936F
:1043C0007A01A0937B01B0937C01E091E503EE0FAD
:1043D000FF0BE650FE4F808191818330910539F1CA
:1043E00084309105C9F1029761F480E090E0A3E484
:1043F000B3E48093750190937601A0937701B09315
:10440000780182E092E0B6DF10927D0110927E0189
:1044100010927F01109280018AE192E0ABDF8091DF
:10442000E5038F5F8430ECF48093E503089580E02A
:1044300090E0A3E4B3E48093750190937601A09398
:104440007701B09378018093790190937A01A093DA
:104450007B01B0937C01D5CF80E090E0A3E4B3E48E
:10446000F2CF1092E5030895B0E0A0E0EAE3F2E2B3
:104470000C9409EB20E24F8158856E818D810E945A
:10448000CBC5E2E00C9425EB80912707909128079B
:104490000C9441CB609127078FEF0C944BCB80910C
:1044A0002707682F0C944BCB6FEF809127070C9454
:1044B0004BCB61E570E582E00C94D9C765E570E50A
:1044C00081E00C94D9C769E570E580E00C94D9C708
:1044D0006DE570E583E00C94D9C7109264070C94E5
:1044E0003CD84FE350E06AE874E086EE96E00C9426
:1044F0006AED8091391390913A13891B8F7011F4F2
:104500000C94237981E0089580916A01882341F019
:104510006091DD037091DE0341E081E00C946BC596
:104520000895CF93DF93EC010E94C1D21B82DF91EB
:10453000CF910895CF93DF93EC01462F41706C85A6
:104540007D858E859F850E94D2CF882351F08889F2
:1045500020E2829FC001112489569F4EDF91CF91A6
:10456000089590E080E0FACFCF93DF93EB01FC0158
:104570002381211104C080E0DF91CF910895225062
:10458000223028F48FE28883198281E0F5CF60E041
:10459000D1DF009781F3DC0160E080E09EE22D91A5
:1045A000203299F0883031F49E01260F311DF90137
:1045B00090836F5F9E01260F311DAD01415051095F
:1045C000FA014081F90140836F5F8F5F8B3039F7CB
:1045D000FE01E60FF11D1082D8CFACE0B0E0E3EFB2
:1045E000F2E20C94FAEA5C01DC0159968D909C9001
:1045F000F40181859285A385B4859C01AD012F5F6F
:104600003F4F4F4F5F4F29873A874B875C87D501D4
:1046100014964D905D906D907C90179741145104C5
:104620006104710409F459C0BFEF4B1A5B0A6B0AAD
:104630007B0A312C730162011D821E821F82188643
:10464000F40181859285A385B4852D813E814F81BA
:104650005885281739074A075B0708F056C089852F
:104660009A85AB85BC858C159D05AE05BF0550F4BC
:1046700082E0C82ED12CE12CF12C92E0492E512C55
:10468000612C712C9E012F5F3F4FB701A601C40121
:104690000E94DCD18823C9F189819A81AB81BC81D8
:1046A000892B8A2B8B2B01F1260137019FEF491AA9
:1046B000590A690A790A2D813E814F8158852F5FF9
:1046C0003F4F4F4F5F4F2D833E834F8358873FEFC0
:1046D000C31AD30AE30AF30AB3CF40805180628041
:1046E000738033243394A6CFC414D504E604F704AE
:1046F00011F70FEF1FEF2FEF3FE0B701A601C40145
:104700000E9462D1782E811106C0712C872D2C96C3
:10471000E1E10C9416EBF5014481558166817781C6
:10472000411551056105710539F097018601C401F4
:104730000E9462D1882349F3D5011496CD92DD926F
:10474000ED92FC921797332051F0D701C6010196E4
:10475000A11DB11DF40180839183A283B383F50170
:1047600085899689A789B08D892B8A2B8B2B71F629
:10477000C58AD68AE78AF08E818180688183C6CF18
:1047800040E050E0BA010C940AD34F925F926F92CE
:104790007F92AF92BF92CF92DF92EF92FF920F93F0
:1047A0001F93CF93DF931F92CDB7DEB78C017B01B0
:1047B0005A01C22EDB0159968D919C91F801928F7E
:1047C000818FCB01DDDF712CF70180859185A2857A
:1047D000B385418952896389748984179507A6072F
:1047E000B70708F052C055E0B695A79597958795FD
:1047F0005A95D1F7F82FFF70DF2ED70113968C91C1
:10480000823010F480E0DAC041E050E0BE016F5F1A
:104810007F4FC7010E9405D40197A1F7F70180855A
:104820009185A285B3854F96A11DB11D8087918783
:10483000A287B387F0E2DF9EB001112469567F4E54
:1048400061157105F9F2DB018C91882341F0853EF9
:1048500009F04BC0772029F077247394B5CF7110FD
:104860000EC08091971290919812A0919912B091D8
:104870009A12F80184879587A687B787D08ADB01CB
:104880008C918111E9CF772473948C2D82748234BA
:1048900009F0B8CF772009F4A1C0F801D08861E011
:1048A000C80148DE009709F4ADCF20E2DC011D927B
:1048B0002A95E9F72BE0F501DC0101900D922A958C
:1048C000E1F721E238E2FC01318B208B40E058E037
:1048D00057874687338B228B318F208F578B468BA0
:1048E0000E9489CF811109C08DCF4BE050E0C501F6
:1048F0000E941AED892B09F067CFF0E2DF9ED0010C
:1049000011249D0129563F4EF9018385817121F0C3
:104910008C2D827109F000C1F801818D928D40913A
:104920009712509198126091991270919A1244873F
:10493000558766877787D08AFD01E956FF4E448800
:104940005588712C612C320155244424D801559688
:104950004D925D926D927C925897428D538D70E08E
:1049600060E0442955296629772955964D935D9332
:104970006D937C935897D9011B962C91287109F05F
:10498000BDC0848D958DA68DB78DF801818B928BDE
:10499000A38BB48B81E083838C2D8F70F80181838E
:1049A000148215821682178210861186128613864B
:1049B00081E0C4FE03C0C8010E948FD30F90DF9135
:1049C000CF911F910F91FF90EF90DF90CF90BF900C
:1049D000AF907F906F905F904F900895D70113969E
:1049E0008C911397823009F40DCF51968D919D9142
:1049F0000D90BC91A02D803E9F4FAF41B10508F0B6
:104A000001CFC701EADD882309F4FCCE0E9489CFDB
:104A1000882309F4F7CED7015996ED91FC915A9766
:104A200014964D905D906D907C901797B2E04B1A64
:104A3000510861087108858504C0440C551C661C2A
:104A4000771C8A95D2F786859785A089B189480E0B
:104A5000591E6A1E7B1E81E080939B124092971222
:104A6000509298126092991270929A12E7E9F0E1CE
:104A700080E092E0DF019C011D9221503040E1F77F
:104A8000DD24D394D7015996ED91FC918481D816F9
:104A9000C0F480919C1290919D12DC01ED91FC91EB
:104AA0000288F389E02D27E930E1B301A2014D0D21
:104AB000511D611D711D0995882309F4A3CED3945E
:104AC000E1CF258580E092E0A0E0B0E004C0880F4F
:104AD000991FAA1FBB1F2A95D2F7F7014189528956
:104AE00063897489840F951FA61FB71F818B928BD2
:104AF000A38BB48B87E990E1D12CD7CE203161F420
:104B000098012F5E3F4F0E9458D2882329F084E0FD
:104B1000D80113968C9340CFD80113961C9272CE75
:104B2000FC0123812111FDCC0895A1E4B0E0EBE963
:104B3000F5E20C94F9EA4C015B017A01222E19820C
:104B40001C821C8E1F8E6115710569F410E0CE0168
:104B50004C96E6DFCE010196E3DF812FCF5BDF4F7E
:104B6000E2E10C9415EBFC0183818111EFCFFA0196
:104B700080818F3251F18B01CE0101966C012C01A5
:104B800080E2382E360122963FAE229721963FAE24
:104B900021973FAE3EAE3DAE3CAE3BAE3AAE39AEF7
:104BA00038AE3FAA970190E047E0D9018D91882364
:104BB00009F447C08F3209F444C08E3209F54A30F7
:104BC00029F298E04AE09D01F0CFFB0183818250F9
:104BD0008230A0F0618D728DCE014C960E94EDD78F
:104BE000882309F4B3CF8E01045E1F4FC7017C01F7
:104BF0000196F70120812F32D1F3BECF8B01F6CF82
:104C0000E2E4F3E12491222321F031968213FACFDA
:104C10009DCF491708F49ACF813208F497CF8F3788
:104C200009F494CF3FE9380F3A3108F420EEE7E376
:104C3000F0E0EC0FFD1FE90FF11D820F80839F5FF5
:104C4000C2CF8FA9803209F481CF7901F901808127
:104C50002F5F3F4F8F32C9F38823C1F021E0AE01AF
:104C6000495C5F4FB801C60190DD882309F46ECF1F
:104C70000A151B0511F0C80154DCCE014C964C14EA
:104C80005D0409F0C30186016C017DCF222DAE01C8
:104C9000495C5F4FB801C40178DD182F58CFEF92FF
:104CA000FF921F93CF93DF93CDB7DEB728970FB650
:104CB000F894DEBF0FBECDBF182F8CEAE82E82E13C
:104CC000F82EF70160857185072E000C880B990B73
:104CD0000E9419E46D837E838F839887F701848116
:104CE0009581A681B78189839A83AB83BC83AE010A
:104CF0004B5F5F4FBE016F5F7F4F80E09CDA9BE2AE
:104D0000E92E97E0F92EF70160857185072E000CDA
:104D1000880B990B0E9419E46D837E838F8398879B
:104D2000F70184819581A681B78189839A83AB83BA
:104D3000BC83AE014B5F5F4FBE016F5F7F4F8FEF54
:104D40007ADA87E11802F0011124E455FD4E6285FC
:104D500070E08EE393E10E94FE87F701628570E0C8
:104D600089E393E10E94FE8728960FB6F894DEBF90
:104D70000FBECDBFDF91CF911F91FF90EF900895AF
:104D80000F930FB70F9300916E000B7F00936E008F
:104D900078940F930BB70F930CB70F921F922F932A
:104DA0003F934F935F936F937F938F939F93AF93B3
:104DB000BF93EF93FF9311240E946563FF91EF91DE
:104DC000BF91AF919F918F917F916F915F914F9123
:104DD0003F912F911F900F900CBF0F910BBF0F9120
:104DE0000460F89400936E000F910FBF0F91189517
:104DF000CF93DF9310929703CCEAD2E119861886FD
:104E00000E940CCB1A865D98CBE2D7E019861886F3
:104E10000E94AB671A865C98DF91CF910895B0E04D
:104E2000A0E0E5E1F7E20C94FFEAB0E4A0E06A2F2D
:104E300070E0AB014B0F511D55954795411111C0C5
:104E4000EDE6F9E265917491072E000C880B990B41
:104E50000E9419E4CDB7DEB7ECE00C941BEBB42F45
:104E6000E8CFA41711F0B41303C0E9E6FAE2EACFE1
:104E70009A0121503109220F331F220F331FF901EC
:104E8000E559F64DE590F490F901E159F64DC591DB
:104E9000D4918E159F051CF3A42FC817D9070CF4C5
:104EA000C6CFF901E359F64D05911491F901EF5878
:104EB000F64DC590D490BC016E197F09072E000CE9
:104EC000880B990B0E9419E44B015C01B601601B31
:104ED000710B072E000C880B990B0E9419E49B01A3
:104EE000AC01C501B4010E9478E44B015C01BE0134
:104EF0006E197F09072E000C880B990B0E9419E48C
:104F00009B01AC01C501B4010E94A8EB6B017C01BF
:104F1000B801012E000C880B990B0E9419E49B012B
:104F2000AC01C701B6010E9431EB94CFEF92FF9222
:104F30000F931F93CF93DF93C82F7B018A0180913A
:104F40002607833090F00E94EC85C7010E94AD7F58
:104F50008CE992E10E94AD7FCF3F79F588E992E13B
:104F60000E94AD7F8AE00E948C7F42DFA8958091ED
:104F7000800481113EC081E08093800482E08093B0
:104F8000260736DFD5E1D150149A49F169E170E086
:104F900080E090E00E9474CAA895149868E270E0DE
:104FA00080E090E00E9474CAA89568E270E080E01A
:104FB00090E00E9474CAA895E6CFC7FDD3CF86E9DA
:104FC00092E10E94AD7F6C2F0C2E000C770B880BAA
:104FD000990B0E94ABAD8AE00E948C7FC3CF6FE833
:104FE00072E1CF3F11F063E972E140E0C8010E9435
:104FF0004188CDB7DEB7E6E00C9421EBB0E0A0E04D
:10500000E4E0F8E20C94FBEAEC016B014A01B22EF9
:10501000FA014080518062807380A30192016D810A
:105020007E818F8198850E9413E48823A1F04D82B0
:105030005E826F827886AA24A39420E030E0A901E2
:10504000F40160817181828193810E9494EC181631
:105050000CF0A12CAC828C818230A1F0833009F459
:105060004FC08130D1F52D813E814F815885F601A9
:1050700060817181828193810E9413E487FD2DC03C
:1050800082E08C83B7010F2C000C880B990B0E94D7
:1050900019E49B01AC016D817E818F8198850E940E
:1050A00030EB9B01AC01F6016081718182819381BB
:1050B0000E9494EC87FD16C00E9400CB6B017C011E
:1050C0009801A8EEB3E00E946DEAC60ED71EE81E56
:1050D000F91EC882D982EA82FB82CDB7DEB7E0E151
:1050E0000C9417EB0E9400CB088119812A813B8127
:1050F000601B710B820B930B97FDEFCF83E08C83CA
:1051000046E153E166E273E18B2D10DFE6CF4AEB17
:1051100052E167EC72E10ACFCF93DF93A8958091BB
:10512000AE129091AF120E9423AF6093B0127093B1
:10513000B1128093B2129093B31280912D07909187
:105140002E076DDE60932F07709330078093310731
:1051500090933207C091AE12D091AF12809163014B
:1051600090916401C817D90714F480E0D0DF8091D2
:10517000B4129091B512181619066CF48091610161
:10518000909162018C179D0734F447EF52E164E07F
:1051900073E180E0CBDE20912D0730912E078091C6
:1051A000DE069091DF062817390714F48FEFAFDF82
:1051B0008091330790913407181619068CF42091CA
:1051C0002D0730912E0780915F0190916001821729
:1051D000930734F447EF52E164E073E18FEFA6DE0A
:1051E000DF91CF910895A4E0B0E0E9EFF8E20C94EC
:1051F000FFEA80912607811106C0A8952496ECE06D
:105200000C941BEB28C1809195048111F7CF81E0AC
:105210008093950480919803811107C010929504A2
:105220002496ECE00C941BEB16C176DF10929803E9
:105230000E9400CB4B015C010E94C6AD6B017C015A
:105240006091670170916801072E000C880B990B23
:105250000E9419E49B01AC01C701B6010E9494ECC5
:1052600018160CF4E7C06091B4127091B512072EB5
:10527000000C880B990B0E9419E469837A838B8355
:105280009C8334E0E32EF12C08E210E020E0AE0134
:105290004F5F5F4F60EB72E186E193E1AFDEC0905C
:1052A000B012D090B112E090B212F090B3126091AF
:1052B000650170916601072E000C880B990B0E9406
:1052C00019E49B01AC01C701B6010E9494EC1816C9
:1052D000CCF46091670170916801072E000C880B77
:1052E000990B0E9419E49B01AC01C701B6010E9411
:1052F00013E487FF07C00E94CFAD0E9410EC7595A4
:10530000679501C060E06093B6128091A8129091F9
:10531000A912A091AA12B091AB120097A105B105F4
:10532000C1F0A5019401281B390B4A0B5B0BDA0174
:10533000C901B7FD0EC00E94C6AD0E9410EC2091BD
:10534000A6123091A712621773070CF47DC00E9459
:105350000CCB0E94171920E030E04AEF52E40E9483
:1053600094EC18160CF463C080919303909194030D
:10537000A0919503B09196030097A105B105A1F006
:10538000881A990AAA0ABB0AB7FC0EC00E9417190C
:105390000E9410EC209191033091920362177307E1
:1053A0000CF44BC00E94AB676091330770913407D7
:1053B000072E000C880B990B0E9419E469837A83ED
:1053C0008B839C8392E0E92EF12C04E110E02FEF17
:1053D000AE014F5F5F4F6FE277E08FE193E10EDE4A
:1053E00080902F0790903007A0903107B09032073F
:1053F00020E030E040EA50E4C501B4010E9494ECA2
:1054000087FD11C020E030E04AEF52E4C501B4014D
:105410000E9413E418163CF00E94C3170E9410EC7F
:105420007595679501C060E060933507F7CE8FEF03
:105430006EDE9ACF80E06BDE16CF49ED52E168EE6A
:1054400072E18FEF73DDB0CF49ED52E168EE72E1AA
:1054500080E06CDD7ECFCF92DF92EF92FF92CF9310
:10546000DF93EC01C880D980EA80FB8085E892E177
:105470000E94AD7FC701B6010E949073CC80DD8091
:10548000EE80FF8084EA9DE20E94AD7FC701B601F5
:105490000E949073C884D984EA84FB8480EA9DE2E8
:1054A0000E94AD7FC701B6010E9490738AE00E94FE
:1054B0008C7FDF91CF91FF90EF90DF90CF90089598
:1054C000BC012091610430916204409161045091CB
:1054D00062042417350731F481E02617370709F0F5
:1054E00080E008959A01F1CF0F930FB70F930091C9
:1054F0006E000F930B7F00936E0000916F000D7F85
:1055000000936F000F930BB70F930CB70F921F927E
:105510002F933F934F935F936F937F938F939F93BB
:10552000AF93BF93EF93FF931124F9D4FF91EF91C1
:10553000BF91AF919F918F917F916F915F914F91AB
:105540003F912F911F900F900CBF0F910BBF0F91A8
:105550000260F89400936F000F9100936E000F911A
:105560000FBF0F91189500C000C08091E20680FF28
:105570001FC0459A8FEF80931A048091E20681FF45
:105580001AC0479A8FEF80931B048091E20682FF36
:1055900015C02A988FEF80931C048091E20683FF48
:1055A00010C028988FEF80931D0400C000C008959C
:1055B000459881E0E0CF479881E0E5CF2A9A81E0E5
:1055C000EACF289A81E0EFCF80918803982F977FC8
:1055D00090938803982F937081E011F080E00895F4
:1055E0005E9A08955E98809188038860809388030E
:1055F0000895E82FF0E021E030E0082E02C0220FED
:10560000331F0A94E2F720953095909188039223F6
:1056100090938803EA50FE4F2081922321E019F0F5
:1056200020E0822F0895813079F038F08230C9F778
:10563000159A909177079B7F04C05E9A90917707A7
:105640009E7F90937707EDCF5E9A909177079D7F2D
:10565000F8CF80E0CEDF81E0CCDF82E0CADFB4CFDC
:10566000813079F070F0823071F021E030E001C0DB
:10567000220F8A95EAF780918803822B8093880312
:1056800008955E98F2CF1598F0CFB0E0A0E0EBE47B
:10569000FBE20C9401EBCBE6DDE001E917E08BE7E0
:1056A000A82E8DE0B82EC12CD12C7601C39469911F
:1056B0007991899199910E9417E4288939894A89B9
:1056C0005B890E9478E40E9415ECF8016193719364
:1056D000819391938F01C616D706E806F90610F458
:1056E0006B017C01AC16BD0611F76FEF7FEFCB01AC
:1056F000A70196010E9441EA2093A1073093A207D7
:105700004093A3075093A407CDB7DEB7EAE00C940B
:105710001DEB0F931F93CF93DF930FE71DE0CAEAB2
:10572000D7E0F80121913191419151918F0160E0D1
:1057300070E080E89FE30E94A8EB699379938993D6
:105740009993F7E0CA3BDF0761F70E94E7C09DDF4E
:10575000DF91CF911F910F910895DBCFDACFD9CF91
:10576000D8CF9091391380913A13981306C0809145
:10577000B30D9091B40D892B21F080E00E942C890B
:10578000F0CF08959091391380913A13981307C080
:105790008091B30D9091B40D892B09F45ACF80E01C
:1057A0000E942C89EFCFCF92DF92EF92FF92CF939E
:1057B000DF932091AE02222319F1EC0108960E949A
:1057C000F4746B017C0120E030E0A9010E9413E435
:1057D00020E030E0A901882349F0CE010E946C75D9
:1057E000A70196010E9478E49B01AC016885798548
:1057F0008A859B850E9430EB688779878A879B879B
:10580000DF91CF91FF90EF90DF90CF900895CF92EE
:10581000DF92EF92FF92CF93DF932091AE0222238B
:1058200019F1EC0108960E94F4746B017C0120E0F0
:1058300030E0A9010E9413E420E030E0A9018823B0
:1058400049F0CE010E946C75A70196010E9478E490
:105850009B01AC01688579858A859B850E9431EB27
:10586000688779878A879B87DF91CF91FF90EF9038
:10587000DF90CF900895AEE1B0E0E1E4FCE20C945B
:10588000FBEA9E8F8D8F5B018A01FC01EA5BFF4F73
:105890002081318142815381298B3A8B4B8B5C8BE8
:1058A000CA01B9010E9417E46B017C01D5012D9159
:1058B0003D914D915C910E9478E40E9495EB2B0103
:1058C0003C01F8012081318142815381C701B60139
:1058D0000E9478E40E9495EB4B015C01C301B20188
:1058E0000E9415EC6D8B7E8B8F8B988F68377105BE
:1058F0008105910540F428E730E040E050E02D8B31
:105900003E8B4F8B588FC501B4010E9415EC698FF7
:105910007A8F8B8F9C8F683771058105910540F4D4
:1059200088E790E0A0E0B0E0898F9A8FAB8FBC8FC2
:10593000ED8DFE8DEE5AFF4F2081318142815381E2
:1059400029873A874B875C87CA01B9010E9419E40D
:105950002B013C016D897E898F89988D0E9417E407
:105960006D837E838F83988720E030E0A901C30197
:10597000B2010E9413E4882309F4BBC1A701960178
:10598000C701B6010E9478E44B015C012D813E8184
:105990004F815885CA01B9010E9478E49B01AC018E
:1059A000C501B4010E9430EB4B015C01A3019201DF
:1059B000C301B2010E9431EB9B01AC01C501B401EE
:1059C0000E94A8EB0E9495EB0E9415EC69837A83F4
:1059D0008B839C8369857A858B859C859095809542
:1059E000709561957F4F8F4F9F4F0E9419E44B0137
:1059F0005C01698D7A8D8B8D9C8D0E9417E469877F
:105A00007A878B879C8720E030E0A901C501B4012B
:105A10000E9413E4882309F470C129853A854B85D7
:105A20005C85CA01B9010E9478E46D877E878F8703
:105A3000988BA7019601C701B6010E9478E49B01EB
:105A4000AC016D857E858F8598890E9430EB6B0156
:105A50007C01A5019401C501B4010E9431EB9B01B9
:105A6000AC01C701B6010E94A8EB0E9441ECAD8DCC
:105A7000BE8D95962D913D914D915C9198972D8776
:105A80003E874F87588B69017A0129813A814B8182
:105A90005C81C21AD30AE40AF50A0E9415ECC61A00
:105AA000D70AE80AF90AF7FE8CC02D813E814F81A2
:105AB0005885CA01B9010E9478E46B017C0120E09D
:105AC00030E0A901C301B2010E9413E4882309F464
:105AD00018C16D857E858F8598890E9417E49B018A
:105AE000AC010E9431EBA30192010E9478E44B01CA
:105AF0005C0129853A854B855C85CA01B9010E9404
:105B000078E49B01AC01C501B4010E9431EBA7010F
:105B100096010E9430EB4B015C0120E030E040E850
:105B200050E4C301B2010E9478E49B01AC01C501BD
:105B3000B4010E94A8EB0E9495EB4B015C0120E0B0
:105B400030E0A9010E9494EC87FF03C0812C912CC6
:105B50005401C501B4010E9415EC69837A838B83DB
:105B60009C832D853E854F85588926173707480722
:105B7000590720F429833A834B835C8369817A81B6
:105B80008B819C810E9417E44B015C01A30192016F
:105B9000C301B2010E9431EB9B01AC01C501B4010C
:105BA0000E9478E4A70196010E9431EB0E94CDEC9F
:105BB0000E9415EC698B7A8B8B8B9C8BC12CD12C22
:105BC000760169897A898B899C892D893E894F89DB
:105BD000588D621B730B840B950B0E9417E4A30175
:105BE00092010E94A8EB20E034E244EF59E40E94C5
:105BF00078E40E9415EC4B015C0169897A898B89F4
:105C00009C89298D3A8D4B8D5C8D621B730B840BA7
:105C1000950B0E9417E4A30192010E94A8EB20E0DB
:105C200034E244EF59E40E9478E40E9415EC6D835D
:105C30007E838F839887C501B4010E9481192B014F
:105C40003C016D817E818F8198850E948119298117
:105C50003A814B815C81AD8DBE8D99962D933D939C
:105C60004D935C939C9789019A010C0D1D1D2E1D6F
:105C70003F1DFD0105A716A727A730ABE65BFF4F29
:105C80002D893E894F89588D2083318342835383E8
:105C9000D5968D929D92AD92BC92D8972D813E81E2
:105CA0004F815885D9962D933D934D935C93DC9706
:105CB0003D97408251826282738234966083718301
:105CC0008283938329893A894B895C89D1962D9364
:105CD0003D934D935C93D4973D96298D3A8D4B8D92
:105CE0005C8D20833183428353836E96E0E10C9474
:105CF00017EB60E070E0CB0165CE60E070E0CB01B7
:105D0000B4CE60E070E0CB0116CF90916F0081E0DF
:105D100091FD02C080E0089590916F009D7F909367
:105D20006F000895EFE6F0E080818260808308953F
:105D3000CF93C82FEADF94E0C99F90011124F901A5
:105D4000EC59FB4F20593B4FD9014D915D916D911D
:105D50007C91408351836283738391E090936304C9
:105D60008111E0DFCF910895CF93DF938091E10619
:105D7000811105C08091E306882309F464C08091F5
:105D8000F503329B63C081608093F5038091F50336
:105D9000339B5EC082608093F5038091F503349B52
:105DA00059C084608093F5038091F503029B54C031
:105DB00088608093F503C0915404C0FF0FC08091A8
:105DC000E20680FF0BC08091F50380FF07C0809141
:105DD000760781608093760780E0AADFC1FF0FC05D
:105DE0008091E20681FF0BC08091F50381FF07C01F
:105DF0008091760782608093760781E099DFC2FF09
:105E000022C08091E20682FF1EC08091E3068111CC
:105E10000BC08091F50382FF07C0809176078460F4
:105E20008093760782E084DF8091E306882359F02F
:105E30008091F50383FF07C0809176078860809387
:105E4000760782E075DFDF91CF9108958E7F9CCF3A
:105E50008D7FA1CF8B7FA6CF877FABCF56DF1092F0
:105E6000A5071092A6071092A7071092A807811104
:105E700059CF08950F931F938091391390913A133E
:105E8000891B8F7009F449C090913613992361F0F2
:105E9000833040F48FEF890F29F08093361390E020
:105EA00080E038C01092361380913A132BE5829F20
:105EB000C00111248654984FFC01208120FDEFCFB2
:105EC0004091A5075091A6076091A7077091A80778
:105ED000E95AFF4F0081118122813381401B510B10
:105EE000620B730B4093A5075093A6076093A70717
:105EF0007093A80720913A132F5F2F7020933713C8
:105F000030913A1320913813321304C02091371383
:105F1000209338131F910F910895A0DFC0CFA3E104
:105F2000B0E0E5E9FFE20C94F9EA8FEF9FEF909380
:105F30008900809388002AE02983312C212C7894D1
:105F400080915D0490915E04A0915F04B091600423
:105F5000892B8A2B8B2B09F0C2C180916304882383
:105F6000D1F0809161049091620410926304892BB6
:105F700091F0109262041092610410925404909176
:105F8000391380913A13981731F080913A138F5F4B
:105F90008F7080933A138091610490916204892BF1
:105FA00009F49DC14091590450915A0460915B04D9
:105FB00070915C048091550490915604A09157040F
:105FC000B091580400914B0410E030E020E0841BB5
:105FD000950BA60BB70B081719072A073B0710F4F8
:105FE000D901C8018A8B840F951FA61FB71F809304
:105FF000590490935A04A0935B04B0935C04E1E0CD
:10600000C0902204D0902304E0902404F090250452
:106010008091320490913304A0913404B0913504FE
:10602000C80ED91EEA1EFB1EC0923204D092330461
:10603000E0923404F0923504F7FC33C040911A0426
:10604000042E000C550B660B770B80917004909119
:106050007104A0917204B0917304840F951FA61F60
:10606000B71F8093700490937104A0937204B0934F
:10607000730480911E0490911F04A0912004B0919C
:106080002104B701A601481B590B6A0B7B0BDB01EE
:10609000CA018093320490933304A0933404B093E4
:1060A0003504009126041091270420912804309192
:1060B00029048091360490913704A0913804B0915E
:1060C0003904080F191F2A1F3B1F00933604109331
:1060D0003704209338043093390437FD33C040919E
:1060E0001B04042E000C550B660B770B8091740477
:1060F00090917504A0917604B0917704840F951F58
:10610000A61FB71F8093740490937504A093760420
:10611000B093770480911E0490911F04A0912004F5
:10612000B091210428013901481A590A6A0A7B0AE8
:10613000D301C2018093360490933704A0933804AE
:10614000B093390440912A0450912B0460912C049F
:1061500070912D0480913A0490913B04A0913C04ED
:10616000B0913D04480F591F6A1F7B1F40933A04AA
:1061700050933B0460933C0470933D0477FD33C01F
:1061800080901C04082C000C9908AA08BB08809178
:10619000780490917904A0917A04B0917B04880DE1
:1061A000991DAA1DBB1D8093780490937904A09338
:1061B0007A04B0937B0480911E0490911F04A091F7
:1061C0002004B09121043A014B01681A790A8A0A25
:1061D0009B0AD401C30180933A0490933B04A0939B
:1061E0003C04B0933D0480902E0490902F04A09026
:1061F0003004B090310480913E0490913F04A0910E
:106200004004B0914104880D991DAA1DBB1D8093C7
:106210003E0490933F04A0934004B0934104B7FD23
:1062200033C040901D04042C000C55086608770804
:1062300080907C0490907D04A0907E04B0907F04B8
:10624000840C951CA61CB71C80927C0490927D0443
:10625000A0927E04B0927F0480901E0490901F0450
:10626000A0902004B09021042C013D014818590849
:106270006A087B085301420180923E0490923F04D9
:10628000A0924004B0924104E11104C0E091840066
:10629000F0918500F7FE5F9A37FF469A77FF2B9AB9
:1062A000B7FF299AE0918400F0918500E091840085
:1062B000F0918500F7FE5F9837FF469877FF2B989F
:1062C000B7FF29985A88552021F080918400909139
:1062D00085002A8921502A8BE0E0211191CE8091FE
:1062E0005D0490915E04A0915F04B0916004892BDD
:1062F0008A2B8B2B09F0B0C6409061045090620449
:106300005B8A4A8A4114510409F402C780915904F6
:1063100090915A04A0915B04B0915C0440915504A3
:106320005091560460915704709158048417950752
:10633000A607B70708F449C01092620410926104DE
:10634000109254049091391380913A13981709F4DC
:10635000DFC680913A138F5F8F7080933A13A0ED60
:10636000CA2EA7E0DA2EE12CF12C809161049091E5
:106370006204892B09F068C67DDD909362048093E6
:106380006104892B09F460C6409061045090620456
:106390005B8A4A8AD2018C9183FF08C5C201459667
:1063A0000E94201910926204109261041092540409
:1063B0009091391380913A139817F1F280913A1322
:1063C0008F5F8F7080933A13D7CF409150045091D4
:1063D00051046091520470915304481759076A0799
:1063E0007B0708F40FC240914C0450914D0460911A
:1063F0004E0470914F04EA89FB8985A996A9A7A943
:10640000B0AD481759076A077B0708F0D0C141159E
:1064100051056105710509F066C080908D0390906B
:106420008E03A0908F03B090900385E692E1A1E0E7
:10643000FC010591159125913491081519052A053E
:106440003B0558F4B694A79497948794AA0F0496A2
:10645000E1E8F2E1E817F90759F7A0934B04F0E2FD
:106460008F169104A104B10428F4E0E28E2E912C41
:10647000A12CB12C20E2821A9108A108B108811444
:1064800038E09306A104B10408F49AC1A4E09A9EEE
:10649000C00111248B59914FFC0132962591349102
:1064A000B82DEE27B39F8001B29F010D1E1F0694E9
:1064B0000E1F1E1F112430E020E0FC01C590D49077
:1064C000F12CE12CC01AD10AE20AF30A4C0D5D1D31
:1064D0006E1D7F1D40934C0450934D0460934E04F9
:1064E00070934F0442CF10E00A81942F852E862F9F
:1064F000BC81AD81FE81EF81388529854B80E0919B
:106500008903E99FA12DFF2730918A03399FA00DB0
:10651000F11D10908B03199EF00DE89DA00DF11D4B
:10652000389DF00DE89FF00D4A2EBF2F4A9EE12DB9
:10653000332722274F9EE00D311D211FBA9FE00D0A
:10654000311D211FBF9F300D211D432EB22F4A9EAA
:10655000012D332722274F9E000D311D211FBA9F89
:10656000000D311D211FBF9F300D211D432EB22F65
:10657000EE2790918D0380908E0380918F03009081
:10658000A604012A09F483C03091A204349DE119C4
:10659000910B810A810B2091A304249DE01991099C
:1065A000810A810B0091A404049D90198108810B3C
:1065B0003B9FE0199109810A810B2B9F901981085B
:1065C000810B0B9F801881094A9E012D33272227BA
:1065D0004F9E000D311D211FBA9F000D311D211F3F
:1065E000BF9F300D211D432EB22F30919E04349D4C
:1065F000E10D911F811E811F20919F04249DE00DBC
:10660000911D811E811F0091A004049D900D811C8D
:10661000811F3B9FE00D911D811E811F2B9F900DBF
:10662000811C811F0B9F800C811D4A9E012D3327E9
:1066300022274F9E000D311D211FBA9F000D311DD5
:10664000211FBF9F300D211D432EB22F30919A0480
:10665000349DE119910B810A810B20919B04249DAB
:10666000E0199109810A810B00919C04049D901905
:106670008108810B3B9FE0199109810A810B2B9FB7
:1066800090198108810B0B9F8018810982C030917D
:10669000A204349DE10D911F811E811F2091A3044E
:1066A000249DE00D911D811E811F0091A404049D75
:1066B000900D811C811F3B9FE00D911D811E811F4C
:1066C0002B9F900D811C811F0B9F800C811D4A9E6A
:1066D000012D332722274F9E000D311D211FBA9F08
:1066E000000D311D211FBF9F300D211D432EB22FE4
:1066F00030919E04349DE119910B810A810B209108
:106700009F04249DE0199109810A810B0091A00446
:10671000049D90198108810B3B9FE0199109810A22
:10672000810B2B9F90198108810B0B9F8018810989
:106730004A9E012D332722274F9E000D311D211F18
:10674000BA9F000D311D211FBF9F300D211D432E0B
:10675000B22F30919A04349DE10D911F811E811F4B
:1067600020919B04249DE00D911D811E811F0091AD
:106770009C04049D900D811C811F3B9FE00D911D89
:10678000811E811F2B9F900D811C811F0B9F800CF0
:10679000811D11244B820A83BC83AD83FE83EF836A
:1067A00038872987982C892EB12CA82E3ECEAA890D
:1067B000BB89D1968D909D90AD90BC90D49735CEED
:1067C000D501C401B695A795979587958C7F8B5970
:1067D000954FFC01C590D490FC01329625913491DF
:1067E000E82DE7708E2EE29FC001E39F900D1124EB
:1067F00033E0969587953A95E1F7C81AD90AF12CB6
:10680000E12C64CE409147045091480460914904C2
:1068100070914A04481759076A077B0708F030C28D
:106820008090420490904304A0904404B0904504AA
:1068300080914604EA89FB8981117CC0EF5BFF4FA0
:10684000E080F18002811381EA89FB89E25BFF4FDE
:106850002081318142815381AA89BB89D1966D9172
:106860007D918D919C91D4970E942919B1E0B093AC
:106870004604EA89FB8941A952A963A974A985E65E
:1068800092E1A1E0FC010591159125913491041745
:1068900015072607370758F4769567955795479556
:1068A000AA0F0496E1E8F2E1E817F90759F7A09377
:1068B0004B04403251056105710520F440E250E07F
:1068C00060E070E040525109610971094115F8E03A
:1068D0005F076105710508F4B3C124E0529FC00150
:1068E00011248B59914FFC01329625913491AA279E
:1068F000439FF001429FE10DFA1F0694EA1FFA1F21
:106900001124AF0170E060E0FC01C590D490F12C3F
:10691000E12CC41AD50AE60AF70A8C0C9D1CAE1CA1
:10692000BF1C8092420490924304A0924404B0920F
:1069300045041BCD81AD92ADA3ADB4AD88169906CB
:10694000AA06BB0608F072C181149104A104B10427
:1069500049F440918D0350918E0360918F037091A3
:1069600090038DCFA0E0BA85982D492D8A2DFB8507
:10697000EC857D856E855F853889298950918903ED
:10698000599F712D662730918A03399F700D611DC3
:1069900010908B03199E600D549F700D611D349FE4
:1069A000600D589F600DF72FE62FF79F512D33276D
:1069B0002227F69F500D311D2A1FE79F500D311DD4
:1069C0002A1FE69F300D211DF32FE22FF79FB12DD7
:1069D00033272227F69FB00D311D2A1FE79FB00DE8
:1069E000311D2A1FE69F300D211DF32FE22F552761
:1069F00090918D0340918E0380918F030090A604A7
:106A00000A2A09F483C03091A2043F9F51199A0BBE
:106A10004A0B8A0B2091A3042F9F501991094A0B0E
:106A20008A0BB091A404BF9F901941098A0B3E9F25
:106A3000501991094A0B8A0B2E9F901941098A0B14
:106A4000BE9F40198109F79FB12D33272227F69F5A
:106A5000B00D311D2A1FE79FB00D311D2A1FE69F83
:106A6000300D211DF32FE22F30919E043F9F510DD9
:106A70009A1F4A1F8A1F20919F042F9F500D911D1E
:106A80004A1F8A1FB091A004BF9F900D411D8A1F0D
:106A90003E9F500D911D4A1F8A1F2E9F900D411D34
:106AA0008A1FBE9F400D811DF79FB12D33272227DE
:106AB000F69FB00D311D2A1FE79FB00D311D2A1F13
:106AC000E69F300D211DF32FE22F30919A043F9F56
:106AD00051199A0B4A0B8A0B20919B042F9F501936
:106AE00091094A0B8A0BB0919C04BF9F90194109F0
:106AF0008A0B3E9F501991094A0B8A0B2E9F9019C1
:106B000041098A0BBE9F4019810982C03091A204BD
:106B10003F9F510D9A1F4A1F8A1F2091A3042F9F48
:106B2000500D911D4A1F8A1FB091A404BF9F900D64
:106B3000411D8A1F3E9F500D911D4A1F8A1F2E9F87
:106B4000900D411D8A1FBE9F400D811DF79FB12DE5
:106B500033272227F69FB00D311D2A1FE79FB00D66
:106B6000311D2A1FE69F300D211DF32FE22F30919A
:106B70009E043F9F51199A0B4A0B8A0B20919F0448
:106B80002F9F501991094A0B8A0BB091A004BF9F07
:106B9000901941098A0B3E9F501991094A0B8A0BA3
:106BA0002E9F901941098A0BBE9F40198109F79FBA
:106BB000B12D33272227F69FB00D311D2A1FE79FE5
:106BC000B00D311D2A1FE69F300D211DF32FE22F3E
:106BD00030919A043F9F510D9A1F4A1F8A1F20919E
:106BE0009B042F9F500D911D4A1F8A1FB0919C043A
:106BF000BF9F900D411D8A1F3E9F500D911D4A1F42
:106C00008A1F2E9F900D411D8A1FBE9F400D811D22
:106C10001124BA87FB87EC877D876E875F87388B67
:106C2000298B542F492F70E0682F29CE2A893B8960
:106C3000225B3F4FD9014D915D916D917C911FCEAB
:106C4000DB01CA01B695A795979587958C7F8B59DF
:106C5000954FFC01C590D490FC013296259134915A
:106C60004770429FC001439F900D1124A3E0969569
:106C70008795AA95E1F7C81AD90AF12CE12C4DCED7
:106C800080912E0190912F01A0913001B09131019E
:106C9000B7FF61C0EA89FB89EA5BFF4FC080D18002
:106CA000E280F38085E692E121E0FC014591559177
:106CB000659174914C155D056E057F0558F4F69449
:106CC000E794D794C794220F049641E852E14817FD
:106CD000590759F720934B0450E2C516D104E1043B
:106CE000F10428F470E2C72ED12CE12CF12C60E2E3
:106CF000C61AD108E108F108C11478E0D706E1040A
:106D0000F10408F431C0A4E0DA9EC00111248B59CB
:106D1000914FFC01329625913491BC2D6627B39F8B
:106D2000A001B29F410D561F0694461F561F112405
:106D300070E060E0FC0185919491B0E0A0E0841BDC
:106D4000950BA60BB70B80932E0190932F01A09368
:106D50003001B0933101C0902E01D0902F01E0900E
:106D60003001F090310101CBD701C601B695A7954E
:106D7000979587958C7F8B59954FFC012591349180
:106D8000FC01329645915491EC2DE770E49FC001CF
:106D9000E59F900D112463E0969587956A95E1F73C
:106DA000281B390BC901B0E0A0E0CDCFEA89FB89EF
:106DB00085889688A788B08C81E081149104A1040D
:106DC000B10409F480E0AA89BB895996CD90DD9081
:106DD000ED90FC905C97C114D104E104F10409F03A
:106DE0008260EA89FB89458D568D678D70A14115BA
:106DF00051056105710509F0846080935404109277
:106E000042041092430410924404109245041092DC
:106E10004C0410924D0410924E0410924F04EA89D3
:106E2000FB8985A196A1A7A1B0A580935504909355
:106E30005604A0935704B0935804442455243201B7
:106E4000481A590A6A0A7B0A409232045092330463
:106E500060923404709235044092360450923704A4
:106E6000609238047092390440923A0450923B0484
:106E700060923C0470923D0441A052A063A074A0B3
:106E8000440C551C661C771C880C991CAA1CBB1C46
:106E90008092220490922304A0922404B0922504AC
:106EA000CC0CDD1CEE1CFF1CC0922604D0922704E3
:106EB000E0922804F0922904440F551F661F771FA3
:106EC00040932A0450932B0460932C0470932D0458
:106ED00040922E0450922F0460923004709231043C
:106EE000880F991FAA1FBB1F80931E0490931F0435
:106EF000A0932004B09321041092590410925A04D4
:106F000010925B0410925C0481A592A5A3A5B4A580
:106F10008093500490935104A0935204B09353046F
:106F200085A596A5A7A5B0A980934704909348048A
:106F3000A0934904B0934A04EB5BFF4F808190918A
:106F4000E206891721F08093E2060E94B32A0E948C
:106F5000B42E44244A94542C320140922E01509273
:106F60002F016092300170923101EA89FB89FD9610
:106F7000E080F18002811381AA89BB89D1962D918D
:106F80003D914D915C91D4976D01BAE4CB0ED11C2B
:106F9000F60160817181828193810E94291910928A
:106FA0004604D6014D915D916D917C9185E692E10B
:106FB000A1E0FC0105911591259134910417150765
:106FC0002607370758F47695679557954795AA0F82
:106FD0000496E1E8F2E1E817F90759F7A0934B04AA
:106FE000403251056105710520F440E250E060E057
:106FF00070E040525109610971094115F8E05F07DD
:107000006105710508F462C024E0529FC00111249B
:107010008B59914FFC01329625913491AA27439FB9
:10702000F001429FE10DFA1F0694EA1FFA1F112496
:10703000AF0170E060E0FC01C590D490F12CE12C30
:10704000C41AD50AE60AF70AC0925D04D0925E041B
:10705000E0925F04F092600480915D0490915E0480
:10706000A0915F04B0916004AC01BD01009731E0D4
:10707000A307B10520F04FEF5FEF60E070E0841BE5
:10708000950BA60BB70B80935D0490935E04A093C1
:107090005F04B0936004F89480918400909185001F
:1070A0004096A981A150A983AA2381F1240E351EFF
:1070B0002816390610F40C949F2F309289002092E4
:1070C000880078946396E2E10C9415EBDB01CA0129
:1070D000B695A795979587958C7F8B59954FFC0111
:1070E000C590D490FC013296259134914770429F0F
:1070F000C001439F900D112433E0969587953A95F2
:10710000E1F7C81AD90AF12CE12C9ECF1C01D5CF8A
:1071100080EDC82E87E0D82EE12CF12C2DC9CF931D
:10712000DF938091391390913A13891B80958F706A
:1071300019F40E942C89F5CF809139138F5F8F70DD
:10714000A09139139BE5A99FD0011124FD01E654BC
:10715000F84FEF0119929A95E9F798E09083A153BF
:10716000B84F90E1EBE3F3E101900D929A95E1F7CE
:107170002091391390913A13291303C094E6909308
:107180003613809339130E94922EDF91CF91089588
:10719000FC01208131814281538160918B0D70917E
:1071A0008C0D80918D0D90918E0D0E9478E40E943F
:1071B00099EC60934713709348138093491390930D
:1071C0004A139091391380913A13981709F0A7CF79
:1071D0000E94B12B0E94852E409147135091481375
:1071E0006091491370914A1340937C0450937D043D
:1071F00060937E0470937F0481110C94922E089505
:107200004F925F926F927F928F929F92AF92BF92B6
:10721000CF92DF92EF92FF92CF93DF93EC01209118
:107220008B0D30918C0D40918D0D50918E0D6C8594
:107230007D858E859F850E9478E40E9499EC6B0184
:107240007C012091870D3091880D4091890D5091DE
:107250008A0D688579858A859B850E9478E40E94DD
:1072600099EC4B015C012091830D3091840D40918C
:10727000850D5091860D6C817D818E819F810E944C
:1072800078E40E9499EC2B013C0120917F0D309114
:10729000800D4091810D5091820D688179818A81A4
:1072A0009B810E9478E40E9499EC60933B13709359
:1072B0003C1380933D1390933E1340923F135092A2
:1072C0004013609241137092421380924313909244
:1072D0004413A0924513B0924613C0924713D09224
:1072E0004813E0924913F0924A1390913913809118
:1072F0003A13981781F013DFDF91CF91FF90EF9051
:10730000DF90CF90BF90AF909F908F907F906F90C5
:107310005F904F9008950E94B12B0E94852EC82F38
:107320008BE393E10E942019CC2331F30E94922E2B
:10733000E3CFCF92DF92EF92FF92CF93DF93C82FEC
:107340000E94852E94E0C99FE0011124FE01E059BE
:10735000FB4FC080D180E280F38081110E94922E89
:10736000C655D84FC701B6010E9419E4288139815A
:107370004A815B810E9478E4DF91CF91FF90EF908A
:10738000DF90CF900895CF92DF92EF92FF92CF934C
:10739000DF93C82F0E94852E94E0C99FE00111243D
:1073A000FE01EC59FB4FC080D180E280F380811157
:1073B0000E94922EC655D84FC701B6010E9419E40B
:1073C000288139814A815B810E9478E4DF91CF91E5
:1073D000FF90EF90DF90CF900895A1E0B0E0E3EF51
:1073E000F9E30C9409EB898360E0CE0101960E94D9
:1073F0007B1A61E0CE0101960E947B1A62E0CE0109
:1074000001960E947B1A89812196E2E00C9425EB7B
:10741000A2E1B0E0EEE0FAE30C9405EBDEDF8823B6
:10742000C1F1EDB6FEB64DE852E082FF02C044E87D
:1074300052E02DE832E081FF02C026E832E080FD14
:1074400025C08DE892E05F934F933F932F939F93D6
:107450008F938AED96E09F938F938E010F5F1F4F5E
:107460001F930F930E94ACE30E94EF85C8010E9416
:107470009E7FC8010E9450BF0FB6F894DEBF0FBEBA
:10748000CDBF81E06296E6E00C9421EB88E892E0C3
:10749000DACF80E0F7CFA0E2B0E0E1E5FAE30C94C8
:1074A000F9EA80911201882309F4BEC08091080492
:1074B000082F10E080FF3CC0C0901401D09015014F
:1074C000E0901601F090170120919E0230919F02EA
:1074D0004091A0025091A102C701B6010E9494EC14
:1074E000181644F4C0929E02D0929F02E092A0022D
:1074F000F092A102C0902001D0902101E0902201E1
:10750000F090230120919E0230919F024091A002B1
:107510005091A102C701B6010E9413E487FF08C081
:10752000C0929E02D0929F02E092A002F092A1022D
:1075300001FF3CC0C0901801D0901901E0901A01E1
:10754000F0901B012091A2023091A3024091A4026D
:107550005091A502C701B6010E9494EC181644F49C
:10756000C092A202D092A302E092A402F092A502DD
:10757000C0902401D0902501E0902601F0902701D1
:107580002091A2023091A3024091A4025091A50241
:10759000C701B6010E9413E487FF08C0C092A2028F
:1075A000D092A302E092A402F092A50202FF3CC096
:1075B000C0901C01D0901D01E0901E01F0901F01B1
:1075C0002091A6023091A7024091A8025091A902F1
:1075D000C701B6010E9494EC181644F4C092A602AA
:1075E000D092A702E092A802F092A902C0902801CE
:1075F000D0902901E0902A01F0902B012091A60261
:107600003091A7024091A8025091A902C701B6018A
:107610000E9413E487FF08C0C092A602D092A7027E
:10762000E092A802F092A90280916A0D83FD61C0E8
:107630002091810130918201409183015091840118
:107640006091AA027091AB028091AC029091AD0260
:107650000E9413E4882309F44CC00E94A3B0182FA1
:10766000882331F00E94EF858FEB96E00E94AD7F7A
:1076700020918101309182014091830150918401D8
:107680006091AA027091AB028091AC029091AD0220
:107690000E9430EB9F7720916F01309170014091F3
:1076A0007101509172010E9478E420E030E046E1DF
:1076B00054E40E9494EC1816D4F40E94EF8580EAFA
:1076C00096E00E94AD7F8091AA029091AB02A091BA
:1076D000AC02B091AD028093810190938201A0939E
:1076E0008301B09384018AEA92E052DD02C0111155
:1076F000EACF2AE037ED43E25CE360910C01709140
:107700000D0180910E0190910F010E9478E46B01B0
:107710007C016091100170911101072E000C880B03
:10772000990B0E9419E49B01AC01C701B6010E94AC
:1077300078E4698B7A8B8B8B9C8B8091AE0288234B
:1077400009F18090AF029090B002A090B102B09089
:10775000B202C090A602D090A702E090A802F090DA
:10776000A90220E030E0A901C501B4010E9413E4A0
:107770008823F9F0A7019601C501B4010E9494EC99
:107780001816BCF020E030E0A901BE016F5E7F4F0B
:107790008EE992E00E94C4C080E1EEE9F2E0A5E744
:1077A000B1E001900D928A95E1F7A096E2E10C9488
:1077B00015EB209175013091760140917701509140
:1077C000780160919E0270919F028091A002909139
:1077D000A1020E9430EB4B015C01209179013091B4
:1077E0007A0140917B0150917C016091A2027091DD
:1077F000A3028091A4029091A5020E9430EB6D8BB0
:107800007E8B8F8B988F20917D0130917E014091EE
:107810007F0150918001C701B6010E9430EB6D8F4E
:107820007E8F8F8F98A320918101309182014091AA
:107830008301509184016091AA027091AB02809102
:10784000AC029091AD020E9430EB698F7A8F8B8FE2
:107850009C8F20E030E0A901C501B4010E9413E42F
:1078600081110CC020E030E0A9016D897E898F89EB
:10787000988D0E9413E4882309F484CFA501940114
:10788000C501B4010E9478E46B017C012D893E8919
:107890004F89588DCA01B9010E9478E49B01AC015F
:1078A000C701B6010E9431EB6B017C012D8D3E8D2D
:1078B0004F8D58A1CA01B9010E9478E49B01AC0127
:1078C000C701B6010E9431EB6B017C01298D3A8D15
:1078D0004B8D5C8DCA01B9010E9478E49B01AC011B
:1078E000C701B6010E9431EB6B017C010E94CDEC17
:1078F0002B013C012CEC3CEB4CE85BE2C701B601F0
:107900000E9413E487FF06C0498C5A8C6B8C7C8CD8
:10791000E89477F82DEB37E346E855E3C301B2016D
:107920000E9413E487FD38CF2DEC3CEC4CE45EE381
:10793000C301B2010E9478E40E9415EC1B01672B81
:1079400019F422242394312CB10190E080E00E94AC
:1079500017E49B01AC0160E070E080E89FE30E94C7
:10796000A8EB6B017C01AC019B01C301B2010E9439
:1079700078E42B013C01A7019601C501B4010E94E6
:1079800078E44B015C01A70196016D897E898F899E
:10799000988D0E9478E46D8B7E8B8F8B988FA701DA
:1079A00096016D8D7E8D8F8D98A10E9478E46D8FEC
:1079B0007E8F8F8F98A3A7019601698D7A8D8B8D0D
:1079C0009C8D0E9478E4698F7A8F8B8F9C8F80E1E9
:1079D000E5E7F1E08E010F5F1F4FD80101900D9296
:1079E0008A95E1F70E9400CB6B017C0128ECC20E66
:1079F000D11CE11CF11C81E0281A310809F454C0A3
:107A00000E9400CB9B01AC012C193D094E095F0976
:107A100057FD4DC06B017C0128ECC20ED11CE11C4E
:107A2000F11C80E00E942C89A501940169817A8172
:107A30008B819C810E9431EB69837A838B839C8349
:107A40002D893E894F89588D6D817E818F819885E2
:107A50000E9431EB6D837E838F8398872D8D3E8DC1
:107A60004F8D58A169857A858B859C850E9431EB65
:107A700069877A878B879C87298D3A8D4B8D5C8DA2
:107A80006D857E858F8598890E9431EB6D877E8715
:107A90008F87988BA3019201BE016F5E7F4FC80153
:107AA0000E94C4C08111A7CFA30192016ECE0E9493
:107AB000F328BACF8091040490910504A0910604A4
:107AC000B091070480930C0190930D01A0930E01D7
:107AD000B0930F01809102049091030490931101DF
:107AE00080931001089580910C0190910D01A09157
:107AF0000E01B0910F018093040490930504A093AC
:107B00000604B093070480911001909111019093A5
:107B100003048093020484E690E090931101809323
:107B200010010895ACE0B0E0E8E9FDE30C94FBEA55
:107B30002B013C0129873A874B875C874701580115
:107B4000D601CD90DD90ED90FC9020E030E0A901D1
:107B5000C701B6010E9413E4811171C080916B01CD
:107B600090916C01A0916D01B0916E0189839A830F
:107B7000AB83BC8320E030E0A901C701B6010E94BD
:107B800013E4811106C0C12CD12C80E8E82E80E4DA
:107B9000F82ECD82DE82EF82F886A50194016091F5
:107BA0007D0170917E0180917F01909180010E9402
:107BB00013E487FF0CC080927D0190927E01A09219
:107BC0007F01B0928001CE0105960E94BA214092B9
:107BD00075015092760160927701709278018985E3
:107BE0009A85AB85BC858093790190937A01A093A7
:107BF0007B01B0937C01CE0101960E94BA21A501C0
:107C0000940160917D0170917E0180917F0190913E
:107C100080010E9494EC181664F480927D01909289
:107C20007E01A0927F01B0928001CE0105960E9454
:107C3000BA210E94B12B2C96E0E10C9417EBD701EE
:107C4000C60194CFCF92DF92EF92FF920F931F93D2
:107C50006B01FC01E080F18002811381E5E7F1E036
:107C60002481358146815781608171818281938130
:107C700059DF1F910F91FF90EF90DF90CF90089503
:107C80008F929F92AF92BF92CF92DF92EF92FF922C
:107C90001F93CF93DF93CDB7DEB760970FB6F894FD
:107CA000DEBF0FBECDBF182F80E043DB4B015C0170
:107CB0008092F6039092F703A092F803B092F90332
:107CC00081E037DB6B017C01C092FA03D092FB03A9
:107CD000E092FC03F092FD0382E02BDB6093FE0355
:107CE0007093FF0380930004909301041D861E8609
:107CF0001F86188A89829A82AB82BC82CD82DE82FC
:107D0000EF82F88669877A878B879C8783E011DB0F
:107D10006D877E878F87988BCE0101960E94D32B2B
:107D20001E3FD9F480E1FE013196A5E7B1E0019054
:107D30000D928A95E1F760960FB6F894DEBF0FBEFC
:107D4000CDBFDF91CF911F91FF90EF90DF90CF904B
:107D5000BF90AF909F908F90089584E0189FF0019E
:107D60001124DF01AB58BE4F81E090E08C0F9D1FC6
:107D7000E80FF91F40815181628173814D935D93BA
:107D80006D937C931397D7CF0C94E7C0CF930E9449
:107D9000852EC82F80913A1380933913809338131E
:107DA0008093371384E6809336130E942E2F80ED44
:107DB00093E09093B40D8093B30DC1110E94922E65
:107DC00081E0809363040E94B12B8EEF59DFDCDFEA
:107DD000CF910895ACE0B0E0E0EFFEE30C9409EB46
:107DE0000E9462B00E94852E9CE0E0E7F4E0DE0194
:107DF000119601900D929A95E1F781110E94922EB1
:107E0000CE0101960E942B2A2C96E2E00C9425EBE1
:107E1000B0E0A0E0EEE0FFE30C94FBEA40907501D7
:107E20005090760160907701709078018090790190
:107E300090907A01A0907B01B0907C01C0907D0170
:107E4000D0907E01E0907F01F09080010E94452B50
:107E500060912C0170912D01072E000C880B990B5D
:107E60000E9419E42AE037ED43E25CE30E9478E4E3
:107E700060936F0170937001809371019093720110
:107E800004E111E0D0E0C0E0CE01875E954F0E9492
:107E9000EE74F80161937193819391938F01CE01F8
:107EA000835F954F0E94EE74F80160877187828727
:107EB00093872496CC30D10539F760E086E194E0D1
:107EC0000E94CF770E949C780E94892BA301920187
:107ED00060917501709176018091770190917801A0
:107EE0000E9413E481111BC0A501940160917901E6
:107EF00070917A0180917B0190917C010E9413E442
:107F000081110DC020917D0130917E0140917F0152
:107F100050918001C701B6010E9413E481115ADF1C
:107F2000CDB7DEB7E0E10C9417EB86E896E00E944F
:107F3000AD7F86B160E876E082FB882780F90E94F9
:107F4000A72186B16AE776E083FB882780F90E9443
:107F5000A72186B164E776E0829581700E94A7210F
:107F600080B16CE676E082FB882780F90C94A7212B
:107F70008091E106811103C08091E30681110C9488
:107F8000B42E0895ACE0B0E0E8ECFFE30C9409EB0C
:107F9000ABE6BDE090E080E0FC01EB5AF54F459187
:107FA0005591659174914D935D936D937D93FC0113
:107FB000EB5BF54F459155916591749150964D93BA
:107FC0005D936D937C935397FC01EB5CF54F45916A
:107FD00055916591749190964D935D936D937C93BB
:107FE0009397049680319105B9F680E29EE4A0E073
:107FF000B0E080937B0D90937C0DA0937D0DB093AA
:108000007E0D80E090E0AAEFB3E480939F0D909303
:10801000A00DA093A10DB093A20D8093A30D9093FA
:10802000A40DA093A50DB093A60D8093A70D9093DA
:10803000A80DA093A90DB093AA0D1092AB0D1092AC
:10804000AC0D1092AD0D1092AE0D1092AF0D1092BE
:10805000B00D1092B10D1092B20D8AE097EDA3EA27
:10806000BDE380938D0790938E07A0938F07B09305
:10807000900780E090E0A0E2B1E480931604909332
:108080001704A0931804B09319040E9485778CE01C
:10809000E5E8F1E0DE01119601900D928A95E1F795
:1080A00089819A81AB81BC81809328139093291395
:1080B000A0932A13B0932B138D819E81AF81B88535
:1080C00080932C1390932D13A0932E13B0932F1302
:1080D00089859A85AB85BC85809330139093311345
:1080E000A0933213B09333138EEB90E09093430739
:1080F000809342078CE390E0909345078093440778
:10810000109247071092460786EE90E09093490739
:108110008093480786E490E090934B0780934A074A
:1081200010924D0710924C078FE892ECADE8B1E445
:108130008093B7129093B812A093B912B093BA1269
:108140008CE998EFA5E4BEE38093BB129093BC1238
:10815000A093BD12B093BE1281E49CEBABECB3E4F0
:108160008093BF129093C012A093C112B093C21219
:1081700080E090E0AFEAB3E480933607909337074E
:10818000A0933807B093390785E996E2A5E2B1E4F8
:1081900080933A0790933B07A0933C07B0933D0729
:1081A00080EA9CE6ACE2B5E480933E0790933F07FB
:1081B000A0934007B09341071092E1061092E006A9
:1081C000D7DE26DE2C96E2E00C9425EB8091760734
:1081D000882319F010927607089540E070E060E07F
:1081E0008CE496E00E9441881F920F920FB60F9286
:1081F00011240BB60F922F933F934F935F936F937E
:108200007F938F939F93AF93BF93EF93FF930E94BE
:10821000B42EFF91EF91BF91AF919F918F917F917C
:108220006F915F914F913F912F910F900BBE0F90E7
:108230000FBE0F901F9018950F931F938091870783
:10824000813019F50E9400CB0091ED031091EE03EF
:108250002091EF033091F003601B710B820B930BA5
:1082600028EE33E040E050E00E9441EA6091E903EB
:108270007091EA038091EB039091EC03620F731FFE
:10828000841F951F1F910F9108956091F1037091C4
:10829000F2038091F3039091F403D6CF10928707F5
:1082A0001092ED031092EE031092EF031092F00380
:1082B0001092F1031092F2031092F3031092F40360
:1082C0001092E9031092EA031092EB031092EC0370
:1082D0000895809187078130E1F08230C1F4ACDFEE
:1082E0006093E9037093EA038093EB039093EC03AC
:1082F00081E0809387070E9400CB6093ED03709329
:10830000EE038093EF039093F00381E00895C6DFBE
:10831000EFCF80E008950E9478C10E9436798823CB
:1083200051F08091B71482FD06C087EE91E09093E2
:10833000E5068093E406CDCF80918707813079F4FC
:1083400082E0809387070E9400CB6093F1037093D3
:10835000F2038093F3039093F40381E0089580E0A7
:108360000895809187078150823070F410928707BA
:108370000E9400CB6093F1037093F2038093F303A8
:108380009093F40381E0089580E008952091B41261
:108390003091B512263531053CF4209133073091E8
:1083A0003407263031051CF0882331F092CF662344
:1083B00019F0D7DF0C9478C108959C0197FF26C06F
:1083C000EE27FF27E81BF90B2D398FEF38070CF04C
:1083D0005DC08DE280939902CF0164E670E00E9457
:1083E000A9EACB012AE030E0B9010E94A9EA805D48
:1083F00080939A02CF01B9010E94A9EACB01B90189
:108400000E94A9EA805D80939B022AC0283E83E0F7
:108410003807B4F1C90168EE73E00E94A9EACB0104
:10842000EAE0F0E0BF010E94A9EA805D8093990232
:10843000C90164E670E00E94A9EACB01BF010E9475
:10844000A9EA805D80939A02C901BF010E94A9EA4E
:10845000CB01BF010E94A9EA805D80939B02F901D4
:10846000CF016AE070E00E94A9EA805D80939C02DF
:1084700089E992E008958DE237FDC5CF80E2C3CF50
:10848000F90180E2243631050CF0A4CF80E280931C
:10849000990280939A02EA30F1056CF38DE237FF7E
:1084A00080E280939A02CF016AE070E00E94A9EA1C
:1084B000605D60939B02D4CF9C0197FD2DC080E24C
:1084C000243631055CF0C90164E670E00E94A9EA37
:1084D000CB016AE070E00E94A9EA805D80939A0275
:1084E00080E22A3031055CF0EAE0F0E0C901BF012A
:1084F0000E94A9EACB01BF010E94A9EA805D809396
:108500009B02C9016AE070E00E94A9EA805D809345
:108510009C028AE992E008953195219531098DE216
:10852000DDCFCF92DF92EF92FF92FC01C080D1802D
:10853000E280F38020E030E0A901C701B6010E948B
:1085400013E487FD26C06DEB77E386E095E3A70192
:1085500096010E9431EB6B017C0120E030E0A90123
:108560000E9413E420E030E040E05FE387FF04C0B6
:1085700020E030E040E05FEBC701B6010E9431EB44
:108580000E9410ECCB0198DFFF90EF90DF90CF902E
:1085900008956DEB77E386E095EBD9CFA4E0B0E0EA
:1085A000E4EDF2E40C9409EB0E9419E469837A8308
:1085B0008B839C83CE010196B4DF2496E2E00C9479
:1085C00025EBFC0160817181828193810E9410EC16
:1085D000CB0172CFA4E0B0E0E0EFF2E40C9409EB41
:1085E0000E9419E469837A838B839C83CE01019670
:1085F000E8DF2496E2E00C9425EB0F931F930E9492
:1086000000CB0091DA061091DB062091DC06309158
:10861000DD060115110521053105D9F520914D1310
:108620002223A1F1E0914B13215020934D1321E01F
:108630002E0F20934B1330914E13231302C0109230
:108640004B1324E0E29FF0011124E15BFC4E00811A
:108650001181228133810093D6061093D70620938F
:10866000D8063093D906600F711F811D911D60934C
:10867000DA067093DB068093DC069093DD0680912A
:10868000D8069091D906892B09F0149A1F910F9161
:108690000895601B710B820B930B97FDF7CF149815
:1086A0001092DA061092DB061092DC061092DD06BC
:1086B000EDCF0F931F93CF93DF938C01EB0190913C
:1086C0004D1320914E13921304C097DF0E94F3289C
:1086D000F6CF80914C1334E0839FF0011124E15BCD
:1086E000FC4E11830083D383C2839F5F90934D130D
:1086F0008F5F281739F080934C13DF91CF911F9132
:108700000F91089510924C13F8CF882351F063E92C
:1087100072E084E690E0CDDF6AEB72E084E690E000
:10872000C8CF68EB71E084E190E0FACF2BDC81E008
:10873000ECCF8F929F92AF92BF92EF92FF920F93E6
:108740001F93CF93DF93EC018B01E42EF22E8091E7
:108750005F13909160138C179D07C9F120E6C53B0C
:10876000D20709F03FC08454994771F40E9400CBAE
:108770006E517B4F8F4F9F4F6093D9037093DA03F5
:108780008093DB039093DC03D0936013C0935F135B
:1087900030E020E00093690710936A0720936B078D
:1087A00030936C07E0926407F0926507C454D94790
:1087B00021F4109295021092D80382E080936A010E
:1087C00081E080936607109294021092E403DF9197
:1087D000CF911F910F91FF90EF90BF90AF909F901E
:1087E0008F90089529E7C434D20771F6855B9046CF
:1087F000D9F40E9400CB8090D9039090DA03A09026
:10880000DB03B090DC03681979098A099B0997FF9B
:108810000BC0809177078770873031F40E947922EE
:10882000CAE1D4E58111B0CFC4E4D9E7ADCF20E0EF
:1088300040E070E060E088E692E27BCF0E94A3B067
:10884000882339F020E040E070E060E08CE393E5BD
:1088500070CFEDCF21E020939502FC0180819181C2
:10886000A281B3818093080190930901A0930A012A
:10887000B0930B0120E040E070E060E0809153078E
:108880009091540756CFA4E0B0E0E9E4F4E40C94EE
:1088900009EB8DEC9CECACECBCE389839A83AB8355
:1088A000BC83CE010196D6DF2496E2E00C9425EB42
:1088B000A4E0B0E0EEE5F4E40C9409EB8DEC9CEC64
:1088C000ACECBDE389839A83AB83BC83CE01019674
:1088D000C1DF2496E2E00C9425EBA4E0B0E0E3E7EE
:1088E000F4E40C9409EB80E090E0A0E8BFE3898316
:1088F0009A83AB83BC83CE010196ACDF2496E2E081
:108900000C9425EBA4E0B0E0E8E8F4E40C9409EB67
:1089100080E090E0A0E2B1E489839A83AB83BC83DA
:10892000CE01019697DF2496E2E00C9425EB81E0DE
:1089300080939502809177078770873051F010926D
:1089400077071092080486EB95E09093E5068093F4
:10895000E4068091AE028093E60380E00E944377B4
:1089600020E040E070E060E087EB94E4E2CE8091AC
:108970006A01882331F041E062EA73E082E00E94FC
:108980006BC5809108048770873071F41092E503FD
:1089900020E040E070E060E08CEB93E5CADE81E02F
:1089A0008093E4030C94C221089520E040E070E03D
:1089B00060E084E499E7BDCE1092A9070E94F826F2
:1089C000F4CFB0E0A0E0E7EEF4E40C9403EBCDB616
:1089D000DEB6EAE7F7E0DF010D900020E9F7CD0110
:1089E000825797402DB73EB7281B390B0FB6F89426
:1089F0003EBF0FBE2DBF0DB71EB70F5F1F4FFF93BA
:108A0000EF9389E195E09F938F931F930F930E94BB
:108A1000ACE3780134E0E30EF11C0F900F900F905F
:108A20000F900F900F90D7018D917D01882349F011
:108A3000082E000C990B0E9412EDF70131978083EC
:108A4000F2CF64E175E0C8010E9445E34FE350E0D6
:108A5000B80186EE96E00E946AED0FB6F894DEBE8D
:108A60000FBECDBEA2DF0E9478C1E8E00C941FEBE0
:108A70008093270720E040E070E060E08AED93E516
:108A800058CEA2E8B0E0E7E4F5E40C94F9EAADB61C
:108A9000BEB684E690E09093A01280939F1210924D
:108AA000C4121092C31241E064E070E0CE01875816
:108AB0009F4F0E94AAAF43E050E0BE0167587F4F2E
:108AC00082E292E00E945CED892BF9F0ED968FAD89
:108AD000ED97882339F08FE3EA968FAFEA97EB960C
:108AE0001FAEEB9782E0C4DF81E080931504909184
:108AF000150481E089270FB6F894BEBE0FBEADBE47
:108B0000CE57DF4FE2E10C9415EB41E062E070E0FC
:108B1000CE0183589F4F0E94AAAFE9961CAE1DAEAE
:108B20001EAE1FAEE9971092C4121092C312CE016E
:108B30008F579F4F0E948121EDB6FEB6CF57DF4F72
:108B4000C880C158D040D12C23E0C20ED11CCC0C1F
:108B5000DD1CCC0CDD1C8DB79EB78C199D090FB6A2
:108B6000F8949EBF0FBE8DBFEDB7FEB731963F01A3
:108B70008C199D090FB6F8949EBF0FBE8DBFEDB73F
:108B8000FEB731964F018C199D090FB6F8949EBF20
:108B90000FBE8DBF0DB71EB70F5F1F4FB601C301CC
:108BA0000E9486214091870381E0482764E070E0BD
:108BB0008BE79DE00E94AAAFB601C4010E94862106
:108BC000B601C8010E94862190918703CE57DF4FDE
:108BD0009883C258D04091114BC0CF57DF4F888146
:108BE000C158D04090E00296ABE6BDE050E040E0D6
:108BF00030E020E061E67AE0E1E5CE2EEAE0DE2E2C
:108C0000821793070CF495C0F301E40FF51F208041
:108C10003180428053802D923D924D925D92821719
:108C200093070CF48CC0F401E40FF51F2080318011
:108C30004280538050962D923D924D925C92539774
:108C4000821793070CF481C0F801E40FF51F208010
:108C500031804280538090962D923D924D925C924D
:108C600093972F5F3F4F4C5F5F4F2430310541F6A4
:108C70008FE99DE00E94592183EA9DE00E945921DD
:108C800087EA9DE00E9459218BEA9DE00E945921CC
:108C90008FEA9DE00E945921CE018B589F4F0E9480
:108CA0005921CE018B589F4F0E945921CE018B58DC
:108CB0009F4F0E945921CE018B589F4F0E945921EE
:108CC0008DE897E00E9459210FB6F894FEBE0FBEC2
:108CD000EDBE8E010F5F1F4FC8010E947921CE01AA
:108CE00083599F4F0E946121C8010E94592186E14A
:108CF00094E00E945921CE018B589F4F0E94592128
:108D0000CE0183599F4F0E948121C8010E94812179
:108D1000AE96CFACAE978981C89E60011124E1E088
:108D2000CE1AD108C8F0CE018B589F4F0E9459210E
:108D3000F6CFFB0125903590459054906CCFF6010D
:108D4000259035904590549075CFE1E4FAE0259058
:108D50003590459054907FCF88E293E10E9479212D
:108D60008AE0D82EDA94CE01DD2029F08B589F4F6F
:108D70000E945921F7CF80589F4F0E948121CE0138
:108D800081589F4F0E948121C058DF4F8881C05871
:108D9000D040873009F05DC1C158DF4F8881CF577F
:108DA000D040873009F055C1CE57DF4F2881C258D7
:108DB000D040211103C080E00E9443778FE793E009
:108DC0000E94712187E793E00E94712140918703FF
:108DD00081E0482764EC70E083EB92E00E94AAAF48
:108DE000C8010E946921CE0183599F4F0E946121D1
:108DF00040918703FF24F3944F2560E170E0C801A0
:108E00000E94AAAFC8010E946921409187034F25A3
:108E10006CE070E082E497E00E94AAAF4091870383
:108E20004F2564E170E0C8010E94AAAFF09087036B
:108E3000F11030C089819A81AB81BC818093B712D7
:108E40009093B812A093B912B093BA122CEA35ECF1
:108E500047E25EE36D817E818F8198850E9478E490
:108E60006093BB127093BC128093BD129093BE129C
:108E700020E030E543EC50E469857A858B859C855C
:108E80000E9478E46093BF127093C0128093C11265
:108E90009093C21241E04F2562E070E0C8010E9449
:108EA000AAAFC8010E945121D0908703D11030C0D1
:108EB00089819A81AB81BC81809336079093370773
:108EC000A0933807B09339072CEA35EC47E25EE30C
:108ED0006D817E818F8198850E9478E460933A0746
:108EE00070933B0780933C0790933D0720E030E56B
:108EF00043EC50E469857A858B859C850E9478E4F3
:108F000060933E0770933F0780934007909341071B
:108F1000C8010E945121C8010E946121C8010E941C
:108F20006121C8010E94612185E0F80111928A95B2
:108F3000E9F7FF24F3944D2D4F2565E070E0C8015B
:108F40000E94AAAFC8010E946921409187034F2562
:108F500060E270E0C8010E94AAAFCE0183599F4F22
:108F60000E946921409187034F2569E070E0C801A4
:108F70000E94AAAF409187034F2562E170E0C801CB
:108F80000E94AAAF409187034F2564E270E0C801B8
:108F90000E94AAAF409187034F2560E170E0C801AD
:108FA0000E94AAAF409187034F2569E070E0C80195
:108FB0000E94AAAFC8010E945921409187034F2502
:108FC0006CE070E0C8010E94AAAF409187034F2572
:108FD0006CE670E0C8010E94AAAF19821A821B8257
:108FE0001C821D821E821F82188619861A861B8685
:108FF0001C86C8010E945121409187034F2568E0DB
:1090000070E0C8010E94AAAFC8010E947921CE0178
:1090100081589F4F0E946121CE0183599F4F0E942A
:10902000592180919F129091A0128C37934089F51D
:10903000109215042091C3123091C412EF968EAD98
:109040009FADEF972817390741F1F092150480E0A2
:1090500023C0CE0183599F4F0E947121C8010E94F5
:109060007121C058DF4FC880C058D040C158DF4F71
:109070008881CF57D040C89E6001112481E0C81A72
:10908000D10808F4ADCECE018B589F4F0E945921D4
:10909000F5CFF092150481E0EBDC8091870381111C
:1090A00026CD80911504811122CD0E94083F1FCD4D
:1090B00081E080938703E5DC10928703882309F021
:1090C000E0CC0E94C23F80E00895F2DF1ECBCF9338
:1090D000DF93C091D803CC23B1F0C150C093D80323
:1090E00089E0C89FE0011124CE55DC4F6A817B8165
:1090F0002F814E81888199811CDB88858093950220
:10910000DF91CF91089551DCFBCFA4E0B0E0EBE814
:10911000F8E40C94FCEA0E947FC6F09064076F2C80
:1091200085E0782E7F0C86E0E82EEF1885E0D82EBB
:10913000DF18AA24AA94B12C84E0C82ECF1882E0AC
:10914000982E9F1881E0882E8F185F2C5194F11073
:109150005AC080916707882309F444C080916A014E
:10916000882359F081E090916707911180E024E015
:1091700047E456E0652D0E94CBC58091A9078093F6
:10918000270724E0F212F7C0109273078091670757
:10919000843009F4DDC080916A018823E1F011E098
:1091A00080916707843009F010E08091270724E65A
:1091B000829FC001112481589F4FB5010E94A9EAE6
:1091C000862F0E944E1C00E09C014CE256E06C2D64
:1091D000812F0E94EC72F394F710B9CF87E080934F
:1091E00065070DC080914E0710924E07882309F441
:1091F000B5CF6DDF80916607882309F4AFCF249641
:10920000EFE00C9418EB21E0F21243C08091670765
:10921000813041F180916A018823F9F011E0809159
:109220006707813009F010E0609110017091110121
:10923000072E000C880B990B0E9419E469837A832E
:109240008B839C83CE010196BCD900E09C0141E454
:1092500056E0682D812F0E94EC728091A9078093BF
:109260002707B9CF80914E0710924E07882391F2BD
:1092700010E000E027EE33E04AE050E060E171E00A
:1092800081E496E00E9444C780916607882311F22A
:10929000B6CF82E0F812D7C080916707823021F103
:1092A00080916A018823C9F211E0809167078230BA
:1092B00009F010E06091B4127091B512072E000C05
:1092C000880B990B0E9419E469837A838B839C83B2
:1092D000CE01019676D900E09C014AE356E0692D63
:1092E000812F0E94EC7249CF80914E0710924E0759
:1092F0008823B1F20E9473C60FE411E225EF30E03B
:1093000050E040E064EB72E18AE396E00E9444C7DB
:1093100080916607882321F272CF80914E071092C8
:109320004E07882309F497C00E9473C60BEA17E61C
:1093300023E730E050E040E063E377E086E396E047
:109340000E9444C780916607882309F484C057CFE0
:1093500080914E0710924E07882309F41CCF0E947B
:1093600073C68CE296E00E94B9C980916607882393
:1093700009F411CF44CF85E0F8123DC08091670712
:10938000853011F180916A01882309F424CF11E01E
:1093900080916707853009F010E060912C01709191
:1093A0002D01072E000C880B990B0E9419E469838C
:1093B0007A838B839C83CE01019603D900E09C01C4
:1093C00047E256E06D2D04CF80914E0710924E0774
:1093D0008823C1F20FE61CE127EE33E04AE050E0BB
:1093E0006CE271E087E296E00E9444C780916607D4
:1093F000882341F204CF26E0F212EDCE8091670778
:10940000863091F080916A01882309F4E4CE81E0EE
:1094100090916707963009F080E023E048E156E03C
:109420006E2D0E94CBC5D7CE80914E0710924E076D
:10943000882341F38AE194E50E94D5C680916607AE
:10944000882301F3DCCE83E0F81297CE8091670782
:10945000833009F462CF80916A01882309F4FDCE3C
:1094600011E080916707833009F010E060913307C5
:1094700070913407072E000C880B990B0E9419E499
:1094800069837A838B839C83CE0101969AD863E0AB
:10949000661900E09C0146E356E022CFA4E0B0E06C
:1094A000E4E5FAE40C94FAEAEE24E3948091B41231
:1094B0009091B512892B09F4E12C0E947FC6F0909F
:1094C00064074F2C95E0592E5F0C88248A94912CC8
:1094D00083E0B82EBF1882E0A82EAF1881E0782E66
:1094E0007F183F2C319486E0682E6F18F11015C05C
:1094F00080916707882309F4D7C080916A01882387
:1095000009F475C181E090916707911180E024E032
:1095100043E156E0632D0E94CBC58091B412909137
:10952000B512909328078093270721E0F212E8C034
:1095300080916707813009F4C8C080916A0188234F
:1095400009F44DC011E080916707813009F010E007
:109550006091270770912807072E000C880B990B44
:109560000E9419E469837A838B839C83CE010196E0
:1095700028D800E09C014CE056E0672D812F0E9426
:10958000EC728091A9078093270793E0F91227C016
:109590001092730780916707833009F4F4C08091BB
:1095A0006A018823E1F011E080916707833009F0B8
:1095B00010E08091270724E6829FC0011124815882
:1095C0009F4FB4010E94A9EA862F0E944E1C00E022
:1095D0009C014EEF55E06B2D812F0E94EC72D12C37
:1095E000C12C14E00F2D0419C0922707F1121FC0DF
:1095F000F601EE0FFF1FE951FA4F85919491909378
:10960000750780937407809167078F1509F4CEC0A2
:1096100080916A01882359F081E090916707911346
:1096200080E023E044EF55E0602F0E94CBC5812FFE
:109630009FEFC91AD90A15E08530B1F6809133073A
:1096400090913407892B19F4EE2009F4CEC026E05E
:10965000F21221C080916707863009F4B8C080916A
:109660006A018823C1F08CED94E49F938F938BEE75
:1096700095E09F938F936F9281E09091670796306A
:1096800009F080E08F930E9434220F900F900F908A
:109690000F900F900F9087E0EE24E394F394F51071
:1096A00025CF809365070DC080914E0710924E071D
:1096B000882309F422CF0BDD80916607882309F403
:1096C0001CCF2496E1E10C9416EB80914E0710928A
:1096D0004E07882309F431CF0E9473C604E412E2D6
:1096E00025EF30E050E040E067E277E08CE096E084
:1096F0000E9444C780916607882309F41ECFE1CFFA
:1097000082E0F8123ECF80916707823019F1809194
:109710006A01882309F463CF11E0809167078230E2
:1097200009F010E06091330770913407072E000CA8
:10973000880B990B0E9419E469837A838B839C833D
:10974000CE0101960E94E14200E09C0148E056E013
:109750006A2D14CF80914E0710924E078823B9F2DC
:109760000E9473C60BEA17E623E730E050E040E0C2
:1097700063E377E088E096E00E9444C78091660743
:10978000882329F29ECF80914E0710924E0788239E
:1097900009F405CF0E9473C68EEF95E00E94B9C907
:1097A00080916607882309F4FACE8BCF80914E070B
:1097B00010924E07882309F42BCF80E09CE40E948E
:1097C000D5C680916607882309F422CF7ACF80918D
:1097D0004E0710924E07882309F441CFEDD88091AF
:1097E0006607882309F43BCF6CCF86E057CF809182
:1097F000B4129091B5129093280780932707C1CE99
:10980000B0E0A0E0E6E0FCE40C94FBEA009127075E
:109810000E947FC6C091640710E0000F111F09511C
:109820001A4F95E0592E5C0E2FEBE22E25E0F22E1A
:10983000D3E0DC1B34E5C32E32E2D32E4DECA42E54
:1098400045E0B42E82E0782E7C1A54EF852E55E048
:10985000952E81E0682E6C1A4C2E4194C1112AC0BD
:10986000809167078823B1F080916A01882359F0BD
:1098700081E090916707911180E024E04BED55E085
:10988000642D0E94CBC5CF5FC511E8CF84E08093E3
:1098900065070BC080914E0710924E07882321F375
:1098A00016DC809166078823F9F2CDB7DEB7E0E1D8
:1098B0000C9417EBC13059F5F80185919491909370
:1098C00075078093740780916707813081F08091DC
:1098D0006A018823C1F21F929F928F926F9281E05A
:1098E00090916707913009F474C080E072C0809154
:1098F0004E0710924E07882351F380912707682F57
:109900000E944BCB80916607882309F3CECFC230EB
:1099100009F042C0F8018591949190937507809366
:109920007407809167078230D1F080916A018823A3
:1099300009F4A9CFDF92CF92BF92AF927F9281E0DC
:1099400090916707923009F080E08F930E94342253
:109950000F900F900F900F900F900F9094CF8091D9
:109960004E0710924E07882301F30E9454228091E3
:1099700066078823D1F299CF80914E0710924E0747
:109980008823C1F0609127078FEF0E944BCB809115
:109990006607882379F089CFC33009F074CFF801C6
:1099A00085919491909375078093740780916707D0
:1099B000833011F380916A01882309F464CF1F92E8
:1099C000FF92EF92DF9381E090916707933009F067
:1099D0008CCF8F930E9434220F900F900F900F9096
:1099E0000F9051CFB0E0A0E0E8EFFCE40C9400EB66
:1099F0000E947FC6C091640785E0E82EEC0E9BE9CB
:109A0000C92E95E0D92ED4E0DC1B13E01C1B26EBFD
:109A1000A22E25E0B22E02E00C1B81E0F82EFC1AEB
:109A20009C2E9194C1112AC0809167078823B1F0C0
:109A300080916A01882359F081E090916707911124
:109A400080E024E04AEB55E0692D0E94CBC5CF5F52
:109A5000EC12E8CF85E0809365070BC080914E073C
:109A600010924E07882321F332DB8091660788230A
:109A7000F9F2CDB7DEB7EBE00C941CEBC13011F579
:109A800080916707813079F080916A018823F9F22B
:109A900081E090916707913009F080E023E048E190
:109AA0005CE26F2DD2CF80914E0710924E07882333
:109AB00059F38FEC9DE40E94D5C6809166078823F8
:109AC00019F3D7CFC23009F053C090916707923095
:109AD00071F080916A01882309F4B9CF81E0923056
:109AE00009F080E020E24CEA55E0602FAECF809193
:109AF0004E0710924E07882361F3B092E506A092BC
:109B0000E40680916607882321F3B3CF809167072D
:109B1000833081F080916A01882309F498CF81E035
:109B200090916707933009F080E023E04FE955E01A
:109B3000612F8BCF80914E0710924E07882351F3EF
:109B400089E29BE50E94D5C680916607882311F3C0
:109B500090CF80914E0710924E07882391F0D092BB
:109B6000E506C092E40680916607882351F081CF14
:109B7000C33061F2C43009F06ACF90916707943026
:109B800041F380916A01882309F461CF81E0943028
:109B900009F080E020E24AE855E06D2F56CFB0E0B2
:109BA000A0E0E5EDFDE40C9404EB0E947FC6C091BB
:109BB000640785E0E82EEC0ED4E0DC1B13E01C1BF0
:109BC00002E00C1B81E0F82EFC1ADC2ED194C111AE
:109BD0002AC0809167078823B1F080916A018823A9
:109BE00059F081E090916707911180E024E043E80B
:109BF00055E06D2D0E94CBC5CF5FEC12E8CF85E01C
:109C0000809365070BC080914E0710924E07882302
:109C100021F35DDA809166078823F9F2CDB7DEB7CC
:109C2000E7E00C9420EBC13011F58091670781309B
:109C300079F080916A018823F9F281E090916707B9
:109C4000913009F080E023E04EE35CE26F2DD2CF4B
:109C500080914E0710924E07882359F383E692E2D3
:109C60000E94D5C680916607882319F3D7CFC230EA
:109C700009F055C080916707823081F080916A01B8
:109C8000882309F4B9CF81E090916707923009F0F9
:109C900080E023E047E35CE2602FACCF80914E0789
:109CA00010924E07882351F38EE592E20E94D5C6AA
:109CB00080916607882311F3B1CF809167078330C5
:109CC00081F080916A01882309F496CF81E0909118
:109CD0006707933009F080E023E040E35CE2612F06
:109CE00089CF80914E0710924E07882351F389E562
:109CF00092E20E94D5C680916607882311F38ECF29
:109D000080914E0710924E07882391F08EE194E4E3
:109D10000E94D5C680916607882351F07FCFC3305B
:109D200061F2C43009F068CF80916707843041F355
:109D300080916A01882309F45FCF81E090916707E1
:109D4000943009F080E023E042E25CE26D2F52CFD4
:109D5000ACE0B0E0EEEAFEE40C94FAEA9C878B8774
:109D6000362E80914E0710924E07882339F01092BC
:109D70009502ADD92C96E1E10C9416EB6091690740
:109D800070916A0780916B0790916C07611571055E
:109D90008105910509F45CC020911201222309F488
:109DA000AEC0209113012111AAC021E0321609F49E
:109DB00084C0E2E03E1609F491C0C0901401D09036
:109DC0001501E0901601F09017014090200150908D
:109DD000210160902201709023010E9419E42091DA
:109DE00008013091090140910A0150910B010E9434
:109DF00078E46F83788789879A87F4E03F9E8001B3
:109E00001124C8018B589E4F9E838D83FC012081B5
:109E10003181428153816F81788589859A850E943D
:109E200031EB4B015C01A3019201C701B6010E9415
:109E300013E4811173C0F801EB58FE4F80829182C8
:109E4000A282B382832D0E94966B81E080936A0187
:109E50001092690710926A0710926B0710926C07B4
:109E600080916A01882309F485CF24E0329EF001B5
:109E70001124EB58FE4FC080D180E280F380C9826C
:109E8000DA82EB82FC822DEC3CEC4CEC5DE36091E1
:109E900008017091090180910A0190910B010E94C3
:109EA00094EC87FD65C0CE0101960E949C1ABC010E
:109EB0008B859C850E9485725DCFC0901801D090E3
:109EC0001901E0901A01F0901B014090240150907C
:109ED000250160902601709027017FCFC0901C0162
:109EE000D0901D01E0901E01F0901F0140902801CC
:109EF0005090290160902A0170902B016ECF412C67
:109F000020E5522E23EC622E27E4722EC12C30E580
:109F1000D32E33ECE32E37ECF32E5FCF20E030E08E
:109F2000A9016F81788589859A850E9413E487FF4E
:109F30000FC0A7019601C501B4010E9413E487FF79
:109F40007ACFED81FE81C082D182E282F3827ACF24
:109F5000A3019201C501B4010E9494EC18160CF003
:109F60006ACFED81FE8140825182628273826ACF24
:109F700020E030E44CE156E4C701B6010E9478E4E9
:109F80004B015C0120E030E0A901C701B6010E944D
:109F900013E420E030E040EA50E487FF04C020E012
:109FA00030E040EA50ECC501B4010E9431EB2DECE9
:109FB0003CEC4CEC5DE30E9478E40E9410EC6B01F9
:109FC0007C01F7FC64C020EA36E841E050E00E94E2
:109FD000BCEACA01B9012AE030E040E050E00E944A
:109FE000BCEA605D60939602C701B60120E137E2EA
:109FF00040E050E00E94BCEA8AE0882E912CA12C1F
:10A00000B12CCA01B901A50194010E94BCEA605DAE
:10A0100060939702C701B60128EE33E040E050E0BC
:10A020000E94BCEACA01B901A50194010E94BCEAE0
:10A03000605D609398028EE280939902C701B60139
:10A0400024E630E040E050E00E94BCEACA01B901D9
:10A05000A50194010E94BCEA605D60939A02C70169
:10A06000B601A50194010E94BCEA6B017C01CA0102
:10A07000B901A50194010E94BCEA605D60939B0256
:10A0800080E3C80EC0929C0286E992E010CFF09463
:10A09000E094D094C094C11CD11CE11CF11C6DE271
:10A0A000A1CF62E080E39CE253CE61E087E39CE2D3
:10A0B0004FCE60E08EE39CE24BCEA4E0B0E0E3E65E
:10A0C000F0E50C9409EB80914E0710924E0788231F
:10A0D00041F0109295020E9467482496E2E00C94A9
:10A0E00025EB6091690770916A0780916B079091E9
:10A0F0006C07611571058105910561F10E9419E4F4
:10A10000209108013091090140910A0150910B0101
:10A110000E9478E420918101309182014091830175
:10A12000509184010E9431EB609381017093820110
:10A13000809383019093840183E00E94966B81E079
:10A1400080936A011092690710926A0710926B0758
:10A1500010926C0780916A01882309F4BECF209188
:10A160004F0730915007409151075091520760912D
:10A1700081017091820180918301909184010E94FC
:10A1800030EB69837A838B839C83CE0101960E9496
:10A190009C1ABC0182E29CE20E9485729ECFB0E0D4
:10A1A000A0E0E5EDF0E50C9404EB0E947922082F85
:10A1B0000E947FC6C0916407FC2E85E0E82EEC0E5D
:10A1C00011E01C1BDC2ED194C11114C080916707D3
:10A1D0008823F9F080916A01882309F474C081E032
:10A1E00090916707911180E024E04CE753E06D2DDA
:10A1F0000E94CBC501113AC0D2E0C130C1F58091B7
:10A2000067078130B9F080916A01811122C0D2E0E4
:10A2100044C080914E0710924E078823D9F20E94C5
:10A220006748809166078823A9F2CDB7DEB7E7E0DB
:10A230000C9420EB80914E0710924E07882319F35F
:10A2400080E891E50E94D5C6809166078823D9F2FF
:10A25000ECCF81E090916707913009F080E023E036
:10A2600043E753E0612F0E94CBC5D1CFD1E0DC138F
:10A2700014C0809167078D17B9F080916A01882317
:10A2800061F06C2F6F1981E0909167079C1380E05B
:10A2900023E047E653E00E94CBC5CF5FCE1194CFB9
:10A2A000DF5FD0936507C1CF80914E0710924E07B4
:10A2B000882319F383EA96E50E94D5C68091660744
:10A2C0008823D9F2B2CFD1E0002309F4A0CFE5CFA3
:10A2D00080E090E0A0E8B0E480937D0190937E015F
:10A2E000A0937F01B09380018AE192E00E94BA219D
:10A2F0008091E6030E944377109295020C94674880
:10A30000B0E0A0E0E6E8F1E50C9402EB0E947FC625
:10A31000C091640785E0C82ECC0ED4E0DC1B13E0AE
:10A320001C1B82E0F82EFC1A81E0E82EEC1ABC2EF1
:10A33000B194C1112BC0809167078823B1F080913F
:10A340006A01882359F081E090916707911180E0BC
:10A3500024E045E553E06B2D0E94CBC5CF5FCC12C6
:10A36000E8CF85E0809365070CC080914E0710927E
:10A370004E07882321F30E9467488091660788234F
:10A38000F1F2CDB7DEB7E9E00C941EEBC13089F5F0
:10A39000809167078130C1F080916A018823F1F2D2
:10A3A000DD24D39480916707813009F0D12C8FE7A9
:10A3B0009DE00E94821D00E09C014AE453E06E2D66
:10A3C0008D2D0E94EC72CACF80914E0710924E07DD
:10A3D000882311F30E9473C640EB5BE26FE77DE0D8
:10A3E0008AE493E00E94E4C6809166078823A1F284
:10A3F000C8CFC23009F073C0809167078230B1F0D6
:10A4000080916A01882309F4A9CFDD24D394809137
:10A410006707823009F0D12C83E89DE00E94821DFD
:10A4200000E09C014FE353E06F2DCACF80914E07AF
:10A4300010924E07882321F30E9473C64FEA5BE215
:10A4400063E87DE08FE393E00E94E4C680916607B5
:10A450008823B1F296CF809167078330B1F0809165
:10A460006A01882309F47ACFDD24D39480916707A9
:10A47000833009F0D12C87E89DE00E94821D00E026
:10A480009C0144E353E0612F9BCF80914E071092D3
:10A490004E07882321F30E9473C64EEA5BE267E809
:10A4A0007DE084E393E00E94E4C680916607882300
:10A4B000B1F267CF80914E0710924E078823C9F002
:10A4C0000E9473C64DEA5BE26BE87DE089E293E0AF
:10A4D0000E94E4C680916607882359F052CFC330AA
:10A4E00009F4B9CFC43009F039CF809167078430BF
:10A4F00009F380916A01882309F430CFDD24D394D5
:10A5000080916707843009F0D12C8BE89DE00E9490
:10A51000821D00E09C0149E253E06D2F51CFA3E082
:10A52000B0E0E5E9F2E50C94F9EA4C013B015A018F
:10A530001901280181E080939502409169075091AB
:10A540006A0760916B0770916C07411551056105B1
:10A55000710571F0141615060CF080E08093E40389
:10A560001092690710926A0710926B0710926C079D
:10A570001091E40380914E078B8310924E07811156
:10A5800005C080916A01882309F46FC0C2010E944E
:10A590003E6C082F80E0C114D10419F0C6010E945E
:10A5A0003E6C1A821982E114F104B1F4402F50E09C
:10A5B000282F30E0CA01820F931F46976CF485E183
:10A5C00090E0841B950B821B930B97FD019695954C
:10A5D00087958A8381E0898301E02EE336E6A20134
:10A5E000BE016F5F7F4FCE0102960E94966DE1140F
:10A5F000F10491F08A81882321F01A8289818F5F8A
:10A60000898300E021E436E6A701BE016F5F7F4F3A
:10A61000CE0102960E94966DC114D10459F000E05B
:10A620002EE336E6A601BE016F5F7F4FCE01029694
:10A630000E94966D41E04127B30181E00E94BCCDAC
:10A64000C4010E943E6C412FB40194E1981B892FF4
:10A650000E94BCCDEB81EE2341F0111101C05101EC
:10A66000A114B10431F0F50109952396E2E10C94AF
:10A6700015EB0E946748F9CFCF92DF92EF92FF92DD
:10A680000F931F9384E6C82E85E0D82EF12CE12C81
:10A6900006E615E030E020E047E154E466E775E0C7
:10A6A0008BE795E03CDF1F910F91FF90EF90DF90DB
:10A6B000CF900895B0E0A0E0E0E6F3E50C9401EB64
:10A6C000ADB6BEB6809125106AE777E0882311F019
:10A6D00065E270E1FB0101900020E9F7CF01861BE4
:10A6E000970B01962DB73EB7281B390B0FB6F89480
:10A6F0003EBF0FBE2DBF8DB79EB701967C0180E295
:10A70000EDB7FEB78183C70101960E9455ED80E247
:10A71000C82E85E0D82E02E215E030E020E041EEC0
:10A7200054E46EE275E085E395E0F9DE0FB6F89447
:10A73000BEBE0FBEADBEEAE00C941DEBCF92DF9221
:10A74000EF92FF920F931F938EE7C82E84E0D82ECE
:10A75000F12CE12C01EF14E030E020E041E053E681
:10A7600060E874E085E894E0DADE1F910F91FF90D5
:10A77000EF90DF90CF900895CF92DF92EF92FF920B
:10A780000F931F938AE8C82E83E0D82EF12CE12C7A
:10A790000CE813E028E631E542EC51E268E973E0A9
:10A7A0008DE993E0BCDE1F910F91FF90EF90DF9059
:10A7B000CF900895B0E0A0E0E0EEF3E50C9401EB5B
:10A7C000ADB6BEB683E392E00E943E6C90E0019687
:10A7D0002DB73EB7281B390B0FB6F8943EBF0FBEFE
:10A7E0002DBF8DB79EB701967C0163E372E00E9496
:10A7F0005BE38091270700E012E0813031F00BEE3F
:10A8000011E0823011F003E112E084E2C82E82E010
:10A81000D82E25ED34E440ED5EE566E272E08DE28F
:10A8200092E07DDE0FB6F894BEBE0FBEADBEEAE08C
:10A830000C941DEB8F929F92AF92BF92CF92DF92BA
:10A84000EF92FF920F9380914E0710924E0788234C
:10A8500071F0109295020E9467480F91FF90EF905F
:10A86000DF90CF90BF90AF909F908F90089581E040
:10A87000809395028091690790916A07A0916B0778
:10A88000B0916C070097A105B10509F44AC05C01BD
:10A89000AA0CBB1CAA0CBB1C1092690710926A0779
:10A8A00010926B0710926C07B5010B2C000C880BF3
:10A8B000990B0E9419E42091B2073091B30740919F
:10A8C000B4075091B5070E9478E42091301330917D
:10A8D000311340913213509133130E9431EB6B01CD
:10A8E0007C0120E030E040EA51EC0E9494EC87FDCE
:10A8F00018C020E030E040EA51E4C701B6010E94F0
:10A9000013E4181674F0C5010E94E9C1C092301317
:10A91000D0923113E0923213F092331382E080939D
:10A920006A0180916A01882309F497CFC09030139F
:10A93000D0903113E0903213F090331320E030E4E4
:10A940004CE156E4C701B6010E9478E44B015C017A
:10A9500020E030E0A901C701B6010E9413E420E025
:10A9600030E040EA50E487FF04C020E030E040EAF5
:10A9700050ECC501B4010E9431EB2DEC3CEC4CECE9
:10A980005DE30E9478E40E9410EC6B017C018BE295
:10A99000F7FE09C0F094E094D094C094C11CD11C7F
:10A9A000E11CF11C8DE280939602C701B60120E103
:10A9B00037E240E050E00E94BCEA6AE0862E912C2B
:10A9C000A12CB12CCA01B901A50194010E94BCEAD5
:10A9D000605D60939702C701B60128EE33E040E066
:10A9E00050E00E94BCEACA01B901A50194010E948D
:10A9F000BCEA605D609398028EE280939902C70181
:10AA0000B60124E630E040E050E00E94BCEACA0112
:10AA1000B901A50194010E94BCEA605D60939A02AD
:10AA2000C701B601A50194010E94BCEA6B01CA01ED
:10AA3000B901A50194010E94BCEA605D60939B028C
:10AA400060E36C0D60939C0266E972E084EF92E033
:10AA50000E948572C0903013D0903113E090321371
:10AA6000F09033138090E0039090E103A090E20314
:10AA7000B090E303A5019401C701B6010E9413E45D
:10AA80008823E9F020E030E0A901C701B6010E9467
:10AA900013E4882309F479C0A5019401C701B60124
:10AAA0000E9413E487FD73C081E08093DF03C092AE
:10AAB000E003D092E103E092E203F092E303D0904E
:10AAC000DF0380919913813188F480919B13833047
:10AAD00068F044E04D195CEDE52E52E0F52E0CE0F7
:10AAE00022E062E485E693E10E94F8CE809199131A
:10AAF000853180F480919B13843160F049EDE42E20
:10AB000042E0F42E01E023E044E16CE385E693E1CA
:10AB10000E94F8CE809199138F3308F09ECE8091D9
:10AB20009B138F3208F499CE40E34D198FEBE82E3A
:10AB300082E0F82E0DE022E06AE585E693E10E94CE
:10AB4000F8CE41E34D1995EAE92E92E0F92E22E084
:10AB500065E085E693E10E94F8CE25E7E22E22E04B
:10AB6000F22E00E123E04FE262E185E693E10E94EC
:10AB7000F8CE35E4E32E32E0F32E23E04FE267E631
:10AB800085E693E10E94F8CE68CE80E08ECF8FEF0D
:10AB90008CCF0F931F93CF93DF93FC01EB01809138
:10ABA000690790916A07A0916B07B0916C07B7FF96
:10ABB00008C01092690710926A0710926B071092F2
:10ABC0006C078091580790915907A0915A07B0914E
:10ABD0005B074091690750916A0760916B0770911C
:10ABE0006C0784179507A607B70744F48093690795
:10ABF00090936A07A0936B07B0936C0780916A01EA
:10AC00008823E1F06091690770916A0780916B0772
:10AC100090916C0700915C0710915D0720915E0791
:10AC200030915F07600F711F821F931F0995BC0150
:10AC300080916207909163070E94857280914E0710
:10AC4000811108C0809155078823A9F180916A017C
:10AC5000882389F180916007909161070097B1F096
:10AC60004091690750916A0760916B0770916C077A
:10AC700000915C0710915D0720915E0730915F079E
:10AC8000400F511F621F731FFE010995E091560787
:10AC9000F0915707309741F080915507811103C01B
:10ACA00080914E078111099580914E0710924E07B1
:10ACB00081110E946748DF91CF911F910F910895F4
:10ACC00068E87CE181EA9CE164CF65E07DE18EEC9F
:10ACD00092E45FCF63E17DE186E39EE15ACF67E2D4
:10ACE0007DE18BE39DE155CF64E77DE18AEE92E45F
:10ACF00050CFE091D803E63028F581E08E0F8093A5
:10AD0000D8034091690750916A0760916B07709171
:10AD10006C0720916407909165078091950239E056
:10AD2000E39FF0011124EE55FC4FA0915F13B09109
:10AD30006013B183A0834283538364837583268326
:10AD4000978380870895A7E0B0E0E9EAF6E50C94E0
:10AD5000F9EA0E947FC6F09064072F2C85E08F0DE2
:10AD60008D833324339483E0E82E98EE892E93E08C
:10AD7000992EA12CB12C84E08F198E839E2D9F19C2
:10AD80009F8382E0D82EDF18C32CCF18F1102CC07F
:10AD9000809167078823C1F080916A01882361F060
:10ADA000622D619581E090916707911180E024E028
:10ADB00045E553E00E94CBC5F3949D81F912E6CF9F
:10ADC00085E0809365070CC080914E0710924E0776
:10ADD000882311F30E946748809166078823E1F277
:10ADE0002796E2E10C9415EB81E0F8122DC09091CA
:10ADF00067079130B9F080916A018823E9F281E018
:10AE0000913009F080E0909197032DE133E09111AA
:10AE100002C029E133E001E040E253E06C2D0E94E2
:10AE2000EC72CACF80914E0710924E07882319F317
:10AE3000809197038F2580939703E0926A01809118
:10AE400066078823C1F2CCCF92E0F912D1C080917D
:10AE50006707823021F180916A01882309F4ACCF21
:10AE600011E080916707823009F010E060910601DF
:10AE700070910701072E000C880B990B0E9419E4B2
:10AE800069837A838B839C83CE0101960E94E14281
:10AE900000E09C0142E153E06D2D812FC0CF8091F5
:10AEA0004E0710924E078823B1F210E000E025EF24
:10AEB00030E050E040E066E071E082E193E00E9423
:10AEC00044C780916607882331F28ACF8091670753
:10AED000833019F180916A01882309F46DCF11E064
:10AEE00080916707833009F010E060910401709150
:10AEF0000501072E000C880B990B0E9419E4698349
:10AF00007A838B839C83CE0101960E94E14200E00C
:10AF10009C014BE053E06F81C0CF80914E071092AF
:10AF20004E078823B9F210E000E025EF30E050E052
:10AF300040E064E071E08BE093E00E9444C78091C0
:10AF40006607882339F24CCF80914E0710924E0746
:10AF5000882309F459C020E030E048EC52E46091C5
:10AF600000017091010180910201909103010E9402
:10AF700078E40E9415EC2B0130926607BADEE0926D
:10AF80006A0183E093E0909363078093620780E017
:10AF900091E0909361078093600710925C07109294
:10AFA0005D0710925E0710925F078092580790929B
:10AFB0005907A0925A07B0925B07712C612C4092FE
:10AFC000690750926A0760926B0770926C078FE670
:10AFD00096E59093601380935F1310925707109239
:10AFE00056071092550780916607882369F0F8CEBE
:10AFF00083E0F81609F46ACF94E0F912DDCE80916F
:10B000006707843009F4A0CF80916A01882309F48E
:10B01000D3CE11E080916707843009F010E04090B2
:10B02000000150900101609002017090030120E046
:10B0300030E0A901C301B2010E9413E42DEB37E314
:10B0400046E055EB87FD04C02DEB37E346E055E3C2
:10B05000C301B2010E9431EB69837A838B839C83A5
:10B06000CE0101960E94121B00E09C0143E053E0D8
:10B070006E8113CFB0E0A0E0E0E4F8E50C9409EBBA
:10B080008D8190919610891778F0809396109E018B
:10B09000285F3F4F4E815F8164E570E081E490E17D
:10B0A0000E94DBE310924010E2E00C9425EB0F933A
:10B0B0001F93CF93DF938C016F3F19F4109296107A
:10B0C00060E020919610862F062E000C990B281711
:10B0D000190609F004F560939610C8010E9462E316
:10B0E000800F911FEC01C01BD10BC535D1053CF081
:10B0F0000197FC012491207C2038D1F3F3CFDD2788
:10B10000AE01B80181E490E10E9483E3CF5BDF4EA2
:10B11000188210924010DF91CF911F910F910895E6
:10B12000A6E8B0E0E6E9F8E50C9403EBC358DF4F7E
:10B13000188219821A821B82CD57D04080918A02D0
:10B1400090918B02A0918C02B0918D02CF57DF4F6E
:10B1500088839983AA83BB83C158D04084E690E05A
:10B160009093A01280939F121092C4121092C31257
:10B170001092150464E070E0CE018F579F4F0E943B
:10B18000A7CA80919F129091A01202969093A0124C
:10B1900080939F121092C4121092C31281E0CA577A
:10B1A000DF4F8883C658D040CE018A579F4F0E94F8
:10B1B000902168E470E08BE69DE00E94A7CA80E1E0
:10B1C000E1E9F1E08E010F5F1F4FD80101900D9270
:10B1D0008A95E1F760E170E0C8010E94A7CA8DE896
:10B1E00097E00E9498218CE0F80111928A95E9F786
:10B1F000C8010E9494217E01FDE6EF0EF11C8FEF45
:10B20000F7018083C7010E94902119821A821B8254
:10B210001C82C8010E9498218091AF029091B002D7
:10B22000A091B102B091B20289839A83AB83BC83AF
:10B23000C8010E949821C358DF4F188219821A82D0
:10B240001B82CD57D04083E0F70180838983CE01F4
:10B2500083589F4F0E949821C7010E949021C801E6
:10B260000E9490213AE0D32EDA94DD2031F0CE0115
:10B2700083589F4F0E949821F7CF88E293E10E9464
:10B280009421C358DF4F188219821A821B82CD572E
:10B29000D0402AE0D22EDA94DD2031F0CE0183585E
:10B2A0009F4F0E949821F7CF87E08983F701808321
:10B2B000C8010E949021C7010E94902168E070E0BF
:10B2C0008FE793E00E94A7CA68E070E087E793E009
:10B2D0000E94A7CA64EC70E083EB92E00E94A7CAC8
:10B2E0001982CC24CA94F701C082C8010E94FDCA09
:10B2F000C7010E94902180E1D82EF8018D2D119276
:10B300008A95E9F760E170E0C8010E94A7CA198236
:10B31000C8010E94FDCA6CE070E082E497E00E94E0
:10B32000A7CA198A1A8A1B8A1C8A80E090E0A0E8C2
:10B33000BFE38D879E87AF87B88B8091B7129091BE
:10B34000B812A091B912B091BA1289839A83AB83D3
:10B35000BC8320E030E543EC50E46091BB12709177
:10B36000BC128091BD129091BE120E9478E46D8350
:10B370007E838F8398872CEA35EC47E25EE3609109
:10B38000BF127091C0128091C1129091C2120E949E
:10B3900078E469877A878B879C8764E170E0C801CD
:10B3A0000E94A7CA84E190E09A83898362E070E0FA
:10B3B000C8010E94A7CA8091360790913707A091D3
:10B3C0003807B091390789839A83AB83BC8320E027
:10B3D00030E543EC50E460913A0770913B0780916F
:10B3E0003C0790913D070E9478E46D837E838F83B4
:10B3F00098872CEA35EC47E25EE360913E07709156
:10B400003F0780914007909141070E9478E4698747
:10B410007A878B879C87C8010E948C218CE0E1EAA7
:10B42000F1E0D80101900D928A95E1F7C8010E94E0
:10B430008C211982C8010E9490218FE78983C8015D
:10B440000E949021C982C8010E94902185E0EDEA06
:10B45000F1E0D80101900D928A95E1F765E070E086
:10B46000C8010E94A7CA1982C8010E94FDCA80E2D1
:10B47000E2EBF1E0D80101900D928A95E1F760E2EC
:10B4800070E0C8010E94A7CAF7011082C7010E949C
:10B49000FDCA1982C8010E94FDCA80E090E0A0EEBA
:10B4A000BFE3C358DF4F88839983AA83BB83CD57FB
:10B4B000D040CE0183589F4F0E949821C358DF4F40
:10B4C000188219821A821B82CD57D040CE01835830
:10B4D0009F4F0E94982182E1F80111928A95E9F725
:10B4E00062E170E0C8010E94A7CA84E2E2EDF1E0E7
:10B4F000D80101900D928A95E1F764E270E0C801ED
:10B500000E94A7CAF8011192DA94E9F760E170E0AD
:10B51000C8010E94A7CA89E0F80111928A95E9F74B
:10B5200069E070E0C8010E94A7CAC358DF4F1882C3
:10B5300019821A821B82CD57D040CE0183589F4F6B
:10B540000E9498219CE0D92EF8018D2D11928A95A8
:10B55000E9F76CE070E0C8010E94A7CA8CE6F80128
:10B5600011928A95E9F76CE670E0C8010E94A7CABB
:10B5700089E094E00E948C21F701108211821282EE
:10B580001382148215821682178268E070E0C70168
:10B590000E94A7CAF7011192DA94E9F7CB57DF4F5F
:10B5A0001882C558D04080E090E0A0E4B0E4ED9669
:10B5B0008CAF9DAFAEAFBFAFED97C7010E94942196
:10B5C000CE018B579F4F0E949021CE0187589F4FED
:10B5D0000E94982180911504811127C000919F122B
:10B5E0001091A0128091C3129091C412F70191831F
:10B5F000808384E690E09093A01280939F1264E091
:10B6000070E082E292E00E94A7CA62E070E0C701A7
:10B610000E94A7CA91E00C37F3E01F0709F490E0FD
:10B6200080911504892B8093150480911504811154
:10B6300004C060E085E29AE03ADD9091150481E073
:10B640008927CA57DF4FE8E00C941FEB69DD0C94A3
:10B650008543A7E0B0E0EFE2FBE50C94F9EA8091C6
:10B6600077078770898380907F0390908003A090F4
:10B670008103B09082030E947FC6209164072E83CD
:10B680003981373009F075C085E194E09B838A8366
:10B690001E81312F3B5F3C8333243394812F81956E
:10B6A0008D83232C211A84E6482E512C612C712C79
:10B6B0002E81222309F462C03981373009F433C264
:10B6C0002E81213009F028C290916707913009F44A
:10B6D00045C180916A01811154C182E0F82E81E058
:10B6E0008F0D8F839981973009F063C020E030E09F
:10B6F000A901C501B4010E9413E4882309F459C0CB
:10B700003F818E81381331C09091AE029F8380912A
:10B7100067072E81821311C080914E0710924E0749
:10B72000882359F093259F8383E080936A010E94C8
:10B730009C218091660781110DC180916A01882347
:10B74000A1F06E81611B81E0909167073E819313A8
:10B7500080E09F8126EF33E0911102C022EF33E0B9
:10B7600001E049EF53E00E94EC72F394F394FF82FE
:10B7700020C020E134E03B832A838ACF8091670791
:10B78000882309F4D9C080916A01882309F494CFF1
:10B7900081E090916707911180E024E043E254E05A
:10B7A0006D810E94CBC58981873009F41DC193E06A
:10B7B0009F838091AF029091B002A091B102B091AD
:10B7C000B2028093270790932807A0932907B0938C
:10B7D0002A072F813E8123131EC08091670782179D
:10B7E00009F407C180916A018823A9F0EE80E11A6B
:10B7F000FF24F394809167073E818313F12C87E245
:10B8000097E00E94914200E09C0146EE53E06E2DCD
:10B810008F2D0E94EC728F818F5F9E81891316C0DD
:10B8200080916707891709F438C180916A018823DC
:10B8300069F06E81611B81E0909167072E81921300
:10B8400080E023E047ED53E00E94CBC58F818E5FFF
:10B850003E81831316C080916707831709F42EC1B8
:10B8600080916A01882369F06E81611B81E090916B
:10B8700067072E81921380E023E04AEC53E00E9498
:10B88000CBC58F818D5F3E81831323C08091670775
:10B89000831709F424C180916A018823D1F085E6D9
:10B8A00098E49F938F938CEB93E09F938F938E817B
:10B8B000811B8F9381E0909167073E81931380E015
:10B8C0008F930E9434220F900F900F900F900F9043
:10B8D0000F908F818C5F9E81891323C080916707B1
:10B8E000891709F40BC180916A018823D1F086E29F
:10B8F0009BE59F938F938DEA93E09F938F938E8127
:10B90000811B8F9381E0909167072E81921380E0D5
:10B910008F930E9434220F900F900F900F900F90F2
:10B920000F903E813F5F3E838C818313C1CE9F8108
:10B930009B5F909365070EC080914E0710924E0753
:10B94000882309F420CF0E946748809166078823E6
:10B9500009F419CF2796E2E10C9415EB80914E077C
:10B9600010924E07882309F4B4CE26EB35E03093CD
:10B97000E5062093E40680916607882309F4A9CEA2
:10B98000E9CF81E0913009F080E020E249E154E024
:10B99000622D0E94CBC5A1CE909167073E8193177F
:10B9A00031F080916A01811113C08E8197CE809110
:10B9B0004E0710924E078823A1F32A813B813093D2
:10B9C000E5062093E40680916607882351F3C2CFF1
:10B9D0006E81611B81E03E81931380E020E246E0AE
:10B9E00054E00E94CBC5E1CF22E02F83FF24F394E3
:10B9F0007DCE80914E0710924E07882309F4F2CE37
:10BA00000E9473C6609127077091280780912907CB
:10BA100090912A070E9415EC6B013092660769D954
:10BA200083E080936A0186EE93E0909363078093AE
:10BA3000620727E237E03093610720936007109296
:10BA40005C0710925D0710925E0710925F074092AC
:10BA500058075092590760925A0770925B07F12C71
:10BA6000E12CC0926907D0926A07E0926B07F092CE
:10BA70006C0785E696E59093601380935F1322EA46
:10BA800031E2309357072093560710925507809163
:10BA90006607882309F4A6CE5DCF80914E071092E9
:10BAA0004E07882309F4C1CE8AE194E50E94D5C6E9
:10BAB00080916607882309F4B8CE4CCF80914E0759
:10BAC00010924E07882309F4CBCE87E994E40E94B4
:10BAD000D5C680916607882309F4C2CE3BCF8091FA
:10BAE0004E0710924E07882309F4D5CE0E94654870
:10BAF00080916607882309F4CECE2CCF80914E0723
:10BB000010924E07882309F4EECEA0DD80916607DF
:10BB1000882309F4E8CE1ECF2E81223009F43CCFD1
:10BB200033E03F8346CE8E81813009F435CF92E0F9
:10BB30009F835CCFB0E0A0E0E0EAFDE50C94FCEA76
:10BB40000E947922D82F0E947FC6C09164075C2E84
:10BB500085E0682E6C0E95E6E92E98E4F92E2BE32D
:10BB6000C22E24E0D22E14E01C1B36E9A32E33E4AF
:10BB7000B32E05E00C1B83E0982E9C1A82E0882EE1
:10BB80008C1A81E0782E7C1AC11141C08091670720
:10BB9000882361F180916A01882361F0652D6195A8
:10BBA00081E090916707911180E024E049E754E03B
:10BBB0000E94CBC5D111EDC0C43009F0A0C0809166
:10BBC0006707843009F47FC080916A01882309F4F3
:10BBD000B6C0FF92EF92DF92CF921F9381E09091D7
:10BBE0006707943009F4A2C080E0A0C080914E079E
:10BBF00010924E07882371F20E9467488091660771
:10BC0000882341F2CDB7DEB7EFE00C9418EBC130DA
:10BC100031F580916707813099F080916A0188231E
:10BC200061F081E090916707913009F080E023E0B6
:10BC300047E654E0672D0E94CBC5D111AAC07FC052
:10BC400080914E0710924E07882339F38FEC90E5D0
:10BC50000E94D5C6809166078823F9F2D3CFC230FF
:10BC600009F06FC080916707823081F080916A018E
:10BC7000882309F48BC081E090916707923009F026
:10BC800080E023E048E554E0682DD5CF80914E0751
:10BC900010924E07882351F38AE194E50E94D5C69D
:10BCA00080916607882311F3ADCF80914E071092E3
:10BCB0004E07882309F44DC0C9DC809166078823AC
:10BCC00009F447C09FCF80914E0710924E078823FA
:10BCD00009F47ACF0E94654880916607882309F4A9
:10BCE00073CF90CF80914E0710924E07882369F052
:10BCF0000E94964380916607882339F083CFC53030
:10BD0000F1F480916707853069F380916A01882397
:10BD1000B1F0BF92AF928AE294E09F938F930F931A
:10BD200081E090916707953009F05ECF8F930E9474
:10BD300034220F900F900F900F900F900F9086E08D
:10BD400029C0C33009F036CF80916707833009F4EA
:10BD5000ACCF80916A018823C9F086E29BE59F936E
:10BD60008F9389E494E09F938F939F9281E09091C9
:10BD70006707933009F080E08F930E9434220F9080
:10BD80000F900F900F900F900F9057CFDD2309F475
:10BD9000B6CF84E0CF5F6C12F7CE8093650732CFC9
:10BDA0000E94C23FBDD90E9485430C94D544A4E0B3
:10BDB000B0E0EDEDFEE50C94FAEA9091E3069817F9
:10BDC00009F474C0382E80E090E0A0E2B1E48983E9
:10BDD0009A83AB83BC8340903013509031136090B2
:10BDE00032137090331320E030E0A901C301B20197
:10BDF0000E9413E487FF0CC0A301920160E070E091
:10BE000080E291E40E9430EB69837A838B839C8388
:10BE1000CE0101960E949BC1409075015090760121
:10BE200060907701709078018090790190907A010C
:10BE3000A0907B01B0907C0163E972E084E690E021
:10BE40000E9459436AEB72E084E690E00E945943F5
:10BE500001EF19E0332011F00EEF19E00E94D544F4
:10BE600063E6C80124D9C8010E940C8860E070E034
:10BE7000CB010E9494CB0E9478C119821A821B8246
:10BE80001C82E0907D01F0907E0100917F01109175
:10BE90008001CE0101966C01A5019401C301B2019C
:10BEA0000E94923D3092E3060E94B83F80E02496C3
:10BEB000E1E10C9416EB4F925F926F927F928F921A
:10BEC0009F92AF92BF92DF92EF92FF920F931F93D8
:10BED000CF93DF93D82EC82FD0E0FE01EA5AF34D5E
:10BEE000F49082E0D81609F4E4C06F2DFF0C770BB4
:10BEF000880B990B0E9419E42B013C01CE01880F9D
:10BF0000991F880F991F875D984F0E94EE744B010F
:10BF10005C01A3019201C501B4010E9478E44B01C8
:10BF20005C017E01EE0CFF1CEE0CFF1CC701835E62
:10BF3000984F0E94EE749B01AC01C301B2010E94B4
:10BF400078E420E030E040EC5FE30E9478E4AB016D
:10BF5000BC0100E010E098018D2D0E94BEC420E0DD
:10BF600030E0A901C501B4010E9413E4882309F45B
:10BF700040C082E000E010E020E830E4D81619F07C
:10BF800000E010E09801B501A40170588D2D0E94C9
:10BF9000BEC4A5019401C501B4010E9431EB4B015F
:10BFA0005C0182E000E010E020E030E4D816E1F02F
:10BFB000FE01E25FF84F6491611107C00E94EF85B6
:10BFC0008CEE96E00E94AD7F6AE070E090E080E049
:10BFD0000E9417E49B01AC0161E070E088E492E408
:10BFE0000E94A8EB8B019C01B501A4018D2D0E943C
:10BFF000BEC481E090E00D2C01C0880F0A94EAF7DE
:10C0000090917707982B9093770790910804892B4C
:10C0100080930804C7018F5E984F0E94EE74F70169
:10C02000EB58FE4F608371838283938382E0D81242
:10C030001AC0209130133091311340913213509136
:10C04000331360917D0170917E0180917F01909109
:10C0500080010E9430EB60937D0170937E0180939C
:10C060007F01909380010E94C43EF701E256FD4F8C
:10C07000D701AB58BE4F8D919D910D90BC91A02DD5
:10C0800080839183A283B38382E0D81202C080E0D0
:10C090008EDEDF91CF911F910F91FF90EF90DF9097
:10C0A000BF90AF909F908F907F906F905F904F90D8
:10C0B000089581E07CDE8111ECCF81E397E00E945E
:10C0C000EE7420E030E0A9010E9413E4882309F413
:10C0D0000CCF6F2DFF0C770B880B990B0E9419E486
:10C0E0002B013C0181E397E00E94EE744B015C015F
:10C0F00020E030E040EA50E40E9494EC87FF09CF52
:10C10000812C912C90EAA92E90E4B92E02CFCF93E6
:10C1100080919A03811109C08CED91E09093DE0328
:10C120008093DD0381E080939A030E94795620E09A
:10C1300040E070E060E084E892E20E949943C1E050
:10C14000C09395020E94B12B0E946748C09395024C
:10C1500060E08CE89CE20E94575888ED91E0909353
:10C16000E5068093E406CF910895A6E0B0E0EBEBFE
:10C17000F0E60C94F9EA0E942379382E8091B714E6
:10C1800084FB662460F8412C84FF03C00E9436794A
:10C19000482E0E947FC6209164072D83522E2B5F6C
:10C1A000298380E00FED14E091E0792E7518952D2C
:10C1B00091959A8397E8E92E90E6F92E2CEFC22EFE
:10C1C00024E0D22E92E095199B8393E095199C83ED
:10C1D0003BE9832E34E0932E40EBA42E44E0B42EB2
:10C1E0009D812981921709F409C2992349F13110DF
:10C1F0006AC00E94797F882309F47AC19D819130B9
:10C2000009F444C122E02E832D818E8128135FC161
:10C2100080916707281709F46EC180916A0188230D
:10C2200009F455C16D81651981E0909167072D81F1
:10C23000921380E023E048ED54E00E94CBC547C153
:10C2400080916707882379F180916A01882379F2C8
:10C2500081E090916707911180E024E048E055E08B
:10C260006A810E94CBC5332021F224E02E839D8178
:10C270002E8192134AC080916707981709F44CC128
:10C2800080916A01882309F440C06D81651981E0BD
:10C29000909167072D81921380E023E04CEC54E0ED
:10C2A0000E94CBC532C080914E0710924E07882362
:10C2B00059F20E94674880916607882329F22696E2
:10C2C000E2E10C9415EB8D81813009F47FC082305E
:10C2D00009F4A6C09D81933041F6809167078330B1
:10C2E00009F4C3C080916A01882309F4BECF81E0BC
:10C2F00090916707933009F080E023E04CEE54E022
:10C300006C810E94CBC584E08E838E818F5F9D817E
:10C31000981316C080916707981709F40EC1809191
:10C320006A01882369F06D81651981E09091670742
:10C330002D81921380E023E04EEB54E00E94CBC5A8
:10C340008E818E5F662009F430C141103BC09D8113
:10C3500098131BC020906707921509F4FFC08091C5
:10C360006A01882391F01F92BF92AF928D81851947
:10C370008F9381E02D81221180E08F930E943422DF
:10C380000F900F900F900F900F908E818D5F9D8179
:10C39000981316C080916707981709F4F5C080912B
:10C3A0006A01882369F06D81651981E090916707C2
:10C3B0002D81921380E023E04FE954E00E94CBC529
:10C3C0008E818C5F9D819F5F9D830ACF80916707DF
:10C3D0008130D1F080916A01882309F446CFFF9221
:10C3E000EF92DF92CF927F9281E090916707913038
:10C3F00009F080E08F930E9434220F900F900F90ED
:10C400000F900F900F9031CF80914E0710924E07F2
:10C41000882301F37CDE809166078823D9F24FCF11
:10C4200080916707823091F080916A01882309F436
:10C430001CCF81E090916707923009F080E023E003
:10C4400041EF54E06B810E94CBC50FCF80914E0726
:10C4500010924E07882341F38EE993E50E94D5C6DA
:10C4600080916607882301F32ACF80914E071092AE
:10C470004E07882309F436CF85E898E40E94D5C694
:10C4800080916607882309F42DCF19CF8091670723
:10C49000813009F180916A01882309F4B3CE8BE8D9
:10C4A00091E49F938F931F930F937F9281E09091DC
:10C4B0006707913009F080E08F930E9434220F903B
:10C4C0000F900F900F900F900F9082E08E838E81CF
:10C4D0008F5F8E83CCCE80914E0710924E078823BB
:10C4E000C9F20E948B4180916607882399F2E7CEBA
:10C4F00091E09E8389CE80914E0710924E0788234B
:10C5000009F48BCE82EF9CE40E94D5C68091660729
:10C51000882309F482CED3CE80914E0710924E0725
:10C52000882309F4ADCE8EE49AE40E94D5C68091AA
:10C530006607882309F4A4CEC2CE80914E071092DC
:10C540004E07882309F4EBCE8AE99DE50E94D5C603
:10C5500080916607882309F4E2CEB1CE80914E0720
:10C5600010924E07882309F4FACE4FE350E06AE8B0
:10C5700074E086EE96E00E946AED8091660788235B
:10C5800009F4EDCE8D811ECF80914E0710924E079B
:10C59000882309F404CF8FE694E60E94D5C68091E3
:10C5A0006607882309F4FBCEEDCF9D81981314C054
:10C5B000909167072D81291791F080916A01882356
:10C5C00059F06D81651981E02D81291380E020E209
:10C5D0004EE854E00E94CBC58E818D5FF3CE8091F2
:10C5E0004E0710924E07882341F39092E506809201
:10C5F000E40680916607882301F3C4CF8093650722
:10C600005ECE10928B07109269010E94367990914C
:10C61000B71480FB97F99093B71460E08AEC91E02F
:10C620000E9457580C94D5440F931F930E9400CB3F
:10C630000091900210919102209192023091930208
:10C64000601B710B820B930B97FD0CC089B183FBB0
:10C65000882780F991E089274A9B8260309B84601B
:10C6600080938F0280918F02817090918F0291FD53
:10C67000826090919903981749F0813009F148F050
:10C68000823079F0833091F0809399031F910F915C
:10C690000895913079F09230B9F790918E029150CF
:10C6A0000CC0992339F09330C1F3EECF9130A9F348
:10C6B000923051F790918E029F5F90938E02E4CF5B
:10C6C000992359F3933001F7F5CF1F93CF93DF935D
:10C6D000809135018F3708F475C08F579091B6124D
:10C6E00090939904992309F46BC05D9A9091350752
:10C6F00090939804992309F46FC05C9A8F5F80939C
:10C7000035018091970491E08927809397048111E6
:10C710008BDF8091340191E0980F85300CF090E030
:10C72000823009F4A8C00CF059C0882309F46EC007
:10C73000813009F495C090933401C0917807D0916D
:10C740007907209709F42DC0F89413B1147082E092
:10C750000E94302B00C000C01C161D060CF0B9C092
:10C760002A9A00C000C02B9A00C0000082E090E02E
:10C770000197F0F72B9800C000C0112309F4ABC05B
:10C780002A9A00C000C07894809178079091790728
:10C790001C161D060CF0A1C0019790937907809399
:10C7A00078078091B30D9091B40D009729F001970F
:10C7B0009093B40D8093B30DDF91CF911F910895A5
:10C7C0005D9894CF90919904891708F05D989091A5
:10C7D0009804891708F492CF5C9890CF843009F4BC
:10C7E00061C00CF45BC0853009F0A5CF20919604A0
:10C7F000211102C080939604809196048150809309
:10C800009604882309F497CF95E095CF8091330162
:10C810008F5F80311CF4809333018DCF10923301F0
:10C8200080919803811113C02091AC123091AD1208
:10C830003093AF122093AE1220912B0730912C072A
:10C8400030932E0720932D0781E080939803109258
:10C85000AD121092AC1210922C0710922B076BCFD6
:10C8600010927B0087E480937C0080917A00806442
:10C8700080937A0060CF80917A0086FD26C0409137
:10C880007800509179002091AC123091AD12240FB4
:10C89000351F3093AD122093AC124DCF10927B0018
:10C8A00086E4E1CF80917A0086FD11C04091780046
:10C8B0005091790020912B0730912C07240F351FC0
:10C8C00030932C0720932B0736CF92E034CF94E09F
:10C8D00032CF2A9846CF2A9854CF01965ECFACE348
:10C8E000B0E0E5E7F4E60C94F9EA80916807882364
:10C8F00069F18091B71410E000E084FF23C080EE5E
:10C9000092E10E94C0238BE1E0EEF2E1DE0191961C
:10C9100001900D928A95E1F710E000E0BE016F5F93
:10C920007F4FCE0181960E94E3D418163CF4CE01CD
:10C9300001960E9456CF080F111DF0CFCE018196AF
:10C940000E9490251093E8030093E7030E947FC69E
:10C9500010916407312E85E0810F8CAF212E219438
:10C9600086ECA82E8CE1B82E91E5892E95E0992EC3
:10C9700001E0011B26E5622E25E0722E111113C085
:10C9800080916707882391F180916A01882359F08B
:10C9900081E090916707911180E024E04FE555E038
:10C9A000622D0E94CBC58091B71486FF3EC0113026
:10C9B000D9F480916707813049F180916A01882319
:10C9C00009F43EC11F927F926F920F9381E0909184
:10C9D0006707913009F080E08F930E9434220F9016
:10C9E0000F900F900F900F9082E04FC080914E07F4
:10C9F00010924E07882341F20E9467488091660793
:10CA0000882311F2EC96E2E10C9415EB80914E072D
:10CA100010924E07882389F2109264070E943CD836
:10CA200080916607882349F2EDCF84FF2DC0113035
:10CA3000D9F6809167078130D1F080916A0188230F
:10CA400009F4FEC0BF92AF929F928F920F9381E044
:10CA500090916707913009F080E08F930E94342213
:10CA60000F900F900F900F900F900F90BDCF80916F
:10CA70004E0710924E07882301F30E94C61C809136
:10CA800066078823D1F2BECF81E090916A01992395
:10CA900009F4D7C0582ED12CC12C412E4318852D16
:10CAA000E090E703F090E803CE14DF0408F0C9C07B
:10CAB0005112A5C091E0E91AF108EC18FD0880EECA
:10CAC00092E10E94C0238BE1E0EEF2E1DE0191965B
:10CAD00001900D928A95E1F7F12CBE016F5F7F4FB7
:10CAE000CE0181960E94E3D418167CF4CE01019603
:10CAF0000E9456CF882389F3EF106BC0BE016F5F91
:10CB00007F4F8AE797E00E9471CFCE0181960E9405
:10CB100090258091B7149091670785FF75C0911398
:10CB200063C080914E0710924E07882309F45CC0C1
:10CB300019821C828091E3126BEF72E1882311F05D
:10CB400060EE72E121E04AE757E0CE0101960E94D3
:10CB50009525882309F43FC08BE1FE013196A0EEB4
:10CB6000B2E101900D928A95E1F78091B7148F7B25
:10CB70008093B714A091AD14AA3080F481E08A0F9D
:10CB80008093AD148BE18A9FD0011124A156BC4E35
:10CB9000E0EEF2E101900D928A95E1F7CE01019667
:10CBA0000E9490251092640782E090E0A0E0B0E03F
:10CBB0008093690790936A07A0936B07B0936C0703
:10CBC00081E0809366071092940283E080936A016B
:10CBD00019CFF39482CF0E94EF856AE777E08BE369
:10CBE00095E00E9431CFDACF80916A01882339F035
:10CBF00081E0911380E041E0642D0E9409C68FEF2F
:10CC0000C81AD80A53944BCF911759F080916A01F2
:10CC10008823A9F381E090916707911380E040E0B9
:10CC2000EBCF80914E0710924E07882379F38AE567
:10CC300093E50E94D5C680916607882339F3E2CE3A
:10CC400082E01F5F9CAD911399CE80936507DACE89
:10CC5000FC01A081B1811C92A281B3818C918F5F74
:10CC60008C930280F381E02D90818CE0989F800D61
:10CC70001124E1E6F3E113AE84AF0895FC01849141
:10CC80000895FC0180810895009751F0FC0180E037
:10CC90009191992331F0907C9038D1F38F5FF8CF48
:10CCA00080E00895119800C087FD43C0419800C0FE
:10CCB000119A00C000C0119800C086FD46C041987E
:10CCC00000C0119A00C000C0119800C085FD3BC093
:10CCD000419800C0119A00C000C0119800C084FDA6
:10CCE00030C0419800C0119A00C000C0119800C027
:10CCF00083FD25C0419800C0119A00C000C0119862
:10CD000000C082FD1AC0419800C0119A00C000C046
:10CD1000119800C081FD0FC0419800C0119A00C059
:10CD200000C0119800C0419800C0119A00C000C016
:10CD30000895419ABCCF419AF0CF419AE5CF419AEC
:10CD4000DACF419ACFCF419AC4CF419AB9CF90E080
:10CD500080E00895CF93DF93DB01F9019C9191303E
:10CD6000C1F0943080F094509C938830D1F480814D
:10CD70009181009771F0019791838083480F591F2B
:10CD8000EA01188206C08C3539F49C5F9C9394307C
:10CD900041F4DF91CF9108958B3339F781E08C9383
:10CDA000F8CF20813181B9016F5F7F4F718360833C
:10CDB000420F531FEA018883808191818F3591054D
:10CDC0006CF7E7CF0F931F9381E00091B31410919C
:10CDD000B4142091B5143091B6144091AF14509111
:10CDE000B0146091B1147091B2140417150726079E
:10CDF000370708F480E01F910F91089590E080E0DC
:10CE000008952091FC05833021F425FD0CC024FDFC
:10CE10000CC030E0A90102C0559547958A95E2F70C
:10CE2000CA018170089581E0089580E0089580919D
:10CE3000170684FD0BC08091190687FD07C09091ED
:10CE40001A06937081E019F480E0089581E0089556
:10CE50002FEB280F2A3108F047C0E22FF0E0809135
:10CE6000170690911806A0911906B0911A0604C0F1
:10CE7000B695A795979587952A95D2F780FD02C01C
:10CE800081700895E350FA4FE081EE2341F18091E3
:10CE9000890790918A07E80FF92FF11D808190EDA5
:10CEA000980F9A3030F08E3251F4818180538A305D
:10CEB00098F4F093ED05E093EC0581E008958D3250
:10CEC00011F08B3249F4818190ED980F9A3088F3FC
:10CED0008E3211F48281EACFF0E0E0E0EACF1092E6
:10CEE000ED051092EC05E9CF80E00895CF93DF9334
:10CEF00085E4AEDF882309F188E040911706509160
:10CF000018066091190670911A06972F9170C92F13
:10CF100090E0D92FCC0FDD1F71FB222720F930E0E4
:10CF2000220F331F220F331FC22B67FB442740F908
:10CF3000C42B8C2BDF91CF91089580E0DECF88DF6A
:10CF4000882341F081E02091EC053091ED05232B01
:10CF500009F480E00895CF93DF93C0913307D09117
:10CF60003407209729F160912F0770913007809145
:10CF70003107909132070E9410EC6E5F7F4F24972B
:10CF80006C177D07ACF470939203609391030E9439
:10CF900000CB605A75418F4F9F4F609393037093FE
:10CFA00094038093950390939603DF91CF91089516
:10CFB000109293031092940310929503109296038B
:10CFC000F4CFB0E0A0E0E7EEF7E60C9402EB6B01E3
:10CFD000E9014A3009F4D5C0453109F081C0DB01CF
:10CFE0001296ED91FC91F28096818781139A00C090
:10CFF0000000E6E2F0E03197F0F7092F182FEF2C50
:10D00000E29420EFE22230E1B32EBF0CE80188EF7A
:10D0100049DE00C0000086E290E00197F0F7BFE132
:10D02000BF1508F49BC08F2D807780683BDE8E2D66
:10D0300039DE00C0000086E290E00197F0F780E85A
:10D0400031DE80E02FDE00C0000086E290E0019734
:10D05000F0F78AEF27DE00C0000086E290E001973B
:10D06000F0F7005F1F4F8881807F1CDE89918295D9
:10D07000807F18DEC017D107B1F700C0000086E23C
:10D0800090E00197F0F7F394E0E1EE0EFB10BECFD5
:10D090001398D6011296ED91FC9180819281980FA0
:10D0A00092832181921708F09FC194819F5F94839E
:10D0B0009381890F821710F08FEF820F8383458150
:10D0C00050E0440F551F70E060E0868197810E9418
:10D0D00030ED81E0CDB7DEB7E9E00C941EEBDEC1A8
:10D0E000FB0102811381423309F485C108F48DC12B
:10D0F000463409F475C1473409F482C14B3349F70A
:10D1000089812B81D80112967C91129713963C91BC
:10D11000213009F4BFC1233009F0A0C148EF480F06
:10D12000582F91E0341708F490E031E0541708F0DC
:10D1300030E0492F432B61E0571708F460E04623A5
:10D1400011F4932331F2FA8030E0F901E65CFD4FEF
:10D15000D0802A5C3D4FF901E08099C180EE8F0DAF
:10D160008068807F9FDD8F2D8295807F9BDD00C052
:10D17000000086E290E00197F0F780E893DD80E818
:10D1800061CF0B9A1398399A4198099A119A139A78
:10D1900000C0000086E290E00197F0F788E790E099
:10D1A000CEE9DFE0FE013197F1F70197D9F788EF7B
:10D1B00079DD00C0000086E290E00197F0F780E2A0
:10D1C00071DD80E06FDD00C0000086E290E0019735
:10D1D000F0F780E067DD80E865DD00C0000086E2F2
:10D1E00090E00197F0F780E05DDD80E15BDD00C05D
:10D1F000000086E290E00197F0F7CE010197F1F789
:10D20000CE010197F1F7CE010197F1F7CE01019719
:10D21000F1F7CE010197F1F7CE010197F1F7CE01B9
:10D220000197F1F7CE010197F1F7CE010197F1F7E0
:10D23000CE010197F1F7CE010197F1F7CE010197E9
:10D24000F1F7CE010197F1F7CE010197F1F72197A0
:10D25000F1F780E227DD80E425DD00C0000086E2F2
:10D2600090E00197F0F780E21DDD80E61BDD00C055
:10D27000000086E290E00197F0F7D0E0C0E08C2F4C
:10D28000807780680FDD8D2F0DDD00C0000086E205
:10D2900090E00197F0F780E805DD80E003DD00C055
:10D2A000000086E290E00197F0F78AEFFBDC00C017
:10D2B000000086E290E00197F0F780E2119800C04C
:10D2C000419800C0119A00C000C0119800C0419858
:10D2D00000C0119A00C000C0119800C0419800C061
:10D2E000119A00C000C0119800C0419800C0119A66
:10D2F00000C000C0119800C0419800C0119A00C041
:10D3000000C0119800C0419800C0119A00C000C030
:10D31000119800C0419800C0119A00C000C0119837
:10D3200000C0419800C0119A00C000C0119800C010
:10D33000419800C0119A00C000C0119800C04198E7
:10D3400000C0119A00C000C0119800C0419800C0F0
:10D35000119A00C000C0119800C0419800C0119AF5
:10D3600000C000C0119800C0419800C0119A00C0D0
:10D3700000C0119800C0419800C0119A00C000C0C0
:10D38000119800C0419800C0119A00C000C01198C7
:10D3900000C0419800C0119A00C000C000C0000049
:10D3A000E6E2F0E03197F0F7815009F087CF88EF9F
:10D3B00079DC00C0000086E290E00197F0F7CF5FD3
:10D3C000D05FC03209F05BCF80E06CDC80EC6ADCBF
:10D3D00000C0000086E290E00197F0F7139879CE44
:10D3E000F8018581888375CE80E0CDB7DEB7E9E0AE
:10D3F0000C941EEB53C0B901C8010E9435CC69CE14
:10D40000D80111968C91888364CE443191F04731D4
:10D4100009F05FCE1882D80112968C9112978983F9
:10D4200015968C91159781508A8313968C918B83D6
:10D4300050CED80115964C91159750E0440F551FCA
:10D4400070E060E016968D919C910E9430EDF8019D
:10D45000128280818150838314823BCE381708F476
:10D4600038CE871708F435CEFA80E12CD12C243041
:10D4700070F46ACEBE01C8010E9435CC89819881C2
:10D480009D0D98838E0D8983FF0C09F422CEF7FE43
:10D49000F6CFF0CF58E0580F482F43CEEF92FF92CF
:10D4A0000F931F93CF93DF93EC018B017A018A8551
:10D4B0009B858617970731F0888199810E9422CE3B
:10D4C0001B870A87B701888199810E9441C62E81F6
:10D4D0003F81820F932F911D9F838E8390E080E088
:10D4E000CDB7DEB7E6E00C9421EBB0E0A0E0EBE7CF
:10D4F000FAE60C9401EBEC017B018A018A859B859D
:10D500008617970731F0888199810E9422CEFB8689
:10D51000EA8688859985019609F5CC80DA808E8126
:10D52000D80EA880B980D5015596ED91FC91C50122
:10D530000995C80E780110E0F70121917F012111B2
:10D540001FC08E819F81810F911D9F838E8390E0EC
:10D5500080E0CDB7DEB7EAE00C941DEBEE80FF80F3
:10D56000B801888199810E9441C68E0D9F2D911D21
:10D57000288539852817390780F681E090E0E9CFC2
:10D580004C2D6D2DC5010E947ACED80E180FD4CF28
:10D59000B0E0A0E0EEECFAE60C9404EBEC01D62E41
:10D5A0001CAD0BAD7C0184E0E80EF11CE98DFA8D19
:10D5B000C7010995412F480F2D2D602FC7010E94EB
:10D5C0007ACE9BAD890F8BAF81E090E0CDB7DEB70F
:10D5D000E7E00C9420EB682F70E090E080E00C9482
:10D5E0004EAD8091EC059091ED05009731F04AE049
:10D5F00050E070E060E00C9434E260E070E0CB0159
:10D6000008958091EC059091ED05009731F04AE086
:10D6100050E070E060E00C9407E160E070E0CB0166
:10D620000895EFDF97FD0AC0ECDF6F3F71058105BC
:10D63000910509F02CF4E5DF862F089580E0089528
:10D640008FEF0895CF93C62F7ADC882311F0E9DF9E
:10D65000C82F8C2FCF9108958091EC059091ED0506
:10D66000892B39F0DEDF91E0811101C090E0892F34
:10D67000089591E0FCCFCF93DF93C82FD62F5FDCC6
:10D68000882321F0E9DFDF91CF9108958C2FE0DB33
:10D690008111F9CF8D2FF7CFB4DFCB010895CF9350
:10D6A000DF93EB014CDC882311F0F6DFEC01CE01B7
:10D6B000DF91CF9108950F931F93CF938091EC0545
:10D6C0009091ED050097D9F0FC018F01C1912C2FAD
:10D6D0002F7D81F0C53411F0C536B9F7F8011082FD
:10D6E00070E060E00E94B1DFF801C083CF911F912C
:10D6F0000F91089570E060E00E94B1DFF7CF60E025
:10D7000070E0CB01F3CFCF92DF92EF92FF926A01EC
:10D710007B0115DC882319F0CEDF6B017C01C7018A
:10D72000B601FF90EF90DF90CF900895CF92DF92F7
:10D73000EF92FF92CF93C82F0E9400CB6B017C0128
:10D7400024EA30E74DE75FE3609108017091090139
:10D7500080910A0190910B010E9413E487FD18C08B
:10D760008AEF90E0A0E0B0E08C0D9D1DAE1DBF1DC6
:10D770008093580690935906A0935A06B0935B067F
:10D78000C0935D01CF91FF90EF90DF90CF9008950F
:10D7900080E090E0DC01E8CFCF93809127068111F3
:10D7A00054C010929C1310929D1310929E131092CD
:10D7B0006A131092691310926C1310926B131092EB
:10D7C0006E1381E080936D1382E280936F13109249
:10D7D000741310927313E8E8F3E126E933E18FEF55
:10D7E00081932E173F07E1F7C1E0C093851322E82C
:10D7F0003BEA30937B1320937A13C0937C131092EF
:10D800007D1310927E1390E490937F1310928013F7
:10D8100021E83BEA309397132093961325E531E0F6
:10D8200030936813209367139EE190938C1391E1DA
:10D8300090938D139CE190938A1380938913809326
:10D8400088130E9474CCC093270681E0809326063B
:10D8500083E191E29093A3128093A2121092A512F9
:10D860001092A41253985B9A52985A9A3898409AF8
:10D870000E94146310928E02CF910895FC0180E003
:10D88000309749F09491992331F0907C903809F0C9
:10D890008F5F3196F7CF0895B0E0A0E0E2E5FCE6B7
:10D8A0000C9401EBEC015B018A01FB01099587FDFA
:10D8B00010C0C82ED12CF12CE12C2196F801C08289
:10D8C000D182E282F382CE01CDB7DEB7EAE00C94DA
:10D8D0001DEB982F907E903CA9F48F7190E0B0E002
:10D8E000A0E06C017D0156E0CC0CDD1CEE1CFF1CA1
:10D8F0005A95D1F7CE010196F50109958F73C82A83
:10D900002296DCCF982F907F903E11F58F7090E09B
:10D91000B0E0A0E06C017D0136E0CC0CDD1CEE1C1B
:10D92000FF1C3A95D1F7CE010196F50109958F7349
:10D93000C82A46E0CC0CDD1CEE1CFF1C4A95D1F732
:10D94000CE010296F50109958F73C82A2396B6CFAA
:10D95000982F987F903F79F5877090E0B0E0A0E035
:10D960006C017D0186E0CC0CDD1CEE1CFF1C8A9551
:10D97000D1F7CE010196F50109958F73C82A96E07B
:10D98000CC0CDD1CEE1CFF1C9A95D1F7CE01029643
:10D99000F50109958F73C82A26E0CC0CDD1CEE1C1E
:10D9A000FF1C2A95D1F7CE010396F50109958F73D7
:10D9B000C82A249683CF982F907C903841F4807C9D
:10D9C000803869F42196CE01F5010995F8CF8E7F54
:10D9D0008D3F28F02196CE01F5010995F8CFC12C95
:10D9E000D12C76016BCF9CE0899F802D112491E092
:10D9F000980F909325062CE0280F2093720730E0B3
:10DA00002E5F3F4F409199134217130619F014F0FF
:10DA100080E0089520919B139217D0F7662341F080
:10DA20008E5F0E9459CD809172078E5F0E9459CD02
:10DA30008091720790919913891750F320919B134D
:10DA400090912506291720F310929C1380939D1323
:10DA500081E0089520912406022E000C330B8217DA
:10DA6000130641F0809324066EE772E285E693E1A7
:10DA70000C9422CE0895ACE0B0E0E1E4FDE60C9415
:10DA800003EB6F3F71058105910509F070F481E6A4
:10DA900093E17EDDE0916913F0916A1331968491F0
:10DAA00090E02C96E8E00C941FEBF0909C13E09033
:10DAB0009D132091260621110FC045EE50E26E2DD8
:10DAC0008F2D0E94D3CE90E080E0F80EF0929C1350
:10DAD000E0929D139927E5CFC0906913D0906A1307
:10DAE00025E633E13A8329832F2D30E03C832B83D5
:10DAF0002E2D30E03E832D8318861F822FEF3FEFBF
:10DB00003A8729871C861B8605E71AE69E012F5F48
:10DB10003F4FAB01BC01C6010E9490ACB60185E647
:10DB200093E10E9422CE8F819885CFCF4F925F9252
:10DB30006F927F928F929F92BF92CF92DF92EF92DD
:10DB4000FF920F931F93CF93DF93CDB7DEB7289744
:10DB50000FB6F894DEBF0FBECDBF7C016A0149014C
:10DB6000FB0190818CE0989F800D1124982FF70184
:10DB70002081822F880F820F880F80939C139093AF
:10DB80009D134115510559F1FA82E9827C836B831B
:10DB900001111EC0AE014B5F5F4FB401C6017CDEB8
:10DBA0006C016D817E818F8198856115710581057C
:10DBB0009105A9F060DFF70180818F5F8083853157
:10DBC00048F3CE01019644D8E5CFB12C860129C097
:10DBD0008A01B12C26C0452846284728B1F7289647
:10DBE0000FB6F894DEBF0FBECDBFDF91CF911F916E
:10DBF0000F91FF90EF90DF90CF90BF909F908F900C
:10DC00007F906F905F904F900895B39407C0B110CC
:10DC10002DC001151105C9F20F5F1F4F0115110528
:10DC2000A9F2AE014B5F5F4FB401C60135DE6C0156
:10DC30004D805E806F8078844114510461047104CA
:10DC4000A9F0F0E24F1651046104710401F3D3010D
:10DC5000C2018D97A109B1090297A105B10530F064
:10DC60004BE2441651046104710479F6F701808196
:10DC7000482F4B0D5527551F4631510534F085303F
:10DC800020F0CE0101960E94286681E041145104E3
:10DC90006104710409F480E0B80EF70180818B0DF6
:10DCA0008083BB2009F497CFBA94AE014B5F5F4FDE
:10DCB000B401C801F1DD8C016D817E818F81988571
:10DCC000DADEEFCFCF93DF93FC0125AD211104C045
:10DCD00021E025AF0E9474CCC0916713D0916813E6
:10DCE000E0919613F091971382E00995E0919613D5
:10DCF000F091971381E0099530E020E044E1BE0106
:10DD000085E693E10E946FCC28E933E147E1BE014B
:10DD100085E693E10E946FCCE0919613F091971302
:10DD200080E00995DF91CF9108954F925F926F92B5
:10DD30007F928F929F92AF92BF92CF92DF92EF929B
:10DD4000FF921F93CF93DF9300D000D0CDB7DEB703
:10DD50000E9400CB6B017C0180915D018F3FC1F17E
:10DD60000E9400CB8090580690905906A0905A06C9
:10DD7000B0905B06681979098A099B0997FD28C04C
:10DD80008091391390913A138F5F8F70891701F149
:10DD9000E0915D01E53008F054C024E0E29FF0011D
:10DDA0001124E25CFD4F80819181A281B38189833E
:10DDB0009A83AB83BC8320E030E0A901BE016F5F92
:10DDC0007F4F85E791E00E94C4C08FEF80935D0193
:10DDD0000E94146380918F0282FF3CC0809167068D
:10DDE00081113AC091E09093670680918B07892753
:10DDF00080934E0710928B0783E080936A01109204
:10DE00008F020E9400CB6C507E4F8F4F9F4F6093CC
:10DE1000900270939102809392029093930268E82B
:10DE200073E182E090E00E94594316E01150A1F0A6
:10DE30000E94FD4262E070E080E090E00E9474CABF
:10DE4000F5CF80916B0190916C01A0916D01B09123
:10DE50006E01ADCF109267068091630690916406C3
:10DE6000A0916506B0916606A7019601281B390BA3
:10DE70004A0B5B0BDA01C901B7FF05C08091940220
:10DE8000882309F4B9C1D701C6018C599F4FAF4F00
:10DE9000BF4F8093630690936406A0936506B0938A
:10DEA000660660918E02062E000C770B77FF03C08A
:10DEB00071956195710990918E0280916206981317
:10DEC00065C0633008F062C010928E0280918E02AD
:10DED00080936206643008F069C080914E0781111A
:10DEE000E7C080915F13909160138454994741F487
:10DEF00080915E01882309F4EDC0815080935E011A
:10DF00000E94852E8090A5079090A607A090A70755
:10DF1000B090A80781110E94922ED501C4013AE069
:10DF2000B695A795979587953A95D1F7009741E0D3
:10DF3000A407B10520F08FEF9FEFA0E0B0E0969529
:10DF4000879520916A012111D7C030919402311137
:10DF500080C180915F13909160138454994709F4B4
:10DF60005FC18091950281115BC180915E069091A5
:10DF70005F06A0916006B0916106C81AD90AEA0A44
:10DF8000FB0AF7FC5BC10E94D54458C1633009F01D
:10DF90009DCF80918E0287FD07C081E0880F880F9A
:10DFA00080938E0264E092CF8FEFF8CF809171075B
:10DFB00021E030E040E050E0882309F456C0809032
:10DFC0006D0790906E07A0906F07B0907007811456
:10DFD0009104A104B104E9F170E090E080E00E94B6
:10DFE00017E420E030E040E85EE30E9478E42B0193
:10DFF0003C01C701B601681979098A099B090E9489
:10E0000017E49B01AC01C301B2010E94A8EB20E020
:10E0100030E04AE754E40E9478E44B015C0120E0E0
:10E0200030E040EA52E40E9494EC24E630E040E024
:10E0300050E087FF12C020E030E040EF51E4C5011E
:10E04000B4010E9494EC2AE030E040E050E087FF09
:10E0500004C021E030E040E050E0C0926D07D09273
:10E060006E07E0926F07F0927007A0918E020A2E61
:10E07000000CBB0B0E94F3EA24E030E040E050E0EB
:10E080000E94BCEA8091690790916A07A0916B0792
:10E09000B0916C07820F931FA41FB51F809369076F
:10E0A00090936A07A0936B07B0936C0710928E024F
:10E0B000D701C6018856954CAF4FBF4F80935E067F
:10E0C00090935F06A0936006B093610681E0809311
:10E0D0006A0107CF8CE080935E0180915C0690918D
:10E0E0005D06009729F0019790935D0680935C068A
:10E0F00081E080936A0104CF009741F040915C0673
:10E1000050915D064817590708F023CF809194027B
:10E11000811111C0223038F0243008F43FC024307F
:10E1200011F410926A0181E693E1CCDD81E08093E5
:10E1300068078093940283E08DDC81E080938513EF
:10E14000E0915F13F0916013099510926807809138
:10E150009402811127C010924E0780915F13909115
:10E1600060138454994709F0FCCE0E9400CBDC0177
:10E17000CB018C199D09AE09BF0980905C06909077
:10E180005D06B12CA12C88169906AA06BB0608F0DC
:10E19000E0CE90935D0680935C06DBCE81E08093B9
:10E1A0006A01C1CF85E693E10E94F2CD91E0811131
:10E1B00001C090E090939402882369F280915F13EC
:10E1C0009091601384549947B9F40E9400CBDC010C
:10E1D000CB018C199D09AE09BF09C0905C06D09097
:10E1E0005D06F12CE12CC816D906EA06FB0620F4E0
:10E1F00090935D0680935C060F900F900F900F90A8
:10E20000DF91CF911F91FF90EF90DF90CF90BF9063
:10E21000AF909F908F907F906F905F904F900895F8
:10E2200048E9C40E4AE3D41EE11CF11CC0925E060C
:10E23000D0925F06E0926006F092610680919402AF
:10E240008111DACF80916A018130B1F610926A01B2
:10E25000D3CF009709F46FCF51CFACE0B0E0E3E348
:10E26000F1E70C9403EBF0909C13E0909D13209148
:10E270002606211112C045EC50E26E2D8F2D0E9412
:10E28000D3CE90E080E0F80EF0929C13E0929D13C4
:10E2900099272C96E8E00C941FEBC0906913D0905E
:10E2A0006A1325E633E13A8329832F2D30E03C833E
:10E2B0002B832E2D30E03E832D8318861F827A8794
:10E2C00069871C861B8605E71AE69E012F5F3F4F74
:10E2D0004EE356E6BC01C6010E9425ADB60185E6B7
:10E2E00093E10E9422CE8F819885CDCFA4E0B0E04B
:10E2F000ECE7F1E70C94FFEA7C01062F5A01122F9C
:10E30000862F660F990B9C012E5C3D4F690186E0BC
:10E31000882E912C11160CF03DC0AE014F5F5F4F5F
:10E320006EE376E6C701B8DA7C0169817A818B8178
:10E330009C81611571058105910561F16D33710550
:10E340008105910509F450C06E377105810591056D
:10E3500009F44AC06A3271058105910501F507FF8C
:10E3600011C089E091E20E3F11F085E091E236E0C4
:10E370001302B001112471DF66E070E00E94A9EA87
:10E38000161B60C065E470E080E090E074DB115023
:10E3900069F510E0812F2496ECE00C941BEB6432BD
:10E3A00071058105910571F4A114B104D1F0E6E085
:10E3B0001E02B0011124C50150DFB4010E94A9EA78
:10E3C000161BA8CF603471058105910551F41150D9
:10E3D000F6016081062E000C770B880B990B4BDB46
:10E3E00099CF49DB115096CF07FDBBCF61E0898102
:10E3F0009A81AB81BC81CD97A105B10509F460E09C
:10E40000600F6A30A4F01150862F6AE00E9488EAFB
:10E41000092F682F880F770B605D7F4F072E000C48
:10E42000880B990B28DB112309F4B3CF602F062E3C
:10E43000000C770B605D7F4F072E000C880B990B4B
:10E440001ADB1150112309F4A4CF86E01802B001A1
:10E450001124C70102DF66E070E00E94A9EA161BE2
:10E4600099CFE1E6F3E183AF64AF6FEF7FEFCA01CD
:10E47000F4CEACE0B0E0EFE3F2E70C9403EBF09005
:10E480009C13E0909D1320912606211112C045EAAD
:10E4900050E26E2D8F2D0E94D3CE90E080E0F80EDA
:10E4A000F0929C13E0929D1399272C96E8E00C942F
:10E4B0001FEBC0906913D0906A1325E633E13A83CD
:10E4C00029832F2D30E03C832B832E2D30E03E839B
:10E4D0002D8318861F827A8769871C861B8605E72D
:10E4E0001AE69E012F5F3F4F41E456E6BC01C6018C
:10E4F0000E9425ADB60185E693E10E9422CE8F8170
:10E500009885CDCF6FEF7FEFB4CFB0E0A0E0EBE820
:10E51000F2E70C9401EB5C016B01B0D9E82EC60167
:10E520000E944466F12C03E110E0081B1109C5E2CA
:10E530000E151F050CF4CFE18C2F90E09C012E5F8F
:10E540003F4F409199134217130609F08CF5099734
:10E5500020919B13281719065CF140917407509184
:10E5600075076091730710929C13C0939D1325E16A
:10E57000C501BCDED1E0C114D104A9F06AE370E0AA
:10E5800080E090E078DA0E151F05A4F4C45F809156
:10E590009913C81740F020919B134C2F4950550BED
:10E5A000241715064CF4CDB7DEB7EAE00C941DEB4A
:10E5B000D0E0E1CFDD23B9F3802F880F080F000FE3
:10E5C00000939C13C0939D1360E270E080E090E0A4
:10E5D00052DAC60197DFE7CFACE0B0E0E2EFF2E756
:10E5E0000C94FFEA982F862F6A017901B02E692FCB
:10E5F000FAD9882309F487C010912606C7010023A1
:10E6000071F13CD9A82E8090691390906A13111172
:10E6100042C02FEF3FEF122F23E12A1940917407D8
:10E620005091750760917307C60160DEAA2009F456
:10E630006AC0B6E08B9F600111246AE370E080E05D
:10E6400090E019DA57E0C516D10408F442C060E240
:10E6500070E080E090E00FDAC81AD90AF3CF0E9488
:10E660004466A82E8090691390906A13112389F252
:10E67000FE0133968AE0DF011D928A95E9F785E66F
:10E6800093E19A8389830EE41AE69E012F5F3F4F40
:10E6900041E456E612C0FE0133968AE0DF011D9286
:10E6A0008A95E9F785E693E19A8389830EE41AE671
:10E6B0009E012F5F3F4F4EE356E6B701C4010E9413
:10E6C00025ADB40185E693E10E9422CE2F813885E5
:10E6D000A2CF40917207212F30E0A6E0AA9EC00190
:10E6E00011242E5F3F4F281739070CF49C0180E856
:10E6F000821B80939C1340939D13BB2041F06FEFCE
:10E700007FEFC701AADD2C96ECE00C941BEBC70150
:10E71000F9DEF9CFE1E6F3E183AF64AFCA01F2CEEF
:10E720000C94ABAD4F925F926F927F928F929F92BB
:10E73000BF92CF92DF92EF92FF920F931F93CF93EE
:10E74000DF9310921C0610921B062FE320931F06E6
:10E7500010921E0610921D061092170610921806AF
:10E760001092190610921A069C01F90190812F5FF0
:10E770003F4F9032D1F39E34C9F4818190ED980FD0
:10E780009A3020F08D3211F08B3281F432969F0155
:10E790002F5F3F4F808180538A3008F46DC09F0106
:10E7A0002F5F3F4F8081803209F468C0F0938A0761
:10E7B000E09389078F010F5F1F4FC0816AE270E00D
:10E7C000C8010E944AED009731F0FC013197808129
:10E7D0008032E1F31182CD3421F0C43511F0C73419
:10E7E000D9F5F80180810F5F1F4F8032D1F380533C
:10E7F0008A3090F5C0931F0690E080E06AE0AF0198
:10E800004F5F5F4F689F9001699F300D1124C901D0
:10E81000C0972081820F911D27FD9A95FA012081D2
:10E8200020532A3060F390931E0680931D06DF016B
:10E8300031962C912032D9F3CD3461F58E3191058A
:10E8400039F0F0F48731910519F08C31910511F50B
:10E85000B0931C06A0931B06DF91CF911F910F91DF
:10E86000FF90EF90DF90CF90BF909F908F907F9020
:10E870006F905F904F900895F90189CFF9018FCF84
:10E880008537910538F08737910510F3803A13E00A
:10E890009107F1F28090890790908A0740E050E05C
:10E8A000BA0130E020E0C12CD12C7601C394FD01E7
:10E8B0003196DC91DD2309F484C0D132F1F4CD34FA
:10E8C000E1F480329105C9F440931706509318067D
:10E8D0006093190670931A06F0931C06E0931B06CA
:10E8E00063E270E0CF010E944AED009709F4B4CFD3
:10E8F000FC011082B1CFDF01DACFD154DA3108F058
:10E900005BC0DF011D91103291F0A0EDA10FAA3084
:10E91000E8F01E3271F4A181A053AA30B8F021159D
:10E92000310519F49F0121503109B12C13C0FD01AB
:10E93000E8CF1D3211F01B3291F7A181B0EDBA0F73
:10E94000BA3020F0AE3259F7A281E6CFBE2EB81809
:10E95000309759F3AD2FB0E02601370104C0440CC5
:10E96000551C661C771CDA95D2F74429552966296F
:10E970007729A350BA4FBC92A081A154AA3108F4C0
:10E98000BACFDF01D191DD2309F491CF00EDB02E94
:10E99000BD0E19E01B15A8F713EDB12EBD0E11E049
:10E9A0001B1578F7DB3269F3FD013196DC91D0322B
:10E9B00009F07DCFDF01F8CF21153105E9F69D0182
:10E9C000DBCF30931C0620931B0640931706509311
:10E9D00018066093190670931A063ECFFC016591E4
:10E9E00075918591949108958F929F92AF92BF9265
:10E9F000CF92DF92EF92FF92CF93DF93EC01809062
:10EA0000AF029090B002A090B102B090B20220E0AC
:10EA100030E0A901C501B4010E9413E4882309F480
:10EA200052C0C880D980EA80FB80A7019601C50149
:10EA3000B4010E9413E418160CF04AC02091E805B6
:10EA40003091E9054091EA055091EB05C701B60107
:10EA50000E9413E4882321F1C092E805D092E905D1
:10EA6000E092EA05F092EB052091E4053091E5058E
:10EA70004091E6055091E705C701B6010E9478E490
:10EA80009B01AC0160E070E080E89FE30E9430EB06
:10EA900060934A0170934B0180934C0190934D0118
:10EAA00060914A0170914B0180914C0190914D0110
:10EAB000DF91CF91FF90EF90DF90CF90BF90AF901C
:10EAC0009F908F90089560E070E080E89FE3F0CF22
:10EAD00060E070E0CB01ECCFB0E0A0E0E2E7F5E76A
:10EAE0000C94FBEAEC01209177033091780340917C
:10EAF000790350917A03688179818A819B810E9490
:10EB000030EB4B015C0120917B0330917C03409101
:10EB10007D0350917E036C817D818E819F810E9457
:10EB200030EB6B017C01A501940160914201709171
:10EB3000430180914401909145010E9413E4882390
:10EB400009F454C08092420190924301A092440182
:10EB5000B09245012091DC053091DD054091DE0544
:10EB60005091DF05C501B4010E9478E42B013C01FE
:10EB70000E9441EC4B015C0120E030E040EA50E4AF
:10EB80000E9413E4181634F4812C912CC0EAAC2EA8
:10EB9000C0E4BC2E20E030E0A901C501B4010E9410
:10EBA00094EC87FF03C0812C912C5401A5019401A2
:10EBB000C301B2010E9430EB6093D4057093D50578
:10EBC0008093D6059093D705C501B4010E9410EC3F
:10EBD0006093D205062E000C770B6F5F7F4F663077
:10EBE000710514F066E070E06093D005D0914001AB
:10EBF0001091D205A70196016091460170914701DD
:10EC000080914801909149010E9413E4811123C031
:10EC1000D11375C02091B8053091B9054091BA055E
:10EC20005091BB056091D4057091D5058091D605B2
:10EC30009091D7050E9478E42091BC053091BD05E4
:10EC40004091BE055091BF050E9431EBCDB7DEB7B4
:10EC5000E0E10C9417EBC0924601D0924701E0929C
:10EC60004801F09249012091E0053091E105409181
:10EC7000E2055091E305C701B6010E9478E44B011B
:10EC80005C010E9441EC6B017C0120E030E040EA35
:10EC900050E40E9413E4181634F4C12CD12CB0EACD
:10ECA000EB2EB0E4FB2E20E030E0A901C701B60155
:10ECB0000E9494EC87FF03C0C12CD12C7601A701E0
:10ECC0009601C501B4010E9430EB6093D8057093A2
:10ECD000D9058093DA059093DB05C701B6010E9440
:10ECE00010EC6093D305062E000C770B6F5F7F4FFF
:10ECF0006630710514F066E070E06093D105C09154
:10ED0000D305D11305C0809141018C1709F470C05F
:10ED10008091D2059091D305909341018093400159
:10ED20000C2E000CDD0B27E01203C0011124FC01A6
:10ED3000EC0FFD1FEE0FFF1FEE0FFF1FED54FD4FF9
:10ED400020813181428153812093CC053093CD05C0
:10ED50004093CE055093CF050091D105002E000CB5
:10ED6000110BFC01E00FF11FEE0FFF1FEE0FFF1F55
:10ED7000ED54FD4F60817181828193810E9430EB5F
:10ED80006093C8057093C9058093CA059093CB051D
:10ED90002091D00537E02303F0011124CE0FDF1FAF
:10EDA000CC0FDD1FCC0FDD1FCD54DD4F2881398105
:10EDB0004A815B812093C4053093C5054093C60505
:10EDC0005093C705E00FF11FEE0FFF1FEE0FFF1F5F
:10EDD000ED54FD4F60817181828193810E9430EBFF
:10EDE0006093C0057093C1058093C2059093C305DD
:10EDF0008090D8059090D905A090DA05B090DB05F9
:10EE00002091C8053091C9054091CA055091CB05A4
:10EE1000C501B4010E9478E42091CC053091CD0564
:10EE20004091CE055091CF050E9431EB6B017C01E2
:10EE3000C092BC05D092BD05E092BE05F092BF0520
:10EE40002091C0053091C1054091C2055091C30584
:10EE5000C501B4010E9478E42091C4053091C50534
:10EE60004091C6055091C7050E9431EBA70196015C
:10EE70000E9430EB6093B8057093B9058093BA0592
:10EE80009093BB05C7CEACE0B0E0E9E4F7E70C94A3
:10EE900008EB182F882379F020E030E0A901609179
:10EEA0007F037091800380918103909182030E947F
:10EEB00013E48823F1F08091AE028117D1F00E9413
:10EEC000B12B8CE0E6E2F2E0DE01119601900D92AA
:10EED0008A95E1F7CE010196FFDD8091AE0288238D
:10EEE00061F085E791E00E94072C1092AE020E942B
:10EEF000C43E2C96E3E00C9424EB81E08093AE02B8
:10EF000085E791E00E94D32BF2CFCF92DF92EF9270
:10EF1000FF9280E0B8DF10927B0310927C03109286
:10EF20007D0310927E031092770310927803109263
:10EF3000790310927A031092830310928403109243
:10EF400085031092860310927F0310928003109223
:10EF500081031092820343EB52E027E0C12CD12CB5
:10EF600060ECE62E6FE7F62E90E080E0FC01EE0FFD
:10EF7000FF1FEE0FFF1FE40FF51FC082D182E28258
:10EF8000F38201968730910589F72150445E5F4FE7
:10EF90002111EACFFF90EF90DF90CF9008954F922C
:10EFA0005F926F927F928F929F92AF92BF92CF9219
:10EFB000DF92EF92FF921F93CF93DF93EC01162F16
:10EFC0002091AF023091B0024091B1025091B20253
:10EFD000688179818A819B810E9413E4882309F4E6
:10EFE00097C0B090AE0280E04EDFC880D980EA8042
:10EFF000FB8020E030E0A901C701B6010E9494EC3B
:10F0000087FF03C0C12CD12C7601C092AF02D092F1
:10F01000B002E092B102F092B2022DEB37E346E883
:10F0200055EBC701B6010E9413E487FD0BC02DEB21
:10F0300037E346E855E3C701B6010E9494EC181681
:10F040000CF076C0A701960160E070E080E89FE3D5
:10F050000E94A8EB6093E4057093E5058093E605B4
:10F060009093E70580EF9FEFA9E7B4EC8093E80564
:10F070009093E905A093EA05B093EB05BB2009F452
:10F0800047C0409075015090760160907701709074
:10F0900078018090790190907A01A0907B01B090E6
:10F0A0007C01C0907D01D0907E01E0907F01F090C6
:10F0B000800181E0E8DE112359F1A3019201609102
:10F0C00075017091760180917701909178010E948D
:10F0D00013E481111BC0A501940160917901709125
:10F0E0007A0180917B0190917C010E9413E481114F
:10F0F0000DC020917D0130917E0140917F015091A2
:10F100008001C701B6010E9413E481110E94EA3E0A
:10F11000DF91CF911F91FF90EF90DF90CF90BF9044
:10F12000AF909F908F907F906F905F904F900895D9
:10F1300060E070E0CB018ECF8F929F92AF92BF9232
:10F14000CF92DF92EF92FF92C0907F03D090800326
:10F15000E0908103F090820320E030E0A901C70134
:10F16000B6010E9413E48823E1F1A701960160E053
:10F1700070E080E89FE30E94A8EB6B017C01809027
:10F18000830390908403A0908503B090860320E0D1
:10F1900030E0A901C501B4010E9413E4882329F1DC
:10F1A000A501940160E070E080E89FE30E94A8EB75
:10F1B000C092DC05D092DD05E092DE05F092DF051D
:10F1C0006093E0057093E1058093E2059093E30579
:10F1D000FF90EF90DF90CF90BF90AF909F908F9077
:10F1E0000895C12CD12C7601CACF60E070E0CB012C
:10F1F000DFCFCF92DF92EF92FF926B017C0183E32E
:10F20000C816D104E104F10470F082E3C81AD108F1
:10F21000E108F10862E370E080E090E00E9474CAC7
:10F220000E94F328ECCFC701B6010E9474CA0E9465
:10F23000F328FF90EF90DF90CF900895BC0190E00D
:10F2400080E00C944EAD80918707813069F09091F9
:10F25000B71492FB882780F992FF07C097FB882795
:10F2600080F991E08927089581E008959091B7147D
:10F2700094FB882780F994FF06C081E09091C81222
:10F28000911101C080E00895A4E0B0E0EAE4F9E75C
:10F290000C94FBEA1092710780914E0710924E0772
:10F2A000882361F020E040E070E060E085EB90E6CC
:10F2B0000E9499432496E0E10C9417EB20911001F1
:10F2C000309111014091690750916A07CA01820F7C
:10F2D000931F2436310509F01DC44730510544F011
:10F2E00006978A3091050CF024C48AE090E02BC484
:10F2F00006964A3F5F4FACF380916807882309F474
:10F30000C8C16091B4127091B512072E000C880B21
:10F31000990B0E9419E4B1E0B9832091B0123091A9
:10F32000B1124091B2125091B3120E9494EC18168F
:10F330000CF019826091330770913407072E000C8E
:10F34000880B990B0E9419E420912F073091300708
:10F3500040913107509132070E9494EC18161CF42A
:10F36000E981E260E983C980C0925706C0907501C7
:10F37000D0907601E0907701F0907801809179014A
:10F3800090917A01A0917B01B0917C0189839A834D
:10F39000AB83BC8380907D0190907E01A0907F0123
:10F3A000B090800120E030E04AE754E4C501B401A8
:10F3B0000E9478E42B013C0120E030E0A901C50166
:10F3C000B4010E9413E420E030E040EA50EC87FDF5
:10F3D00004C020E030E040EA50E4C301B2010E94E2
:10F3E00031EB2DEC3CEC4CEC5DE30E9478E40E94A8
:10F3F00010EC4B015C0180E2B7FE09C0B094A09410
:10F4000090948094811C911CA11CB11C8DE280936E
:10F41000960260E290E1891697E29906A104B10490
:10F420008CF0C501B40120E137E240E050E00E94D9
:10F43000BCEACA01B9012AE030E040E050E00E9495
:10F44000BCEA605D6093970260E2A8EE8A16A3E0D2
:10F450009A06A104B1048CF0C501B40128EE33E092
:10F4600040E050E00E94BCEACA01B9012AE030E065
:10F4700040E050E00E94BCEA605D60939802C501E4
:10F48000B40124E630E040E050E00E94BCEA6AE0CB
:10F49000462E512C612C712CCA01B901A301920195
:10F4A0000E94BCEA605D60939902C501B401A301AA
:10F4B00092010E94BCEA4B01CA01B901A301920169
:10F4C0000E94BCEA882009F44EC32EE220939A02DF
:10F4D000605D60939B02B0E38B0E80929C0266E9B4
:10F4E00072E08FE496E00E9455ED20E030E0A90143
:10F4F000C701B6010E9413E420E030E040E05FEB7A
:10F5000087FD04C020E030E040E05FE3C701B601C2
:10F510000E9431EB0E9410ECCB010E94DD41BC0146
:10F520008AE496E00E9455ED20E030E0A90169816F
:10F530007A818B819C810E9413E420E030E040E0DE
:10F540005FEB87FD04C020E030E040E05FE36981CD
:10F550007A818B819C810E9431EB0E9410ECCB015F
:10F560000E94DD41BC0185E496E00E9455ED80914A
:10F57000B71483FD0AC37ADE882309F409C3809196
:10F58000AF149091B014A091B114B091B21400973F
:10F59000A105B10509F4FCC2BC01CD016D597F4F35
:10F5A0008F4F9F4F24E630E040E050E00E9441EA58
:10F5B0006091B3147091B4148091B5149091B61405
:10F5C0000E9441EA29830E941C414B015C01162FD5
:10F5D00080915C01C9808C15C1F0C0925C0128E467
:10F5E000C29EB001112490E080E00E9417E42AE05E
:10F5F00037ED43E25CE30E9478E40E9415EC6093EF
:10F600004406C110C7C210923F0680915B011817D3
:10F6100009F43FC080925B01C501B40120E13EE0E6
:10F6200040E050E00E9441EA690189019CE3492ED3
:10F63000512C612C712CC501B401A30192010E94CF
:10F6400041EA4B015C01CA01B901A30192010E9488
:10F6500041EAC114D10409F0C4C29F928F927F93F2
:10F660006F9389E291E29F938F938FE296E09F934D
:10F670008F930E94ACE30FB6F894DEBF0FBECDBFF0
:10F6800085E0982F990F990F891B880F80588093D8
:10F690002E060E9400CB0091290610912A06209187
:10F6A0002B0630912C066B017C01C01AD10AE20AAC
:10F6B000F30A9701860137FD11C020912806209595
:10F6C000209328066A547C4F8F4F9F4F60932906E2
:10F6D00070932A0680932B0690932C06D0902806D0
:10F6E000D98281E00E942A6D80919913873180F43C
:10F6F00080919B13843060F08CE0E82E82E2F82E3B
:10F7000003E126E044E064E085E693E10E94F8CE60
:10F7100080915706982F927048E00CE081FD02C05E
:10F7200042E102E080919913843180F480919B132F
:10F73000841760F0992309F473C288EE91E27C018A
:10F7400023E060E585E693E10E94F8CE809199136D
:10F750008431C0F480919B138230A0F0C980CC200A
:10F7600009F461C28091A907882309F45CC28CEA7C
:10F7700091E27C0102E123E042E068E685E693E164
:10F780000E94F8CE809199138C3108F09DC0809032
:10F79000B0129090B112A090B212B090B312C0907B
:10F7A000B412D090B512843198F480919B138830B4
:10F7B00078F08091570680FF39C28EE591E27C0196
:10F7C0000CE022E048E069E385E693E10E94F8CE90
:10F7D00080919913883040F4D7FE2BC242E451E265
:10F7E00067E087E30E943172809199138C31B0F405
:10F7F00080919B13843190F020E030E040E05FE3A3
:10F80000C501B4010E9431EB0E9410EC77FF34C2B5
:10F8100042E451E26CE187E30E943172C0902F070D
:10F82000D0903007E0903107F09032078091991323
:10F83000883060F4809133079091340797FF3FC27E
:10F8400042E451E267E081E50E94317280919913B0
:10F850008C31B0F480919B13843190F020E030E043
:10F8600040E05FE3C701B6010E9431EB0E9410EC5B
:10F8700077FF47C242E451E26CE181E50E943172B8
:10F88000809199138C3100F580919B138431E0F0C5
:10F890008091A9078823C1F024E6829FC00111242A
:10F8A00081589F4F6FEF70E00E94A9EACB010E9440
:10F8B0005C42AC016CE187E60E948A7365E270E00D
:10F8C00080E090E00E943B6DD1DC882379F180914B
:10F8D0009913843358F580919B138A3238F107E0ED
:10F8E00028E04AE26AE285E693E10E949FCD05E0C6
:10F8F00022E04CE262E385E693E10E949FCD24E0A2
:10F900004AE061E38AE20E946FCD609167137091D3
:10F91000681382E3809381138BE28093821321E842
:10F9200033E142E385E693E10E946FCC8091991325
:10F93000853350F480919B13813330F024E04AE406
:10F9400061E386E30E946FCD80919913843368F45C
:10F9500080919B13823348F002E02091440642E3F9
:10F9600067E385E693E10E949FCD809199138033F0
:10F97000D8F480919B138832B8F080913F06882399
:10F9800061F04FE356E060E387E30E948A7365E22B
:10F9900070E080E090E00E943B6D4FE256E060E353
:10F9A00080912E060E948A7380919913883208F004
:10F9B00060C080919B138D3108F45BC02BE040E860
:10F9C0006DE180E00E946FCD80919913873208F03D
:10F9D00050C080919B138F3108F44BC083E080931B
:10F9E0009C1316E210939D1368E570E080E090E0B0
:10F9F0000E943B6D8BE080939C1310939D13C980F4
:10FA0000CC2009F4A1C18AE496E00E94827288E2C7
:10FA100080939C1316E210939D1369E570E080E0DB
:10FA200090E00E943B6D80E380939C1310939D13A4
:10FA3000C980CC2009F4ABC185E496E00E948272B3
:10FA40008DE480939C1316E210939D136AE570E099
:10FA500080E090E00E943B6D85E580939C131093BD
:10FA60009D13C980CC2009F4B5C18FE496E00E94B3
:10FA7000827280919913833338F580919B138B3276
:10FA800018F183E00E942A6D83E080939C1383E346
:10FA900080939D1366E070E080E090E00E943B6DF3
:10FAA00081E00E942A6D80911001909111010E94C5
:10FAB0005C42AC0163E38CE00E948A7365E270E013
:10FAC00080E090E00E943B6D80919913813408F0B2
:10FAD000F1CB80919B13863308F4ECCB10929C13EE
:10FAE0008EE380939D1381E490E10E944466182F79
:10FAF000863108F092C181E490E10E948272153152
:10FB000009F4D8CB60E270E080E090E00E943B6DA9
:10FB10001F5FF5CF243631054CF48536910504F589
:10FB20008A30910534F48AE090E009C0843691056A
:10FB3000BCF0883EA3E09A0714F087EE93E0281704
:10FB4000390709F4D9CB90931101809310011092D9
:10FB5000690710926A0710926B0710926C07CCCB62
:10FB600084E690E0F0CF662351F02EE220939A02D3
:10FB7000605D60939B0280E280939C02B0CC80E247
:10FB800080939B0280939A02F6CFE4E6E9831BCD33
:10FB9000198219CD498180E2443628F0842F64E629
:10FBA0000E947CEA805D80939A02698190E26A30CB
:10FBB00040F02AE0862F622F0E947CEA0E947CEAB5
:10FBC000905D90939B0289816AE00E947CEA905D3F
:10FBD00090939C026AE972E08FE396E00E9455EDF3
:10FBE00014CD0436110538F47F936F93DF92CF92D2
:10FBF0008DE191E238CD7F936F93DF92CF9283E1D5
:10FC000091E29F938F938FE296E09F938F930E9450
:10FC1000ACE30FB6F894DEBF0FBECDBF86E031CDAA
:10FC200082EE91E28CCD86E791E2A3CD86E491E26B
:10FC3000C6CDC6010E945C42FC01808193E0803207
:10FC400029F4818192E0803209F491E043E050E0B0
:10FC5000491B51094E0F5F1F892F880F880F981B72
:10FC6000892F67E0805C0E948A7369E070E080E021
:10FC700090E00E943B6DB8CDCB010E945C42FC013C
:10FC8000808193E0803229F4818192E0803209F40E
:10FC900091E043E050E0491B51094E0F5F1F892F4F
:10FCA000880F880F981B892F6CE1805C0E948A73F3
:10FCB00069E070E080E090E00E943B6DAFCD0E9473
:10FCC0005C42FC01808193E0803229F4818192E0E2
:10FCD000803209F491E043E050E0491B51094E0F96
:10FCE0005F1F892F880F880F981B892F67E0865A1E
:10FCF0000E948A7369E070E080E090E00E943B6DB2
:10FD0000A5CDCB010E945C42FC01808193E0803252
:10FD100029F4818192E0803209F491E043E050E0DF
:10FD2000491B51094E0F5F1F892F880F880F981BA1
:10FD3000892F6CE1865A0E948A7369E070E080E046
:10FD400090E00E943B6D9CCD87E00E94ED3980FFE2
:10FD500013C00AE416E0D8016D918D01662309F401
:10FD600056CE6F320CF06FE3062E000C770B880B2B
:10FD7000990B0E943B6DEFCF8091770780FD43CEBA
:10FD80006FEF7FEF8DE391E20E942D7140CE87E00F
:10FD90000E94ED3981FF13C005E416E0D8016D9192
:10FDA0008D01662309F44CCE6F320CF06FE3062E02
:10FDB000000C770B880B990B0E943B6DEFCF809165
:10FDC000770781FD39CE6FEF7FEF8DE391E20E94DF
:10FDD0002D7136CE87E00E94ED3982FF13C00FE40B
:10FDE00016E0D8016D918D01662309F442CE6F3281
:10FDF0000CF06FE3062E000C770B880B990B0E941A
:10FE00003B6DEFCF8091770782FD2FCE6FEF7FEFB5
:10FE100085E391E20E942D712CCE81E0C980C11052
:10FE200001C080E090912D068917C9F0D090401054
:10FE3000D98280932D0681E490E10E944466D81611
:10FE400008F054C029812F5F2983E22FF0E0EF5B97
:10FE5000FF4E8081807C8038A9F320934010009170
:10FE6000401010E00F5B1F4EC8010E94446689835A
:10FE700060E870E0C8010E9439724981453108F09C
:10FE800019CA60E270E080E090E00E943B6D6981F9
:10FE9000643109F40FCA60E270E080E090E00E94F3
:10FEA0003B6D8981833109F405CA60E270E080E02E
:10FEB00090E00E943B6D9981923109F4FBC9292F92
:10FEC00030E02E5F3F4F4AEF4203B001439F700D79
:10FED000112460587F4F81E490E10E94397260E202
:10FEE00070E080E090E00E943B6DE4C91092401009
:10FEF000B6CF80918707823059F0B8D9882349F06E
:10FF00008091B71482FB882780F991E089270895B2
:10FF100081E0089581E008959091C00095FFFCCFA5
:10FF20008093C6000895CF93DF93EC0189918823D5
:10FF300011F0F2DFFBCFDF91CF910895CF93DF93E4
:10FF4000EC018991882311F0E7DFFBCF8DE0E4DF3E
:10FF50008AE0E2DFDF91CF910895CF93DF93EC0148
:10FF6000FE0184912196882311F0D6DFF9CFDF912D
:10FF7000CF9108950F931F93CF938C01C62F87E8DD
:10FF80009EE1EBDFC801E9DF8AE3C6DF80E38C0F87
:10FF9000C3DF8AE0C1DFCF911F910F910895CF9207
:10FFA000DF92EF92FF926A017B01D7DF42E0C70147
:10FFB000B6010E94F5AFFF90EF90DF90CF900895CB
:10FFC000EEDF8AE0A9CFADE5B0E0E9EEFFE70C9403
:10FFD000F9EA70E060E085E40E944F6B7C01182F25
:10FFE0008F3FB1F1882341F081E890E2B6DFC35A38
:10FFF000DF4FE2E10C9415EB6EEB70E083E50E94BD
:020000021000EC
:100000004F6B5C0165E070E083E40E944F6B6C0114
:1000100060E085E50E943B6B2C968FAF2C9760E0EB
:1000200084E790E20E9457580E9400CB69877A8744
:100030008B879C871F3F09F067C434E7A316B10480
:100040000CF489C189E490E288DF0E9478C1CFCFA7
:100050006CE370E0D3CF20E030E040E05EE32BAF14
:100060003CAF4DAF5EAFABC12AE939E949E15FE38F
:1000700023962CAF3DAF4EAF5FAF2397ADC14090FD
:10008000B0125090B1126090B2127090B31251C27F
:100090002B96EEADFFAD2B974083A4C24BEEC42E42
:1000A000D12CE12CF12C22C384E190E0A0E0B0E05F
:1000B0008D879E87AF87B88B34E1C32ED12CE12C7E
:1000C000F12C24C3CD86DE86EF86F88A1FC32B96DB
:1000D000EEADFFAD2B978083E9C3D501C4012EA5FA
:1000E0003FA548A959A9821B930BA40BB50BB7FDDB
:1000F00047C02D968FAD2D970E944F268AE00CDFCA
:10010000D501C4018053984FAF4FBF4F8EA79FA713
:10011000A8ABB9AB9AA991116FC02BA93CA94DA965
:100120005EA9C301B2010E9494EC18160CF050C0F5
:1001300020E030E040E050E4C301B2010E9431EB26
:100140006BAB7CAB8DAB9EAB2AA53BA54CA55DA54F
:10015000280D391D4A1D5B1D2FAB38AF49AF5AAF73
:100160006D966CAD7DAD8EAD9FAD6D970E9419E41F
:10017000A30192010E9413E4881F8827881F8AAB7D
:1001800089859A85AB85BC85898F9A8FAB8FBC8F0B
:1001900029893A894B895C89281739074A075B07FF
:1001A00020F4298F3A8F4B8F5C8F898D9A8DAB8D80
:1001B000BC8D881A990AAA0ABB0A91E889169FE49D
:1001C000990692E1A906B10460F18DE69FE12DC286
:1001D000D501C4012FA938AD49AD5AAD821B930B8F
:1001E000A40BB50B49ED52E168EE72E1B7FDC8CF43
:1001F000812F0E949627C4CF69966CAD7DAD8EADE0
:100200009FAD69970E9419E49B01AC01C301B20143
:100210000E9413E487FFB4CF46E153E166E273E145
:10022000E7CF2996AEADBFAD2997A215B3050CF067
:100230008FC0B3E02B1631040CF48AC080E19FE13B
:100240008CDE1F3F09F066C0E0E0FFE1FE83ED8336
:100250008FEE9EE182DE8D819E817FDE49815A8113
:100260006B817C818CE09FE1ABDE8FEE9EE175DEE1
:100270008D819E8172DE4D8D5E8D6F8D78A188E0BF
:100280009FE19EDE8FEE9EE168DE8D819E8165DEC0
:1002900049A15AA16BA17CA184E09FE191DE2C963B
:1002A0003FAD2C97332309F4D0CE2CEA35EC47E24E
:1002B0005EE36D8D7E8D8F8D98A10E9478E46B0139
:1002C0007C0120E030E543EC50E469A17AA18BA1E8
:1002D0009CA10E9478E429813A814B815C811F3F77
:1002E000F1F4209336073093370740933807509343
:1002F0003907C0923A07D0923B07E0923C07F09250
:100300003D0760933E0770933F07809340079093AB
:1003100041079BCE2FEE3BE23E832D8399CF209366
:10032000B7123093B8124093B9125093BA12C092D8
:10033000BB12D092BC12E092BD12F092BE1260933A
:10034000BF127093C0128093C1129093C2127DCEDF
:100350000E94956ECEC085E390E2FFDD0E94F826F4
:100360008FE7809335072CE330E0C9A6A8EEB3E011
:100370000E946DEA6AA77BA78CA79DA729853A856D
:100380004B855C85260F371F481F591F2FAB38AF91
:1003900049AF5AAF81E08093690160E081E290E269
:1003A0000E94575802E00E0D023008F054CE8BEA3E
:1003B0009AEAAAEABEE38BAF9CAFADAFBEAF023004
:1003C00008F052CE8DEC9CECACE4BEE323968CAFEF
:1003D0009DAFAEAFBFAF2397023008F4E12C2D964E
:1003E000EFAE2D9789859A85AB85BC85898B9A8BD5
:1003F000AB8BBC8B8EA79FA7A8ABB9AB19A21AA2D7
:100400001BA21CA21D8E1E8E1F8E18A219821A827C
:100410001B821C822FE730E040E050E02D873E87B2
:100420004F87588B80E090E4ACE1B6E48D839E83E7
:10043000AF83B8871D8A1E8A1F8A188EFFE7CF2ECA
:10044000D12CE12CF12C1AAA1BAA1CAA1DAA1EAAA7
:100450001DA21EA21FA218A691E024969FAF24976A
:10046000312C212C412C512C320195010B2C000CEC
:10047000440B550B61962CAF3DAF4EAF5FAF61970C
:1004800049A5042E000C550B29965FAF4EAF299756
:1004900057E11502C0011124DC01AA54BD4E2B9670
:1004A000BFAFAEAF2B97C5014E969C01092E000C35
:1004B000440B550B65962CAF3DAF4EAF5FAF6597C4
:1004C000CC979C01990F440B550B69962CAF3DAF0F
:1004D0004EAF5FAF699736E0A31AB108C5010B2C88
:1004E000000CAA0BBB0B6D968CAF9DAFAEAFBFAF30
:1004F0006D9780916901882309F498C00E9400CB10
:100500004B015C01909198036E969FAF6E97992373
:1005100009F47BC00E948C28109298031F3F09F0B9
:10052000AECD40902F07509030076090310770900B
:100530003207A30192016D897E898F89988D0E946F
:1005400094EC87FF04C04D8A5E8A6F8A788EA3017F
:1005500092016D817E818F8198850E9413E4181627
:1005600024F44D825E826F82788661966CAD7DAD9B
:100570008EAD9FAD61970E9419E4698F7A8F8B8F42
:100580009C8F2496AFAD2497AA2309F454C09B01F5
:10059000AC01C301B2010E9494EC1816B4F5D50168
:1005A000C40129893A894B895C89821B930BA40B6E
:1005B000B50BAC01BD01485853416109710977FD84
:1005C00024C04D855E856F8578894C195D096E095B
:1005D0007F0975956795579547951F3F09F058CD49
:1005E000409335078DA39EA3AFA3B8A7298D3A8D5D
:1005F0004B8D5C8D2D8B3E8B4F8B588F89869A86C9
:10060000AB86BC8624961FAE249765966CAD7DADF7
:100610008EAD9FAD65970E9419E4A30192010E94DF
:1006200013E487FF5ACD8BE89FE197DC10926901B4
:100630000E94F8260ACD298D3A8D4B8D5C8DC30121
:10064000B2010E9413E487FFE0CFD501C4012985E0
:100650003A854B855C85821B930BA40BB50BAC01D3
:10066000BD01485853416109710977FDCECF21146E
:10067000310409F40AC12DA13EA14FA158A5280FAC
:10068000391F4A1F5B1F298B3A8B4B8B5C8B2DA12B
:100690003EA14FA158A5281B390B4A0B5B0BC70184
:1006A000B6010E9432EA29893A894B895C890E9405
:1006B000BCEACD84DE84EF84F888C20ED31EE41E2B
:1006C000F51E34E1C316D104E104F1040CF4ECCCC2
:1006D0004CEEC416D104E104F1040CF0DFCC50E878
:1006E000C516D104E104F1040CF4ECCCCD86DE8611
:1006F000EF86F88A8EEF90E0A0E0B0E09C01AD01BB
:100700002C193D094E095F0969017A0189E190E2DE
:1007100024DC6D857E858F8598890E94907384E1A5
:1007200090E21BDCC701B6010E9490734D815E818F
:100730006F8178858DE090E232DC4D895E896F892A
:10074000788D86E090E22BDC93E0291631040CF4DE
:100750009CC0C701B6010E9419E420E030E040E8E7
:1007600050E40E9478E469837A838B839C832D8193
:100770003E814F8158856D897E898F89988D0E9431
:1007800030EB2BED3FE049EC5FE30E9478E49B0106
:10079000AC0169817A818B819C810E94A8EB2796AC
:1007A0006CAF7DAF8EAF9FAF279769897A898B89B0
:1007B0009C890E9419E42FE632E143E85AE30E9443
:1007C00078E46D837E838F83988723962CAD3DAD2F
:1007D0004EAD5FAD239727966CAD7DAD8EAD9FADD1
:1007E00027970E9478E469837A838B839C839B019B
:1007F000AC010E9431EB2D813E814F8158850E94D2
:10080000A8EB6D8F7E8F8F8F98A32BAD3CAD4DAD38
:100810005EAD6D817E818F8198850E9478E429810B
:100820003A814B815C810E9478E469A37AA38BA30F
:100830009CA327964CAD5DAD6EAD7FAD279780E054
:1008400090E2ADDB4D815E816F8178858AEF9FE11B
:10085000B7DB8BEE9FE1023010F08CED9FE17DDB8A
:1008600049815A816B817C8186ED9FE198DB4D8DBA
:100870005E8D6F8D78A180ED9FE191DB49A15AA13A
:100880006BA17CA18AEC9FE19BDB8D859E85AF856A
:10089000B8898C0D9D1DAE1DBF1DB595A79597956B
:1008A00087951F3F09F013CC809335072996FFAD3C
:1008B0002997FF9329A52F933F922F9286EB9FE1D3
:1008C0009F938F9381EC9FE19F938F931F920E9440
:1008D0003A583FEF231A330A0FB6F894DEBF0FBE23
:1008E000CDBF898D9A8DAB8DBC8D8D839E83AF835B
:1008F000B887898A9A8AAB8ABC8A6E969FAD6E97B2
:1009000024969FAF249781CE8E2C0E2C000C990834
:10091000F40183E0EE0FFF1F8A95E1F7EF59FE4FD8
:10092000868197810F978A159B050CF48BCB85E305
:1009300090E213DB0E94F82687E1889DF001899DF3
:10094000F00D1124E455FD4E8FE7828724E130E05D
:100950000CCDCF93DF9361E078E10E9442C1CBE2FE
:10096000D7E04B855C856D857E8588EF97E117DB49
:1009700020E030E543EC50E46F85788989899A89D5
:100980000E9478E4AB01BC0185EF97E108DB2CEA1B
:1009900035EC47E25EE36B897C898D899E890E94F4
:1009A00078E4AB01BC0182EF97E10ADBDF91CF91E4
:1009B000089563E877E10E9442C160917B0D7091D8
:1009C0007C0D80917D0D90917E0D0E9417E4AB010E
:1009D000BC018AE797E1E3DA4091AB0D5091AC0D91
:1009E0006091AD0D7091AE0D87E797E1D8DA409137
:1009F000AF0D5091B00D6091B10D7091B20D84E7C3
:100A000097E1CDDA40918D0750918E0760918F0765
:100A10007091900781E797E1D3CACF93DF9367E2A4
:100A200077E10E9442C1CBE6DDE04CA95DA96EA949
:100A30007FA98EE197E1B3DA48AD59AD6AAD7BADE0
:100A40008BE197E1ACDA4CAD5DAD6EAD7FAD84E787
:100A500097E1B6DADF91CF910895CF93DF9363E00A
:100A600077E10E9442C1CBE6DDE04CA15DA16EA121
:100A70007FA18AEF96E193DA48A559A56AA57BA5DF
:100A80008FE99CE28CDA4CA55DA56EA57FA58CE96B
:100A90009CE285DA48A959A96AA97BA989E99CE25F
:100AA0008FDADF91CF910895CF93DF936EED76E1EA
:100AB0000E9442C1CBE6DDE0688179818A819B8119
:100AC0000E9417E4AB01BC0185ED96E168DA6C8108
:100AD0007D818E819F810E9417E4AB01BC018FE96B
:100AE0009CE25DDA688579858A859B850E9417E49A
:100AF000AB01BC018CE99CE252DA6C857D858E8568
:100B00009F850E9417E4AB01BC0189E99CE258DA99
:100B1000DF91CF9108958F929F92AF92BF92EF9203
:100B2000FF920F931F93CF93DF9388EB95E115DA34
:100B3000C0E0D7E0D15019F080E2EED9FBCF8C2F86
:100B40000E94EB6ACF5FC730A1F78AE0E5D903EBDB
:100B500012E0C0E080E2E0D98C2F0E94EB6A7801BD
:100B6000D7E080E2D9D9F70180809180A280B3805C
:100B700020E030E0A901C501B4010E9494EC87FD9A
:100B800002C08BE2C9D943E0C501B4010E94F5AFB0
:100B9000D150FCE1EF0EF11CD111E3CF8AE0BCD9BA
:100BA000CF5F0C5F1F4FC730A9F68AE0B5D9DF9140
:100BB000CF911F910F91FF90EF90BF90AF909F90BA
:100BC0008F900895811105C081EB95E1C6D98AE027
:100BD000A3C985EB95E1FACF8AEA95E1BEC984EA1B
:100BE00095E1BBC9CF9384E50E949F67C0E088234D
:100BF000D9F00E94116BC82F1816B4F4F0DF8DE401
:100C00008BD980911D0690911E060E941E7987E265
:100C100098E1A3D96C2FCC0F770B880B990B0E940E
:100C2000ABAD8AE079D9CFEF8C2FCF910895CF93D8
:100C3000C82F67EE77E10E942BC1C11101C0CFDF41
:100C40004091B7125091B8126091B9127091BA12D6
:100C50008EED97E1A4D920E030E543EC50E46091BB
:100C6000BB127091BC128091BD129091BE120E9475
:100C700078E4AB01BC018BED97E191D92CEA35EC1E
:100C800047E25EE36091BF127091C0128091C11281
:100C90009091C2120E9478E4AB01BC0188ED97E10B
:100CA0007ED98AE039D9CF910895ACE1B0E0EBE587
:100CB000F6E80C94F9EA83E50E942867182F882348
:100CC00009F41CC10E942C6B8D8380917501909159
:100CD0007601A0917701B0917801898F9A8FAB8FBF
:100CE000BC8F2091790130917A0140917B01509124
:100CF0007C012D8B3E8B4F8B588F80917D01909185
:100D00007E01A0917F01B09180018D879E87AF8782
:100D1000B88B112331F09D81911103C080E00E94B6
:100D200043778091170690911806A0911906B0910B
:100D30001A0635E1B695A795979587953A95D1F717
:100D40009C01AD01217033274427552729873A8715
:100D50004B875C8720E030E0A90160917F037091B0
:100D6000800380918103909182030E9413E4882381
:100D700009F4C8C083E40E942867882309F493C05B
:100D80000E945B6B698B7A8B8B8B9C8B43EB52E065
:100D90005F834E838A0157E05887412C512C98EC91
:100DA000692E92EC792E812C912C28ECA22E22E433
:100DB000B22E312C212CF101EE0FFF1FEE0FFF1F81
:100DC000E00FF11FC080D180E280F380A70196017F
:100DD000C501B4010E9413E4181614F4460157012A
:100DE000A7019601C301B2010E9494EC87FF02C0E3
:100DF000260137018FEF281A380A97E029163104A7
:100E0000D1F6A885A150A887045E1F4FA111D1CFAC
:100E1000A3019201C501B4010E9431EB20E030E052
:100E200040E05FE30E9478E429893A894B895C8934
:100E30000E9431EB4B015C012DEB37E346E855EBAB
:100E40000E9413E487FD0AC02DEB37E346E855E323
:100E5000C501B4010E9494EC18162CF580E00E94A4
:100E6000437717E0EE80FF8007E0F7016191719111
:100E7000819191917F016F01F4E0CF1AD108A50112
:100E800094010E9430EBD6016D937D938D939C93DA
:100E90001397015051F71150EE81FF817C96FF832B
:100EA000EE831111DFCF89859A85AB85BC85892BAF
:100EB0008A2B8B2B79F020E030E0A90160917F0331
:100EC0007091800380918103909182030E9413E4CA
:100ED000811121DE8AE50E942867882359F00E944B
:100EE0005B6B69837A838B839C8360E0CE01019680
:100EF0000E94CF778D810E94437713C02091AE026C
:100F00002D83E3CEFD81F11108C029853A854B85FB
:100F10005C85232B242B252BE9F261DE80E196E111
:100F20001CD89D81992341F08091AE02811104C0AB
:100F300053DE81EF95E111D852DE83EE95E10DD8B5
:100F40008091AE023FDE4BDE86ED95E106D8C09083
:100F5000AF02D090B002E090B102F090B20220E077
:100F600030E0A901C701B6010E9494EC18160CF0FC
:100F700040C042E0C701B6010E94F5AF8DE00E947B
:100F80008C7F8AE00E948C7F298D3A8D4B8D5C8D01
:100F9000609175017091760180917701909178014F
:100FA0000E9413E481111FC02D893E894F89588DFD
:100FB0006091790170917A0180917B0190917C011F
:100FC0000E9413E481110FC020917D0130917E01B8
:100FD00040917F01509180016D857E858F85988934
:100FE0000E9413E481110E94EA3E6C96E2E10C94A7
:100FF00015EB81ED95E10E94AD7FC6CFCF93DF93D6
:10100000EB010E94AD7FBE01DD0F880B990B0E94A2
:10101000ABADDF91CF9108950E94AD7F8AE00C9433
:101020008C7FCF93DF936EE97EE10E9442C1C09135
:101030003413D0913513488159816A817B8185E9C8
:101040009EE10E94CF7F4C815D816E817F818FE91F
:101050009CE20E94CF7F40913013509131136091F8
:101060003213709133138CE99CE20E94CF7F82E9A6
:101070009EE10E94AD7F8CE89EE1CEDFDF91CF91B3
:101080000895EC018B01F42E0E94F826209709F4B4
:1010900076C0A5DDCE01C0DF0115110511F40FEEFC
:1010A0001BE20E94CC6B1F930F93DF93CF9384E7D7
:1010B00095E19F938F9381E08F930E943A580E940D
:1010C000D544C0916613C695C69581E693E10E940A
:1010D000626EDC2FDD0F1D2F1C0F8DB79EB707969C
:1010E0000FB6F8949EBF0FBE8DBF83E00E942A6D9D
:1010F00041E450E16C2F80E00E948A7310929C13AF
:10110000D0939D136FEF7FEF85E695E10E942D71DF
:1011100010929C1310939D136FEF7FEF88E595E17C
:101120000E942D7185E693E10E94F2CD8111DDCF01
:1011300053DD84E895E10E94AD7F89EE93E001974D
:1011400039F000C00000EEE5F9E03197F0F7F7CF95
:10115000F89489EE93E0019739F000C00000E6EEC4
:10116000F3E03197F0F7F7CF0E94F826FF2021F047
:101170000E94292BA895FECF0E94E42AFBCF0115DF
:10118000110511F40FEE1BE2CBE7D5E18ACF809178
:10119000B50D9091B60D2FEF3FEF981751F0E92F55
:1011A000F0E0EB54F24F228130E09F5F9F77909305
:1011B000B60DC90108951F920F920FB60F92112418
:1011C0000F900FBE0F901F9018951F920F920FB6A1
:1011D0000F9211240BB60F922F938F939F93EF933F
:1011E000FF939091C6002091B60DE091B50D81E07E
:1011F0008E0F8F77281729F0F0E0EB54F24F92838F
:10120000E82FE093B50DFF91EF919F918F912F9172
:101210000F900BBE0F900FBE0F901F9018958EBDB4
:101220000DB407FEFDCF08958FEF8EBD0DB407FE00
:10123000FDCF8EB50895909164009B7F90936400DC
:10124000982F906A96959CBD80FD03C091E08630F2
:1012500009F490E09DBD0895A8E0B0E0E2E3F9E86C
:101260000C94F9EAB82E80919E0E843008F0F6C1F5
:1012700031E6D32E80919E0E843008F021C18091FA
:10128000B50D9091B60D891B8F7709F419C17FDFD9
:1012900097FF0AC0A1DC84EA94E10E94AD7F8091AF
:1012A000B50D8093B60DE6CF8A3019F08D3009F078
:1012B000FEC010929D0E80913B0E90913C0EFC0161
:1012C000E95CF14F1682892B19F40E94F328D2CFE2
:1012D00010923C0E10923B0E0DE31EE0F80181913E
:1012E000803209F446C08E3409F09DC06FE974E184
:1012F000C8010E9492E37C01892B41F06EE470E00A
:10130000C80104960E944AED009709F4C8014AE01A
:1013100050E070E060E001960E9407E12B013C0183
:101320008091370E9091380EA091390EB0913A0EFF
:101330000196A11DB11D481659066A067B0629F0C3
:1013400060E08CE694E1EF2851F16AE270E0C801B8
:101350000E9479ED9C01009729F1982F901BF12CA8
:10136000992349F09150F801E90FF11D8081F82689
:10137000F7CF8F01B3CF4AE050E070E060E0C901E1
:1013800001960E9407E12F2D30E050E040E0621707
:1013900073078407950751F060E08DE494E10E94A3
:1013A00095C068CF60E083E294E1F9CF4092370EB8
:1013B0005092380E6092390E70923A0E8091260744
:1013C0008130E1F467E470E0C8010E944AED0097C3
:1013D000A9F04AE050E070E060E001960E9407E169
:1013E000623071058105910548F482E893E10E941D
:1013F000AD7F60E088E793E10E945758F801808153
:101400008D3481F58381823309F445C0883301F13D
:10141000803341F58181843329F58281813311F54F
:101420000E94C63E1FC08091B71480FFC7CF64E9F9
:101430007BE2C8010E9492E3009731F0FC018381B6
:1014400080538A3008F0BACF60E089EF93E1A7CFEC
:101450008281803339F48181813321F410926901D2
:1014600010928B0780913D0E8B3309F403CF80914E
:101470009E0E843008F0FECE8091A00E8D9DC0019E
:1014800011246DE37EE08F55914F0E9455ED80E071
:101490000E9455C0EFCE8281813321F78181813353
:1014A00009F741E070E060E08CEA99E1EADD2BE3C6
:1014B0003EE04DE35EE06DE97EE00E94AA66DACE92
:1014C0008091B71483FDCAC082FFC8C087FDC6C023
:1014D0001A82198281E6F82E94E0E92E29E6D22EAE
:1014E00080919E0E843008F0B9C00E94E26681119E
:1014F000B5C041E050E0BE016D5F7F4F85EC92E1E9
:101500000E9405D40B8110E0019711F00FEF1FEF3F
:101510008091CD129091CE12A091CF12B091D012A5
:101520008093B3149093B414A093B514B093B614ED
:101530000E94E2660F3F100741F4811106C04CDBA8
:101540008CEB94E10E94AD7FCBCF4091A00E242F75
:1015500030E00A3061F00D3051F0882309F470C09A
:1015600089819A81009719F001969A838983109254
:10157000AA0589819A81F29EF001F39EF00D112453
:10158000E256F14FDF01A80FB91F13961C92892B69
:10159000A9F50E94F3280E94E266882309F4A0CFEF
:1015A00085EC92E10E9491228091AE148823F1F1A2
:1015B00081508093AE148D9DC001112462E0845946
:1015C000994F0E940CD6E091AE1424E0E29FF00106
:1015D0001124E859F94F4081518162817381409310
:1015E000B3145093B4146093B5147093B61485EC8F
:1015F00092E10E940AD30E944DCF72CF1A821982C3
:1016000083818D3479F48481823361F485818533DB
:1016100049F4868180538A3028F08091B7148B7FFB
:101620008093B71481E00E9455C0B5CF0E943FCF90
:101630008091B71488608093B714E092260750CF4A
:101640004F9DA00111244F55514F9E012F5F3F4FD9
:101650006AEA75E0802F0E94AA6642CF0E9400CB02
:101660006B017C01BB2041F0C0922006D092210684
:10167000E0922206F09223068091F8059091F905F8
:10168000A091FA05B091FB050097A105B10529F1DC
:101690004091200650912106609122067091230608
:1016A000840F951FA61FB71FA7019601281B390B92
:1016B0004A0B5B0BDA01C901B7FD0FC08DDA6091EF
:1016C000890770918A078BEC94E10E9431CF40E04A
:1016D00070E060E090E080E0E9CE80914F01909171
:1016E0005001A0915101B0915201892B8A2B8B2B73
:1016F00079F09091391380913A13981709F4C4C086
:10170000C0922006D0922106E0922206F092230693
:101710008091AF059091B005A091B105B091B2054F
:1017200046015701881A990AAA0ABB0AD501C401C1
:10173000B7FDC0C19091391380913A1320913E01B9
:10174000981709F4D5C0E0913A133BE5E39FF00107
:101750001124E05FF74F8081281799F080933E01B4
:101760000E9400CBB0903E010B2D10E084E00E945F
:10177000D6AF0115110509F0BEC060E084E00E94FB
:1017800018CA80919703882309F487C10091060144
:1017900010910701C80102972091B4123091B5123F
:1017A000281739070CF479C180903A138C82812C68
:1017B000912C5401809139132C81821709F4FDC0BA
:1017C000822F90E03BE5389FF001399FF00D112406
:1017D000E654F84F458956896789708D452B462B0D
:1017E000472B81F4418D528D638D748D452B462B93
:1017F000472B41F4458D568D678D70A1452B462BA7
:10180000472BE9F14BE5489F9001499F300D11248A
:10181000C9018654984F1C01FC016181728183814A
:1018200094810E94CDEC6D837E838F839887F10134
:1018300061A172A183A194A10E9417E42B013C0134
:10184000F10165A176A187A190A50E9417E49B01F3
:10185000AC01C301B2010E94A8EB2D813E814F81F2
:1018600058850E9478E42B013C01AC019B01C50125
:10187000B4010E9494EC87FF02C0530142018C81A5
:101880008F5F8F708C8396CFBB2019F01092B305B9
:101890003FCF0E9400CB009120061091210620919D
:1018A00022063091230680904F0190905001A09025
:1018B0005101B0905201080D191D2A1D3B1D601BDE
:1018C000710B820B930B97FDE1CF8091B3058111D2
:1018D0001FCF81E08093B30580E00E94F92A81E068
:1018E0000E94F92A82E00E94F92A0E94E42A10CF7D
:1018F0008091A90731CF0F3F110511F461E03ECF70
:10190000E3EDFBE2E491E150EA3008F051C0F0E091
:10191000E457F3470C94D8EA968C9B8CA08CAA8C45
:10192000D88CD88CB48CBC8CC48CCE8C84B580689C
:1019300084BDB7BC26CF84B5806284BDB8BC21CF3E
:1019400080918000806880938000109389000093CC
:10195000880017CF80918000806280938000109370
:101960008B0000938A000DCF8091B0008068809337
:10197000B000B092B30005CF8091B0008062809338
:10198000B000B092B400FDCE80919000806880934A
:1019900090001093990000939800F3CE80919000EE
:1019A00080628093900010939B0000939A00E9CE90
:1019B000003811050CF0A2CFE0CEB801110F880B52
:1019C000990B0E9419E42B013C01209100013091F8
:1019D00001014091020150910301C501B4010E942F
:1019E00078E4A30192010E9431EB4B015C0100916C
:1019F000040110910501AC019B01C301B2010E94D9
:101A000094EC18168CF0B801012E000C880B990B81
:101A10000E9419E42B013C01A50194010E9413E4EA
:101A2000181614F4240135018090AB059090AC0594
:101A3000A090AD05B090AE05A3019201C501B4011F
:101A40000E9494EC1816D4F420E037ED43EA5CE3EE
:101A5000C301B2010E9478E42B013C0128E431EE7D
:101A60004AE75FE3C501B4010E9478E49B01AC0141
:101A7000C301B2010E9431EB2B013C014092AB0546
:101A80005092AC056092AD057092AE05C301B201F3
:101A90000E9410ECCB010E9441CBF4E6CF0ED11C8A
:101AA000E11CF11CC092AF05D092B005E092B105E7
:101AB000F092B2050E94F32880912607882309F44A
:101AC000D2C010913F01113061F18091B714806450
:101AD0008093B71481E080933F0164EF71E080E070
:101AE00090E00E94F9780E943CD88091B71484FF5E
:101AF000D2C0123028F460E088E095E10E94575887
:101B000083E080936A010E9400CB6C597F4F8F4F16
:101B10009F4F60936306709364068093650690936D
:101B200066060E9400CB6B017C0110914E011123CF
:101B3000F1F080918C078823D1F04091B405509149
:101B4000B5056091B6057091B70546015701841A35
:101B5000950AA60AB70AB501A40177FD1AC0833019
:101B600009F494C00CF083C081300CF088C0212FA0
:101B700030E0A8EEB3E00E946DEAC60ED71EE81E64
:101B8000F91EC092B405D092B505E092B605F09268
:101B9000B7050E94FD420E94956E8091F70588234B
:101BA00079F10E9400CB6B017C018091F30590914B
:101BB000F405A091F505B091F605A7019601281B43
:101BC000390B4A0B5B0BDA01C901B7FD19C0209133
:101BD000F70530E0A8EEB3E00E946DEAC60ED71E0E
:101BE000E81EF91EC092F305D092F405E092F505C7
:101BF000F092F60580E00E944F268AE00E948C7FDA
:101C00008091F205882379F10E9400CB6B017C0161
